:100000000C94342E0C94B12E0C94B12E0C94B12E71
:100010000C94B12E0C94B12E0C94B12E0C94B12EE4
:100020000C94B12E0C94B12E0C94B12E0C94B12ED4
:100030000C94B12E0C946B300C94AB300C94B12E0C
:100040000C94B12E0C94B12E0C94B12E0C94B12EB4
:100050000C94B12E0C94B12E0C94B12E0C94B12EA4
:100060000C94B12E0C94B12E0C94B12E0C94B12E94
:1000700067548054A954B754C954DF5412552F55AE
:100080005A5501200101003808000000000000005E
:100090000000000000000000000000000000000060
:1000A0008100450027FF24FF2A902B1C210C22FBF6
:1000B000850084008903888D81096F0244424700CE
:1000C0004501B083B300B10125118A4F8B03B139CB
:1000D000B439BD39C239CB39D439D939DE39E139EE
:1000E000F439F739FA393B3A00408891D2E4ADB59A
:1000F000B6BEBFFF140900000000000100020304A7
:1001000005000000000000000000000000060708D5
:10011000090A0B0C0D0E0F1011000000000000006A
:1001200012131415161718191A1B1C1D1E1F202137
:1001300000000022232425262728292A2B2C2D00E5
:10014000002E2F3000003132333334353637383912
:100150003A3B3C3D3E3F4041424344454647484987
:100160004A4B4C4D4E4F5051525354555657585977
:100170005A5B5C5D005E5F606162636465666768D0
:10018000696A000000000000006B6C6D6E6F70719A
:1001900072737475767700000000000000000000A4
:1001A00000000078797A7B7C7D0004047E80818267
:1001B00095969798A7A8A9AAB5B6B7B8040483845A
:1001C000857E9798999AA8A9AAABB9BABBBC040432
:1001D000868788899B9C9D9EACADAEAF7EBEBFC01E
:1001E00004048A8B8C8D9C9D9E9FAEAFB0B1C1C222
:1001F000C37E04048E8F9091A0A1A2A38E8F9091B4
:10020000A0A1A2A3040492939293A4A5A4A5B2B31F
:10021000B2B3C4C5C4C50000000000000000000067
:1002200000000000000000000000000000000000CE
:1002300000000000000000000000000000000000BE
:1002400000000000000000000000000000000000AE
:10025000000000000000000000000000000000009E
:10026000000000000000000000000000000000008E
:10027000000000000000000000000000000000007E
:10028000000000000000000000000000000000016D
:10029000010000000000000000000000000000005D
:1002A000000000000000000000000000000000004E
:1002B000000000000000000000000000000000003E
:1002C0000000000009640000000000005B64000002
:1002D0000000005B64BF00000000000000000000A0
:1002E00000000000095B000000095B646464000911
:1002F0005B646464B6BF5B64646DBFBFBFBF6464AE
:10030000BFBFBFBFBFBFBFBFBFBFBFBFBFBFBFBFFD
:10031000BFBFBFBFB6B6000000095B5B00005B5B00
:10032000B6BFBF645B00B6BFBFBFBFBF645BBFBF2C
:10033000BFBFBFBFB65BBFBFBFBF645BBFB6BFBF02
:10034000B6645BB6BFBFB6645B5B64BFBFBF5B5BDD
:1003500009000064BFBF00000000000000000000B2
:100360000000000000000900000000000000640917
:100370000000000000005B640000000000006464F6
:100380005B0000000000BF64640000000000BFBF0D
:100390005B090000000000000000000000000000F9
:1003A000000000000000000000000000000000004D
:1003B000000000000102000000000203040500002C
:1003C0000003040302020000000002030405000011
:1003D0000204050505050000000000000000000003
:1003E0000000000000020000000000000104000006
:1003F00000000002030502000000010205050202E0
:1004000002010102050405050505040402020505B3
:1004100005050505050403040403020100000303A8
:10042000030303030201040404030302020204049D
:10043000050505040403030302030506050503037C
:100440000404030205050302000102030302020281
:100450000200000002030000000000000000000095
:100460000000000000000100000000000000020089
:10047000000000000000040302000000005B05050E
:10048000040300095BB604050505095BB6BF020459
:1004900005045BB6BFBF000000005BB6BFBF000035
:1004A0000964BFBFBFBF000964BFBFBFBFBF5B6DF3
:1004B000BFBFBFBFBFBFB6BFBFBFBFBFBF64BFBFB0
:1004C000BFBFBFBF6464BFBFBFBFBF645B09BFBF67
:1004D000BFBF64090000BFBFBFBFBFB6645BBFBF83
:1004E000BFB6645B0900BFB664645B00000064646F
:1004F000640900000000645B0900000000005B006C
:1005000000000000000000000000000000000000EB
:100510000000000009B609000000000964BF0000E7
:100520000000000009BF0000000000095B6400003B
:1005300000005B64646400000964BFBFBF64005BCB
:10054000BFBFBFBFBFBF64BFBFBFBFBFBFBFBFBF16
:10055000BFBFBFBFBFBFBFBF645B09000000BFBF5D
:10056000B65B5B5B0900BFBFBFB66464645B6DBF15
:10057000BFBFBFB6BFBFB6BFBFBFBFBF6D64BFBF4A
:10058000BFBF645B0952BFBF645B09000052BF5B21
:100590005B090000000000000000000000000000F7
:1005A0000000000000005B5B090000000000BF6469
:1005B0005B0000005B645B5B09095B64B6645252DC
:1005C00064B6BF645B64525BBF64095BB6BF5264D0
:1005D0005B5BB6BFBFBF0000000000000009000069
:1005E0000000005B5B5B00095B6464BFB66464642D
:1005F000BFBFBFBFBFB664BFBFBFBFBFBFBFBFBF6F
:10060000BFBFBFBFBFBFBFBFBFBFBFBFBFBFBFBFFA
:10061000BFBFBFBFBFBF0000000000000000646498
:10062000645B5B5B09006464B6B664646464B6B61C
:10063000B66465646464BFBFBFBFBFBFBFB6BFBFA2
:10064000BFBFBFBFBFBFBFBFBFBFBFBFBFBFBFBFBA
:10065000BFBFBFBFBF64000000000000000000007B
:100660000000000000005B0900000000000064645E
:10067000645B00000000B664B66400000000BFB612
:100680005B0900000000645B0900005252006464D2
:100690000052520000520000000000000000000064
:1006A000000000000000000000000000000000004A
:1006B0000000000000520000000000005252000044
:1006C00000000052525200000000525252520000EC
:1006D00000005252520000000204050505050052B8
:1006E00051020304050552525201020404045252FD
:1006F000520000020304520000000000000000004D
:1007000000000000000000000000000000000000E9
:1007100000000000000005050505050505050505A7
:10072000050505050505040505050505050504037D
:10073000030405050505000000010204050500008D
:1007400000000202020400000000000053520000FA
:1007500000000000ADA4050402030100000005052F
:10076000050504020000050505050505030105054D
:10077000050505050504050505050505050505052A
:10078000050505050505030505050505050502041F
:100790000505040403020203035C64BFBFBF00003D
:1007A0000964BFBFBFBF00005BB6BFBFBFBF0303CD
:1007B0006464BFBFBFBF0505B75BBFBFBFBF050553
:1007C000665BBFBFBFBF05055E5BBFBFBFBF0303A7
:1007D000015BBFBFBFBFBFBFBF6400000000BFBFA2
:1007E000640000000000BF6D5B0000000000BF5B04
:1007F000646400000000BFB65BBF09000000BFBF1B
:100800005BBF5B00005BBFBF656464005BBFBFBFD5
:10081000BF5B645BBFBF00000000005BBFBF0000A8
:1008200000005BBFBFBF00000064BFBFBFBF0009C7
:100830006DBFBFBFBFBF09BFBFBFBFBFBFBFBFBFD0
:10084000BFBFBFBFBFB6BFBFBFBFBFBF6409B6BFDB
:10085000BFBFBF640000BFBFBFBFBFBFBF64BFBFDC
:10086000BFBFBF5B0900BFBFBFBF64000000BFBF09
:10087000BF5B00000000BF640000000000005B00E0
:100880000000000000000000000000000000000068
:100890000000000000005B5B0000000000000000A2
:1008A0000000000000090000000000005BB600002E
:1008B0000000005BBFBF0000000064BFBFBF0000BE
:1008C0000064BFBFBFBF000964BFBFBFBFBF096433
:1008D000BFBFBFBFBFBF005BB6BFBFBFBFBF64BFAF
:1008E000BFBFBFBFBFBFBFBFBFBFBFBFBFBFBFBF18
:1008F000BFBFBFBFBFBFBFBFBFBFBFBFBFBFBFBF08
:10090000BFBFBFBFBFBFBFBFBFBFBFBFBFBFBFBFF7
:10091000BFBFBFBFBFBFBFBFBFBFBFBFBFBFBFBFE7
:10092000BFBFBFBFBFBFBFBFBFBFBFBFBFBFBFBFD7
:10093000BFBFBFBFBFBFBFBFBFBFBFBFBFBFBFBFC7
:10094000BFBFBFBFBFBFBFBFBFBFBFBFBF64BFBF12
:10095000BFBFBFBF645BBFBFBFBFBFB6646DBFBF1C
:10096000BFBF6409645BBFBFBF6409000000BFB6BE
:10097000646400000000BF64640900000000645B60
:100980000900000000005B090000000000000900F1
:100990000000000000005B00000052525200000006
:1009A0000000000052520000000000000052000051
:1009B0000000000000000000000000000000000037
:1009C0000000000000000000000000000000000027
:1009D0000000000000005200000000000000525221
:1009E0005252000000005252525252000000525225
:1009F00052525252000000525252525252000000C3
:100A00005252525252520000005252525252000060
:100A100000000052525200000000000000000000E0
:100A200000000000000000000000000000000000C6
:100A300000000000000000000000000009645200F7
:100A40000000000964BF525200000964BFBF525247
:100A500000095BB6B6BF0000000000000000000007
:100A60000000000000000000000000000000000086
:100A70000000000000005B5B090000000000BF6494
:100A8000090900000000BFBF5B5B00000000BF64FD
:100A9000646400000000000000000000000000008E
:100AA0000000000000000000000000000000000046
:100AB0000052000000010052525200000002525247
:100AC00000000001040452000000020405050000BB
:100AD0000003050505050000005252520000000009
:100AE00052525200000000015301000000000302B6
:100AF00004040301000003040505050403020405C2
:100B00000505050505050505050505050505050595
:100B100005050505050500000000000000000000B7
:100B200000000000000000000000000000000000C5
:100B300000000000000001000000000000000404AC
:100B4000020100000000050505050403020105057A
:100B5000050505050504000000000052ADA40000D5
:100B6000000000A4AD5B0000000052ADAD520000DB
:100B700000005BADA45300000000ADAD5B020000BF
:100B80000052ADAD53040100005BADA402050303A8
:100B90000253AD5B03050205050302520100030584
:100BA00004525BA452000305045BAD5B0000040526
:100BB000035BAD5B00000505035BAD52000005055E
:100BC00002A4A40100010505030353020304050563
:100BD0000504050505050000005BB6BFBFBF0000AA
:100BE00000B664BFBFBF000000BF64BFBFBF00004E
:100BF000005B64BFBFBF0101000064BFBFBF04044E
:100C000003005BBFBFBF050505035BBFBFBF050595
:100C100005055BBFBFBFBFBFBF5B5BB6BF64BFBFE8
:100C2000BF655BBFBF64BFBFBFBF64B6BFBFBFBF51
:100C3000BFBF6D64BFBFBFBFBFBFBF6464BFBFBF27
:100C4000BFBFBF6464BFBFBFBFBFBFBFBFBFBFBF6A
:100C5000BFBFBFBFBFBF64BFBFBFBF64000064BF33
:100C6000BFBFB65B000064BFBFBF5B525BA4BFBF2A
:100C7000BFB652ADA45BBFBFBF5B52525B5BBFBF91
:100C8000640964B6B6BFBFBFBFB6BFBF6D64BFBFA8
:100C9000BFBFB66464B60000000052525B6452529B
:100CA0005B5BA45BB6BFAD5B5B52525BBFBF525296
:100CB0005B5B5B64BFBF64B6AD5B5B64BFBF64641A
:100CC000645B6464BFBF645B09525B64BFB65B096D
:100CD000005B525BBF6464BFBFBFBFBFBFBFBFBFCE
:100CE000BFBFBFBFBFBFBFB6B6B6B6B6B6B6646508
:100CF0005B5B5B09095B5B640000000000000900AE
:100D00000000000000005B000000000000005B002D
:100D1000000000000000BFBFBFBFBFBFBFBFBFBF5D
:100D2000BFBFBFBFBFBFBFBFBFBFBFBFBFBF5B5B9B
:100D300064646464B6BF005252525B5B0964005243
:100D4000525BA4A4525B0000000000525B52000002
:100D5000000000005B52BFBFBFBFBF645B09BFBFE5
:100D6000BFB65B5B5B00BFBFB65B5BADA400B664A8
:100D70005B5BA4A45200BF5B5BADADA40000BF648D
:100D80005BADADAD0000B6BF5B5BADAD5B00ADBFB5
:100D9000B65BA4ADAD52000000000000525200004E
:100DA00000000000005200000000000000000000F1
:100DB000000000000000000000000000000900002A
:100DC0000000000009090000000000005B64000052
:100DD0000000095B64B65252005B5B655BBF525218
:100DE0005B645B5B64B6005BB6BF646464640064B0
:100DF0006464B6B6095B095B64B6BFBF646464B67D
:100E0000BFBFB6BFB65BBFBFB66464BFBFB6B66494
:100E10005B6DBFBFBFBFB65BBF090000000064B61B
:100E20005B000000000064640000000000005B0044
:100E300000000000000009000000000000005B5BF3
:100E40000900000000005B5B645B09000000BF64F8
:100E50005B64645B00000000000000000001000013
:100E6000000000000001000000000002000200007D
:100E7000000104025CA60000010453ADFFFF000066
:100E80000454ADFFFFFF000304ADFFADA4AD0005AA
:100E900003ADAD5BADAD000103050505050502041D
:100EA00005050505050505050505050505055605A1
:100EB000050505050505FFFF5E0505050505FFFFA1
:100EC000FFAF05050505FFFFFFFF55050505ADADA6
:100ED000ADFFFF0505050505050505050505050526
:100EE00005050505050505050505050505050505B2
:100EF00005050505050505050505050505050505A2
:100F00000505050505050505050505050505050591
:100F10000505050505050505040353020505050539
:100F20000505040405050505050505050453050526
:100F30000505050453FF050505050501A4FF050585
:100F4000050502ADADAD050505045BAD5BAD050561
:100F50000553AD5B5BA40505050505050505030205
:100F60000304050505055B52020103050505AD52A5
:100F7000AD52020505055BADFFAD5C020503A4ADF6
:100F8000FFADA5020203AD5BAD5BA4000102ADADF8
:100F90005B5252005200050505055BBFBFBF05054A
:100FA00005055BBFBFBF050505045BBFBFBF0505EA
:100FB000050464BFBFBF0405050164BFBFBF0504CE
:100FC000010064BFBFBF0200005B5BBFBFBF00008A
:100FD000005BBF64BFBFBFBFBFBFBFBFBFBFBFBF9F
:100FE000BFBFBFBFBFBFBFBFBFBFBFBFBFBFBFBF11
:100FF000BFBFBFBFBFBFBFBFBFBFBFBFBFBFBFBF01
:10100000BFBFBFBFBFBFBFBFBFBFBFBFBFBFBFBFF0
:10101000BFBF646464B6BFBFBFBF6D645B09BFBFC1
:10102000BFBFBF5B0000BFBFBFB6645B0000BFBFF8
:10103000BFB664640000BFBFBFBF645B0900BFBF31
:10104000BFBFBF5B0000BFBFBFBFBFB60900BFBF10
:10105000BFBFBFBFB609000000AD525BBF5B000061
:1010600052AD5B64BF09000052A45BB6B65B0000E2
:101070005BA45BBF646400005BA464BF5B640000AE
:10108000AD5B64BF5BBF0000AD525BBF5BBF005296
:10109000AD525BBF5BB6B600000000000000BF00B1
:1010A000000000000000B600000000000000640026
:1010B0000000000000005B000000000000000900CC
:1010C0000000000000000000000000000000000020
:1010D000000000000000000000000000005B0000B5
:1010E00000000000005B000000000000005B00004A
:1010F000000000000052000000000000005200004C
:1011000000000000000000000000000000000000DF
:1011100000000000005B5BB6BF6452ADAD5B52B631
:10112000BFBF5B5BADAD5B5BBFBFB652ADADA45B9C
:10113000BFBFBF525BADA45B64BFBFB652A4AD528C
:101140005BBFBFBFB6525B5B5BBFBFBFBF645B64CF
:10115000BFBFBFBFBFBF00000000000000005200C3
:10116000000000000000A452000000000000AD5B81
:10117000000000000000ADAD000000000000ADADBB
:101180005B000000000052ADAD52000000005BA407
:10119000ADAD0000000900000000000000000000EC
:1011A000000000000000000000000000000000003F
:1011B000000000005BBF000000000064BFBF000033
:1011C000005BBFBFBFBF005BB6BFBFBFBFBF64BFD9
:1011D000BFBFB664B6BF00000964BFBFBF64006490
:1011E000BFBFBFBF645B5B5B645B095B64BFBFBFCA
:1011F000BFBFBFBFBFBFBFBFBFBFBFBFBFBFBFBFFF
:10120000BFBFBFBFBFBFBFBFBFBFBFBFBFBFBFBFEE
:10121000BFBFBFBFBFBF5B64BFBFBFBFBFBFB6BFA6
:10122000BFBFBFBFBFBFBFBFBFBFBFBFBFBFBFBFCE
:10123000BFBFBFBFBFBFBFBFBFBFBFBFBFBFBFBFBE
:10124000BFBFBFBFBFBFBFBFBFBFBFBFBFBFBFBFAE
:10125000BFBFBFBFBFBFBFBFBF645B5B0952BFBFE4
:10126000BFBF645B0900BFBFBFBFBFB65B00BFBFEE
:10127000BFBFBFBFBF5BBFBFBFBFBFBFBFBFBFBFE2
:10128000BFBFBFBFBFBFBFBFBFBFBFBFBFBFBFBF6E
:10129000BFBFBFBFBFBF5252000000000000000030
:1012A000000000000000000000000000000000003E
:1012B0000000000000000900000000000000BF095D
:1012C000000000000000BFB6000000000000BFBF2B
:1012D00064525B5252520000000000000000000007
:1012E00000000000000000000000000000000000FE
:1012F0000000000000000000000000000000AD5BE6
:10130000520000000000FFFFFFAD5200000052FF3E
:10131000FFFFFF520000020553FF5BADFFFF040417
:1013200054FFA45BADAD030304AFFFFFFFAD0002AC
:101330000505AFFFFFFF000305050555AEAE000331
:10134000050505050303000103040404040400006B
:10135000000103040404FFADADFFFF560505ADAD6C
:10136000ADFFFF550505AD5BADFFAE050505FFFF04
:10137000FFAF050505055D55560505050505030582
:10138000050404040505050505040303030404041A
:1013900005050505050505050505050505050504FE
:1013A0000505050505AF03010305050556FF030205
:1013B000040505055DFF05040505050556FF050542
:1013C0000505050505AE0505040404050505050527
:1013D00005030405050555AFAEAF5E050505FFFF26
:1013E000FFFFFFFF5E05FFADADADFFFFFF55FF5BEC
:1013F0005BADADADFFFFAD5BADFFFF5BA4FFFFAD30
:10140000ADADADADADFFAFFFFFFEADADAEA7035DC2
:10141000AFAFA65D5605050503ADAD5BADFF050598
:10142000015BAD5BFFFF05050100520052525604FF
:101430000200000000005E030401000000005604EA
:101440000300000000000504040000520000030433
:101450000200005200005BAD5B52000052005B5284
:10146000000000000000000000000000000000007C
:10147000000000000000000000000000000000006C
:101480000000520000000000005252000000005214
:1014900052520000000000000009B664B6BF000010
:1014A0000000095B5B6D000000000000005B0000B5
:1014B000000000000000000000000000000000002C
:1014C000000000000000000000000000000000001C
:1014D000000000000000BFBF6D0900000009BF6DE3
:1014E0005B0952520000B6095B52ADADAD00090078
:1014F000005B5BADAD52000000525BADADAD0000D6
:1015000000ADADADADFF000000ADFFADADFF000023
:10151000005B5BA4AD5B0964B6BFBFBFBFB6000094
:10152000005BBFBFBFBF520000005B65BFBFAD5BCC
:101530005200000964BFFF525B52000909B6FF5216
:10154000AD5200095B5BFF5BAD5B00005B00ADADC6
:10155000ADAD000009095B525B5264BF6465BF64B6
:101560005B64BFB66464BFBFBFBFBFBF5B64BFBFC8
:10157000BFBFBFBFB6B6BFBFBFBFBFBF5B64BFBF4C
:10158000BFBFBF646464B6BFBFBFBF6464B664BF9F
:10159000BFBFBF64B6BF0000000000000000000035
:1015A000000000000000645B090000000000B6B607
:1015B000B66464646464B6BFBFBFBFBFBFBF6464CA
:1015C000B6BFBFBFB6B6646464B6656464646D6478
:1015D00064BFBFBFB6B6000000000000645B00003F
:1015E000000009095B6400095B5BB6B65BBF64641D
:1015F00064B6BF5BB6BFBFBFBFBFBF5B6464B6B6F8
:10160000BFBFBFB664646464BFBFBFBFBFBFB6B671
:10161000BFBFBFBFBFBF64646464646464B6BFB669
:10162000B6B6645B5BB6BFBFBFBF64646464BFBF74
:10163000646464B6645B6464645B6464BFBF64B622
:10164000BFBFBFBFBFBFBFBFBFBFBFBFBFBFBFBFAA
:10165000BFBFBFBFBFBFB65BA4AD52005BB6BF6428
:101660005BA45264BFBFB6BF5B5BB6BFB66464BF6A
:10167000BFBFBFB66464BFBFBFBFBFB6BFBFBFBF42
:10168000BFBFBFBFBFBFBFBFBFBFBFBFBFBFBFBF6A
:10169000BFBFBFBFBFBFBFBFB66464B6BFBF6D64CF
:1016A0005B64BFBFBFBF5B64BFBFBFBFBFBFBFBFC8
:1016B000BFBFBFBFBFBFBFBFBFBFBFBFBFBFBF6495
:1016C0006DBFBFBFBFBFBFB664BFBFBFBFBFBFBFE0
:1016D000645BBFBFBFBFBFBFBFBFBFBFBFBFBFBFD9
:1016E000BFBFBFBFBFBFBFBFBFBFBFBFBFBFBFBF0A
:1016F000BFBFBFBFBFBFBFBFBFBFBFBFBFBFBFBFFA
:10170000BFBFBFBFBFBFBFBFBFBFBFBFBFB6BFBFF2
:10171000BFBFBFBFFFFFBFBFBFBFBFBFBFBFBFBF59
:10172000BFBFBFBFBFBFBFBFBFBFBFBFBFBFBFBFC9
:10173000BFBFBFBFBFBFBFBFBFBFB7BFBFBFBFB6CA
:10174000FFFFFFFFFFB6FFFFFFFFFFFFFFFFFFFFF2
:10175000FFFFFFFFFFFFBFBFBFBFBFBFBFBFBFBF19
:10176000BFBFBFBFBFBFBFBFBFBFBFBFBFBFBFBF89
:10177000BFBFBFBFBFBFBFBFBFBFBFBFBFBFBFBF79
:10178000BFBFBFBFBFBFB66464BFBFBFBFBFA4649E
:101790005BBFBFBFBFBFBFBFBFADAD5B52ADBFBFC4
:1017A000FFFF5BAD00ADBFB6FFFF5B5B5252BFFFFB
:1017B000FFAD52525B00B6AD5BADAD5B5B00B6AD4D
:1017C00000FFADAD5B00FFFFAD5BADADAD00ADADFE
:1017D000FF5B525BAD5B00ADFFFFFFAD0000005251
:1017E000FFFFFFFF52005200FFFFFFFFAD005B0055
:1017F000ADFFFFFFAD005B52ADFFFFFFFF00525B8F
:10180000ADFFFFFFAD0052ADFFFFFFFF520000AD87
:10181000FFFFFFAD00000000000001030404000012
:1018200000000000010300000000000000000000B4
:1018300000000000000000000000000000000000A8
:101840000000000000000000000000000000000098
:101850000000000000000404030303040405050560
:101860000505050403020001020304040505000048
:101870000000000000000000000000000000000068
:101880000000000000000000000000000000000058
:10189000000000000000050505050505050502021C
:1018A0000304050505050504030201010203010205
:1018B0000203030403030000000000000000000016
:1018C0000000000000000000000000000000000018
:1018D00000000000000003030305050505030504DF
:1018E00004050505040204050505050502050202B7
:1018F00002030302030100010202020000000000D3
:1019000000000000000000000000000000000000D7
:1019100000000000000003040000005252520502C3
:1019200000000000000003000000000000000000B4
:1019300000000000000000000000000000000000A7
:101940000000000000000000000000000000000097
:1019500000000000000052520000000000000000E3
:101960000000000000000000000000000000000077
:101970000000000000000000000000000000000067
:101980000000000000000000000000000000000057
:1019900000000000000000000000ADADADAD000093
:1019A0005200ADFFFFFF000052005BADFFFF0000E3
:1019B00000520052ADFF520000000000005B00002A
:1019C00000000000000000520000000000000000C5
:1019D0005200000000005BFFAD5B5200005B5BAD9E
:1019E000AD5BAD52005BAD5BADADAD520009FF52DA
:1019F000ADADAD000000ADADAD5B5B000000005BC8
:101A00005B00000000000000000000000052000029
:101A10000000000000525BBFBFBFBF6464645BBFD7
:101A2000BFBFBF6464645BBFBFBFBF645B0964BF0B
:101A3000BFBFBF5B6DBF64BFBFBFBF5B09645BBFA0
:101A4000BFBFBF64BFBF005BB6BFBFBFBFBF005B50
:101A5000645B64BFBFBFBFBFBFBFBFBFBFBF646466
:101A6000BFBFBFBFBFBF64BFBFBFBFBFBFBF64BF3C
:101A7000BFBFBFBFBFBFBFBFBFBFBFBFBFBFBFBF76
:101A8000BFBFBFBFBFBFBFBFBFBFBFBFBFBFBFBF66
:101A9000BFBFBFBFBFBFBFBFBFBFBFBFBFBFBFBF56
:101AA000BFBFBFBFBFBFBFBFBFBFBFBFBFBFBFBF46
:101AB000BFBFBFBFBFBFBFBFBFBFBFBFBFBFBFBF36
:101AC000BFBFBFBFBFBFBFBFBFBFBFBFBFBFBFBF26
:101AD000BFBFBFBFBFBFBFBFBFBFBFBF6464BFBFCC
:101AE000BFBF645B5BADBFBFBF5B00005252BFB600
:101AF0005B000000FF5BB60900000000FFADB65BB5
:101B00005B000000ADADBF6D5B000000ADADBFBFC1
:101B10005B0000005BFF5BADADB6BFBFBFBF5B5BF3
:101B2000ADADAD64BFBF5B5B5200005B5B09ADFF59
:101B3000FFFF52520000ADFFFF5BADAD52525BADF7
:101B40005BADAD52ADFF5BADADFF5BADFFFFADADCE
:101B5000FF5BADFFFFFFBFBFBF6464BFBFBFBFBFC1
:101B6000BFBF5BB6BFBF64BFBFBF6D09BFBF00646F
:101B7000BFBFBF5B64BF000064BFBFBF5BB65B009D
:101B800000B6BFBF6D5BFFAD0009BFBFBFADFFFFBC
:101B90005B0009BFBFB6BFBFBFBFB7FFFFFFBFBF7F
:101BA000BFB6FFFFFFFFBFBFFFFFFFFFFFFFBFFF8E
:101BB000FFFFFFFFFFFFFFFFFFFFFFFFFFADFFFF87
:101BC000FFFFFFAD5B52A4ADAD5B52525BADAD5BB1
:101BD00052005BFFFFFFFFFFFFFFFFFFFFFFFFFF65
:101BE000FFFFFFFFFFFFFFFFFF5BFFFFFFFFFFADFB
:101BF000525BFFFFFFFF525BAD00ADFFADAD5BFF82
:101C0000A4A452AD5BADFFFF5BAD5B5BFFFFFFFFCD
:101C10005BFFAD5BFFFF52AD0964BFBFB65BAD5B61
:101C2000B65BBF645B64FFADBF645B64BFBFFFAD09
:101C30005B64BFBFBFBF5BADFFBFBFBFBFBFFFFF29
:101C4000FFFFBFBFBF65FFFFFFFFBFBFB65BFFFF6B
:101C5000FFFF6DBFBFBF5BADFFAD52ADFFFFB6FF76
:101C6000FFFFFFADADFFBFFFFFFFAD52ADFFBFFFF9
:101C7000FFAD52FFFFFFBFADFFFFFFFFFFB65B648D
:101C8000B6B6B6B6BFBF65BFBFBFBFBFBF5BBFBF46
:101C9000BFBFBFBFBFB6525BFFFFAD520000AD007C
:101CA000FFFF52000000FF525B5200000000FFAD3A
:101CB000000000000000BFBF0900000000006464D5
:101CC0000900000000005B5B0900000000005B5B96
:101CD0006409000000000000005200000000000045
:101CE00000005252000000000000000052520000AC
:101CF00000000000000000000000000000000000E4
:101D000000000000000000000000000000000000D3
:101D1000000000000000525200000052520000007B
:101D2000000052000000525252000000000000006B
:101D300000000000000000000000000000000000A3
:101D40000000000000000000000000000000000093
:101D50000000000000000000000000095BB6000069
:101D60000000000000000000000000000000000073
:101D70000000000000000000000000000000000063
:101D80000000000000000000000000000000000053
:101D9000000000000000BFBFBFBFBFBFBFBF0964DE
:101DA000B6BFBFBFBFBF0909095B64B6B6BF005B62
:101DB000645B5B095B640000095B5B5B5B5B000071
:101DC000000000090000000000000000000000000A
:101DD000000000000000BFBFBFBFBFBFBFBFBFBF8D
:101DE000BFBFBFBFBFBFBFBFBFBFBFBFBFBF64B667
:101DF0006DB6B6B6BFBF5B5B6464646464BF095B09
:101E00006464646464640000095B6464B6B60000E2
:101E1000000000095B64BFBF5B00000052FFBFBF52
:101E20005B00000000ADBFBF5B0052000052BFBFAF
:101E3000640052000000BFBFB60952000000646495
:101E4000640900000000B6B6646400000000646429
:101E5000645B00000000FFFF5BADFFFFFFFFFFFFC3
:101E60005BADFFFFFFADFFFF5BADADADAD5BADFFAC
:101E7000AD5B5B5B5BAD52ADFFFFFFFFFFFF005B48
:101E8000FFFFFFFFADAD00005BAD5B5B52000000EC
:101E9000000000000000FFFFAD000064BFB6ADAD64
:101EA000000000006DBFADAD000000005BBFFF5241
:101EB0000000000009B65B000000000000640000A4
:101EC00000000052000900000000000000090000AE
:101ED000000000000000FFFFAD52FFFFFFFFFFFF0B
:101EE000FF52FFFFFFFFFFFFFFAD5BFFFFADFFFFF7
:101EF000FFFF52AD5B52B6FFFFFFAD5BADFFBFB65C
:101F0000FFFFFFFFFFFF6DBFB6FFFFFFFFFF5BBFE0
:101F1000BFB6FFFFFFFFFFFF5B52005BFFFFFF5BF2
:101F200052ADFFFFFFFF525BFFFFFFFFFFADADFFB5
:101F3000FFFFFFFFAD52FFFFFFFFFFAD52ADFFFF01
:101F4000FFFFFFADADB6FFFFFFFFFFFFBFBFFFFF0E
:101F5000FFB6BFB6BFBFFFFFFF5B5BBFBFBFFFFFEB
:101F60005B64BFBFBFBFFFFFB6BFBFBFBFBFADFF9B
:101F7000BFBFBFBFBFBFB6BFBFBFBFBFBFBFBFBF7A
:101F8000BFBFBFBFBFBFBFBFBFBFBFBFBFBFBFBF61
:101F9000BFBFBFBFBF64BFBFBFBFBFBFBFBFBFBFAC
:101FA000BFBFBFBFBFBFBFBFBFBFBFBFBFBFBFBF41
:101FB000BFBFBFBFBF64BFBFBFBFBF645B00BFBF0A
:101FC000B6645B090000B664645B09000000645BF2
:101FD00009000000000064B6BF5B00000000BFBF46
:101FE000B60900000000BF6D090000000000640990
:101FF00000000000000000000000000000000000E1
:1020000000000000000000000000000000000000D0
:1020100000000000000000000000000000000000C0
:10202000000052000000000000000000000000005E
:102030000000000000520052525252525200000062
:102040000000000000000000000000000000000090
:10205000000000000000000000000052520000528A
:10206000000052525200525252525200000052523C
:1020700052520000000000000000000000000000BC
:102080000000000000000000000000000000000050
:10209000000000000000000964BFBFB7B6B6000032
:1020A000005BBFBFBFBF000000000964BFBF0000EE
:1020B0000000000064BF000000000000005B0000A2
:1020C0000000000000000000000000000000000010
:1020D000000000000000B6B7BFBF5B5BBFBFBFBF63
:1020E000645B64646DBFBF5B645B5B5B64BF645BCC
:1020F000B6645B64BFBFBF64B664BFBF645B64BFEC
:10210000B6645B095BB600095B5B5B6DBF64000096
:1021100000095B090000BFBFBFBFBFB65B64BFBFA4
:10212000BFBF645B645BBFBF645B646409006464DD
:1021300064645B00000064BF640900000000B65BDB
:102140000000000000000900000000000000000086
:102150000000000000005B0900000000000000001B
:10216000000000000000000000000000000000006F
:10217000000000000000000000000000000000005F
:10218000000000000000000000000000000000004F
:1021900000000000000029292929292929292929A5
:1021A000292929292929292929292929292929299F
:1021B000292929292929292929292929292929298F
:1021C000292929292929292929292929292929297F
:1021D00029292929292900000707070700000007E6
:1021E0000707070707000707070707070707070786
:1021F000070707070707070707070707070707076F
:10220000070707070707000707070707070000007A
:102210000707070700002929292929292929292908
:10222000292929292929292929292929292929291E
:10223000292929292929292929292929292929290E
:1022400029292929292929292929292929522929D5
:102250002929295252522929292929292929292973
:10226000292929292929292929292929295B2929AC
:1022700029295252525229295B5B525252525B52C7
:1022800052525252525B52525B5B525B5B52525BF8
:1022900052525252525B29292929292929292929AF
:1022A000295252525B525252525B52525B5252521C
:1022B00052525B5B525252525252525252525252EC
:1022C000525252525B52525252525252525B5B52D3
:1022D0005252525252522929292929292929525226
:1022E00052525229292952525252525252525B5B37
:1022F0005252525252525B5B5252525252525252AC
:102300005B52525B52525252525B5B525252525289
:102310005B52525B5B52292929292929292929291C
:1023200029292929292952292929292929295252A2
:10233000525229292929525252525B52292952526A
:102340005252525B52525252525252525252525264
:102350005B5B5252525229292929292929292929E5
:1023600029292929292929292929292929292929DD
:1023700029292929292929292929292929292929CD
:102380002929292929295229292929292929525242
:1023900052292929292929525252525B5252295233
:1023A000525252525252295B525252525252295B4D
:1023B0005B5B52525252295252525B52525229295D
:1023C0005B5B525B5B5B2929525252525252292964
:1023D00052525252525252525252525B5B525252CB
:1023E0005252525252525252525252525252525BC4
:1023F0005B525B5B5B525252525252525252525299
:10240000525B5252525B5B52525252525252525B88
:102410005B52525252525252525252525252525293
:10242000525B5252525252525B5252525B525B5B5F
:102430005B5252525252525252525B5B525B525258
:102440005B5252525B52525252525252525B5B5B3F
:102450005B5252525252525252525252522952527C
:102460005B52525252525252525252525B5B525231
:10247000525B5B525B5B5B5252525252525252520F
:102480005B52525B52525B525B5252525252525208
:102490005B5B5B525B5B295B52525252525252520F
:1024A0005B5B5252525B52525252525252525B52E8
:1024B00052525252525B525B5252525252525B52E1
:1024C0005B5B5B52525252525252525B5B525252BF
:1024D00052525252525B52525B52525252525B5BB8
:1024E0005252525252525252525B5252525B5252BA
:1024F000525B5B5B5252525252525B5B52525B5B7D
:102500005B5252525252525252525B5B525B525287
:10251000525B5252525252525B5252525252525289
:102520005252525252525B5B5252525B5252525270
:10253000525252525B5B5252525252525252525B60
:102540005252525252525B52525252525252525B59
:102550005B525252525252525252525252295B5272
:102560005252525252295B52525252525229525294
:102570005B5B5252522952525B5B525252295B5260
:1025800052525B522929525B5252525B29295252B4
:1025900052525B5229292952525252525B522952AD
:1025A00052525252525B2952525252525252295254
:1025B0005252525252522952525252525B52295244
:1025C00052525252525B2952525252525252295234
:1025D00052525B5B525252525252525252525252C9
:1025E000525B5B5B525B5252525252525B525B5B8C
:1025F0005B52525B5B5252525252525252525252A0
:10260000525B5B525B52525252525252525252528F
:102610005252525B5B5252525252525252525B527F
:102620005B5B5252525252525B5B52525252525266
:10263000525252525252525B52525B525252525268
:102640005B5B5252525B525252525B52525B52523D
:1026500052525252525B5B52525252525229525271
:102660005252525252295252525B525252295B528A
:10267000525B5B5B52295252525252525B29525B5F
:102680005B525B5B522952525252525252295B5258
:10269000525B525252292929292929292929525282
:1026A000525252525252525252525252525252520A
:1026B000525B5B525B5B52525252525252525B5BC4
:1026C0005252525B525252525B52525252525252D8
:1026D000525B5B5252522929292929292929525210
:1026E0005252525B5252525252525B5252525B52AF
:1026F0005B5B5B5252525252525252525B5B525B84
:1027000052525B52525252525252525252525252A0
:102710005B5B5B525252000018181818000000183A
:102720001818181818001818181818181818181841
:102730001818181818181818181818181818181819
:102740001818181818180018181818181800000069
:10275000181818180000292929292929292929297F
:1027600029292929292929292929292929292929D9
:1027700029292929292929292929292929292929C9
:102780002929292929522929292929292952292967
:1027900029292929525229292929525B5B522929A1
:1027A000295252525252292952525B525252295B9B
:1027B000525B525252525252525252525252525BE7
:1027C00052525B525B5B5252525252525B5B5252BC
:1027D00052525252525252525B5B525252525252C7
:1027E000525252525252525B52525B5252525B52AE
:1027F00052525252525252525252525252525252B9
:1028000052525B5252525B5B5252525252525B5284
:1028100052525252525B525B5B5252525B52525274
:1028200052525B5B5B525252525252525B52525264
:102830005252525252525252525B52525B52525266
:1028400052525B5B52525252525252525252525256
:1028500052525B5B5B5252525252292929295252E1
:10286000525B522929295B52525252522929525203
:102870005252525252295B52525B525252525B5246
:102880005252525252525252525252525252525228
:1028900052525252525229292929292929292929B2
:1028A0002929292929292929292929292929292998
:1028B000292929292929292929292929292952295F
:1028C00029292929292952292929292929295252FD
:1028D000292929292929292952525B525252292969
:1028E00029525252525229292952525252522929BE
:1028F000295252525B5B292929295B5252522929BC
:1029000029295B525252292929292952525229290F
:10291000292929525B5B525B52525252525B5252EE
:102920005252525252525252525252525252525287
:1029300052525B525252525B525252525252525B5C
:102940005252525252525252525252525252525267
:1029500052525B5B5B52525252525B5B525252522A
:102960005252525252525252525B52525B52525235
:102970005B5252525252525252525252525252522E
:10298000525252525B5252525B5B5252525252520C
:102990005B52525252525252525B5B5252525252FC
:1029A000525252525B5B52525252525252525252F5
:1029B00052525252525252525252525B52525252EE
:1029C000525252525B5B5252525252525252525BCC
:1029D000525252525B5B5B525252525229295B5205
:1029E0005252522929295B525252522929295252B4
:1029F0005B5B522929295B525252292929295252BB
:102A000052522929292952525B29292929295B5205
:102A10005229292929292952525B5252525B295B9A
:102A20005B5252525B522952525B525252522952BD
:102A3000525252525252295252525B5B52522952B6
:102A40005252525252522952525B5252525B2952A6
:102A500052525B5B525252525252525252525B5B32
:102A60005252525B525252525B5252525252525234
:102A70005252525252525B5B5B52525B5252525212
:102A80005B5252525252525252525252525252521D
:102A90005252525252525252525252525252525B0D
:102AA00052525252525B52525252525252525252FD
:102AB0005B5B525B5B5B525252525B5252525252C0
:102AC00052525252525252525252525252525252E6
:102AD00052525252525B5252525252525B295B52E4
:102AE0005252525252295252525252525229525218
:102AF000525252525229525B5B5252525B295252ED
:102B0000525252525B2952525252525252295B52E5
:102B1000525B525252295252525B5B5252525252A3
:102B2000525252525B52525252525252525B5B5B61
:102B30005252525252525252525252525B5B525263
:102B400052525252525B52525252525252525B5B4A
:102B50005B5252525252525252525252525252524C
:102B60005B5B52525B5B5B52525252525252525218
:102B70005252525252525B525B5B525252525B5211
:102B80005252525252525252525252525252525225
:102B900052525252525200003A3A3A3A0000003A27
:102BA0003A3A3A3A3A003A3A3A3A3A3A3A3A3A3ABF
:102BB0003A3A3A3A3A3A3A3A3A3A3A3A3A3A3A3A75
:102BC0003A3A3A3A3A3A003A3A3A3A3A3A0000004D
:102BD0003A3A3A3A000029292929295252522929F8
:102BE0002929295252522929292952525252292936
:102BF0002929525252522929295252525B522929CB
:102C000029525B525B522929295B5252525229297F
:102C1000525B52525B5252525B52525252525B5B67
:102C2000525B5B52525252525252525B52525B5B57
:102C30005B52525252525B5B5B5252525252525250
:102C40005B52525252525252525252525B52525252
:102C50005252525252525252525252525B5B525242
:102C60005252525252525252525252525252525244
:102C70005252525252525252525252525252525234
:102C800052525B525252525252525252525252521B
:102C900052525B525252525B5B5252525252525BF0
:102CA0005B52525252525B5B5B5B5B525252525BC5
:102CB0005B52525252525252525B525252525B52D9
:102CC0005252525252525252525B5B5252525252D2
:102CD000525B5B525252525252292929292952528F
:102CE0005229292929295B5B525229292929525223
:102CF0005B522929292952525B52522929295252C1
:102D00005252522929295252525252292929525299
:102D10005B5B5B5229292929292929295252292912
:102D200029292929295229292929292929522929C1
:102D30002929292929292929292929292929292903
:102D400029292929292929292929292929292929F3
:102D5000292929292929525252525B52525B525237
:102D600052525252525B5252525B525B5B5B5B520D
:102D7000525B5252525B2952525B52525252292993
:102D80005252525B5B5229292952525252522929DE
:102D90002929525252525252525252525252525265
:102DA0005252525252525B5B5B5252525B525252DF
:102DB00052525252525B5B5B52525252525B5252CF
:102DC0005252525252525B5B5B52525252525B5BB6
:102DD0005B525252525B52525252525252525252C1
:102DE000525B5B52525252525252525B5B5B5B528D
:102DF0005B5B5B5252525B5252525252525252528F
:102E000052525252525252525252525252525B5B90
:102E1000525B5B525B5B525B525252525252525265
:102E2000525B5B525252525B5B525252525252525E
:102E30005252525252525B525B5252525B29525280
:102E40005252525B29295B5252525229292952521D
:102E50005B5229292929525229292929292952290C
:102E600029292929292952292929292929292929A9
:102E700029292929292929292929292929292929C2
:102E800029292929292929292929292929292929B2
:102E90002929292929295252525252525B525252FF
:102EA00052525252525252525252525B525B5252F0
:102EB0005B52525B52525B5B5252525B52525B5BB3
:102EC00052525252525B5B5B5252525252525252C7
:102ED000525252525252525B525252525252525BC0
:102EE0005252525252525B5B5B5B5B525252525B8C
:102EF00052525252525252525B5B525252525B5297
:102F000052525252525252525B5B5B525252525286
:102F10005B5B5B5252520000040404040000000496
:102F20000404040404000404040404040404040465
:102F30000404040404040404040404040404040451
:102F40000404040404040004040404040400000051
:102F500004040404000029295252525252522929D1
:102F600052525252525229295B52525252522952B3
:102F70005252525252522952525252525252295283
:102F8000525B525B5B522952525B5252525229524F
:102F900052525B52525252525252525252525B5BF6
:102FA0005252525B525252525252525B52525B52E6
:102FB000525B52525252525252525252525B5252DF
:102FC000525252525B525252525252525B5B5252C6
:102FD0005252525B5252525B5B5B5B5252525252A4
:102FE000525252525252525252525B5252525B52AF
:102FF0005252525B5B52525B5B5B525B5B52525272
:1030000052525252525252525B5B5252525252528E
:103010005252525252525B5B5B5252525252525275
:1030200052525B5B52525252525252525252525B65
:103030005B5B52525B5252525252525252525B524C
:1030400052525252525B5B5252525252525252524E
:103050005252525252295B5B5252525252525B5B55
:103060005B52525252525252525252525B5252522E
:1030700052525252525B5252525252525252525227
:103080005252525252525252525B5B525252295237
:103090005252525B525B525B5252525252525252F5
:1030A00052525252525252525252525B52525B52EE
:1030B0005252525252525252525252525252525BE7
:1030C00052525252525252525252525B5B5B5B52BC
:1030D0005252525252525B5B5B52525252525252B5
:1030E00052525B52525B5252525B525252525252A5
:1030F000525252525252525B5B525252525B525295
:103100005252525B5B525252525252525252525B84
:103110005B52525252525B5B5252525B29295252BD
:103120005B525252292952525B5252522929525211
:1031300052525252522952525252525252295252C1
:103140005B52525252295252525252525B295B5B8D
:10315000525B5B52522900000000FFFFFFFF00009E
:103160000000FFFFFFFF00000000FFFFFFFF000067
:103170000000FFFFFFFFFFFFFFFF00000000FFFF59
:10318000FFFF00000000FFFFFFFF00000000FFFF47
:10319000FFFF0000000029292929295B5B5B292901
:1031A0002929292929522929292929292929292966
:1031B000292929292929292929292929292929297F
:1031C000292929292929292929292929292929296F
:1031D0002929292929295252525252525B525252BC
:1031E0005B525B5B525B5B5B52525252525B2929D2
:1031F000525252525252292929295B5B5252292993
:1032000029292929295B29292929292929292929FC
:1032100029292929292952525B5252525B5B5B5260
:103220005252525252525B52525B5B5B525252525A
:103230005252525B525252525252525B52525B5253
:103240005252525252522929295B5B525B5B292907
:1032500029292929292952525252525B5B525B5B20
:103260005B5B525B5B525B5B5252525B5B5B5252ED
:1032700052525252525252525B5B525B5B5B525201
:1032800052525252525252525B5B5B2929292929D0
:103290002929292929295252525B5B5B5B525252E0
:1032A0005252525252525252525252525B525252F5
:1032B0005B52525229295B5B525B292929295229E9
:1032C000292929292929292929292929292929296E
:1032D00029292929292952525B29292929295229B1
:1032E000292929292929292929292929292929294E
:1032F000292929292929292929292929292929293E
:10330000292929292929292929292929292929292D
:1033100029292929292952525B525252525B525271
:103320005B525252525252525B5B5B525252525259
:1033300052525252525252525B5B5B5B5252525249
:103340005252525252525B5B5252525B5B5229298B
:103350002929292929295B5B525252525252525231
:1033600052525B525B5B52525B5B52525252525210
:10337000525252525252525B525252525B5B525212
:103380005252525B52525252525252525252292966
:103390002929292929290000000000000000000037
:1033A000000000000000000000000000000000001D
:1033B000000000000000000000000000000000000D
:1033C00000000000000000000000000000000000FD
:1033D00000000000000000000000000000003F3F6F
:1033E0000000000000003F3F00003F000000000020
:1033F000003F0000000000003F0000000000003F10
:103400000000000000003F00003F3F0000000000FF
:10341000003F3F000000000000000000000000002E
:1034200000003F3F00000000003F000000000000DF
:103430003F000000000000003F000000000000000E
:103440003F00000000000000003F000000000000FE
:1034500000003F3F000000000000000000000000EE
:103460003F3F00000000000000003F00000000009F
:103470000000003F000000000000003F00000000CE
:103480000000003F0000000000003F0000000000BE
:103490003F3F0000000000000000000000000000AE
:1034A0003F3F3F000000003F3F003F3F00003F3FE5
:1034B0000000003F3F003F3F0000003F3F003F3F14
:1034C0003F3F3F3F3F003F3F0000003F3F003F3F47
:1034D0000000003F3F0000000000000000003F3FF0
:1034E0003F3F3F3F00003F3F0000003F3F003F3F66
:1034F0000000003F3F003F3F3F3F3F3F00003F3F56
:103500000000003F3F003F3F0000003F3F003F3FC3
:103510003F3F3F3F000000000000000000000000AF
:103520003F3F3F3F0000003F3F00003F3F003F3F25
:103530000000000000003F3F0000000000003F3F8F
:10354000000000000000003F3F00003F3F0000007F
:103550003F3F3F3F000000000000000000003F3FF1
:103560003F3F3F0000003F3F00003F3F00003F3F24
:103570000000003F3F003F3F0000003F3F003F3F53
:103580000000003F3F003F3F00003F3F00003F3F43
:103590003F3F3F00000000000000000000003F3FF0
:1035A0003F3F3F3F3F003F3F0000000000003F3FE4
:1035B0000000000000003F3F3F3F3F3F00003F3F13
:1035C0000000000000003F3F0000000000003F3FFF
:1035D0003F3F3F3F3F0000000000000000003F3F32
:1035E0003F3F3F3F3F003F3F0000000000003F3FA4
:1035F0000000000000003F3F3F3F3F3F00003F3FD3
:103600000000000000003F3F0000000000003F3FBE
:1036100000000000000000000000000000000000AA
:103620003F3F3F3F3F00003F3F00000000003F3F63
:103630000000000000003F3F00003F3F3F003F3FD1
:103640000000003F3F00003F3F00003F3F00000000
:103650003F3F3F3F3F0000000000000000003F3FB1
:103660000000003F3F003F3F0000003F3F003F3F62
:103670000000003F3F003F3F3F3F3F3F3F003F3F95
:103680000000003F3F003F3F0000003F3F003F3F42
:103690000000003F3F000000000000000000003F6D
:1036A0003F3F3F3F3F000000003F3F000000000061
:1036B000003F3F0000000000003F3F00000000000E
:1036C000003F3F0000000000003F3F000000003FBF
:1036D0003F3F3F3F3F0000000000000000000000AF
:1036E000003F3F3F3F00000000003F3F0000000060
:1036F00000003F3F0000000000003F3F00000000CE
:1037000000003F3F00003F0000003F3F0000003F3F
:103710003F3F3F00000000000000000000003F3F6E
:103720000000003F3F003F3F00003F3F00003F3FA1
:10373000003F3F0000003F3F3F3F000000003F3F91
:103740003F3F3F0000003F3F003F3F3F00003F3F03
:1037500000003F3F3F000000000000000000003F6D
:103760003F0000000000003F3F0000000000003F5D
:103770003F0000000000003F3F0000000000003F4D
:103780003F0000000000003F3F0000000000003F3D
:103790003F3F3F3F3F0000000000000000000000EE
:1037A0003F3F3F000000003F00003F3F00003F3F21
:1037B0000000003F3F003F3F0000003F3F003F3F11
:1037C0000000003F3F00003F3F00003F00000000BE
:1037D0003F3F3F000000000000000000000000002C
:1037E000003F3F00000000003F3F3F00000000009E
:1037F000003F3F0000000000003F3F0000000000CD
:10380000003F3F0000000000003F3F000000003F7D
:103810003F3F3F3F3F000000000000000000003F2E
:103820003F3F3F3F00003F3F0000003F3F000000A0
:1038300000003F3F3F0000003F3F3F3F0000003F90
:103840003F3F3F0000003F3F3F00000000003F3F80
:103850003F3F3F3F3F000000000000000000003FEE
:103860003F3F3F3F3F00000000003F3F000000009F
:10387000003F3F00000000003F3F3F3F00000000CE
:103880000000003F3F003F3F0000003F3F00003F7F
:103890003F3F3F3F0000000000000000000000002C
:1038A000003F3F3F000000003F3F3F3F0000003F20
:1038B0003F003F3F00003F3F00003F3F00003F3FD1
:1038C0003F3F3F3F3F00000000003F3F000000003F
:1038D00000003F3F000000000000000000003F3FEC
:1038E0003F3F3F3F00003F3F0000000000003F3FE0
:1038F0003F3F3F3F000000000000003F3F0000004E
:103900000000003F3F003F3F0000003F3F00003FFE
:103910003F3F3F3F000000000000000000000000AB
:103920003F3F3F3F0000003F3F00000000003F3F9F
:103930000000000000003F3F3F3F3F3F00003F3F8F
:103940000000003F3F003F3F0000003F3F00003FBE
:103950003F3F3F3F000000000000000000003F3FED
:103960003F3F3F3F3F003F3F0000003F3F00000020
:1039700000003F3F00000000003F3F00000000004B
:103980003F3F0000000000003F3F0000000000003B
:103990003F3F000000000000000000000000003F6A
:1039A0003F3F3F0000003F3F0000003F00003F3F1F
:1039B0003F00003F0000003F3F3F3F0000003F004E
:1039C000003F3F3F3F003F000000003F3F00003FFF
:1039D0003F3F3F3F00000000000000000000003FAC
:1039E0003F3F3F3F00003F3F0000003F3F003F3F61
:1039F0000000003F3F00003F3F3F3F3F3F000000CF
:103A00000000003F3F00000000003F3F0000003F7B
:103A10003F3F3F00000000000000000000000000E9
:103A200000000000000000003F3F00000000000018
:103A30003F3F000000000000000000000000000008
:103A40003F3F0000000000003F3F0000000000007A
:103A500000000000000000000000000000003F3FE8
:103A60000000003F3F003F3F3F003F3F3F003F3FE0
:103A70003F3F3F3F3F003F3F3F3F3F3F3F003F3FD4
:103A8000003F003F3F003F3F0000003F3F003F3FFF
:103A90000000003F3F0000000000000000003F3F2A
:103AA0000000003F3F003F3F3F00003F3F003F3FDF
:103AB0003F3F003F3F003F3F3F3F3F3F3F003F3FD3
:103AC000003F3F3F3F003F3F00003F3F3F003F3F41
:103AD0000000003F3F000000000000000000003F29
:103AE0003F3F3F3F00003F3F0000003F3F003F3F60
:103AF0000000003F3F003F3F0000003F3F003F3FCE
:103B00000000003F3F003F3F0000003F3F00003FFC
:103B10003F3F3F3F000000000000000000003F3F2B
:103B20003F3F3F3F00003F3F0000003F3F003F3F1F
:103B30000000003F3F003F3F0000003F3F003F3F8D
:103B40003F3F3F3F00003F3F0000000000003F3F7D
:103B50000000000000000000000000000000003F26
:103B60003F3F3F3F00003F3F0000003F3F003F3FDF
:103B70000000003F3F003F3F0000003F3F003F3F4D
:103B8000003F3F3F3F003F3F00003F3F0000003FFE
:103B90003F3F3F003F0000000000000000003F3FAB
:103BA0003F3F3F3F00003F3F0000003F3F003F3F9F
:103BB0000000003F3F003F3F00003F3F3F003F3FCE
:103BC0003F3F3F0000003F3F003F3F3F00003F3F7F
:103BD00000003F3F3F000000000000000000003FE9
:103BE0003F3F3F0000003F3F00003F3F00003F3F9E
:103BF000000000000000003F3F3F3F3F000000008A
:103C00000000003F3F003F3F0000003F3F00003FFB
:103C10003F3F3F3F00000000000000000000003F69
:103C20003F3F3F3F3F000000003F3F0000000000DB
:103C3000003F3F0000000000003F3F000000000088
:103C4000003F3F0000000000003F3F000000000078
:103C5000003F3F00000000000000000000003F3F68
:103C60000000003F3F003F3F0000003F3F003F3F5C
:103C70000000003F3F003F3F0000003F3F003F3F4C
:103C80000000003F3F003F3F0000003F3F00003F7B
:103C90003F3F3F3F000000000000000000003F3FAA
:103CA0000000003F3F003F3F0000003F3F003F3F1C
:103CB0000000003F3F003F3F3F003F3F3F00003FCD
:103CC0003F3F3F3F000000003F3F3F00000000003B
:103CD000003F0000000000000000000000003F3F27
:103CE0000000003F3F003F3F0000003F3F003F3FDC
:103CF000003F003F3F003F3F3F3F3F3F3F003F3FD0
:103D00003F3F3F3F3F003F3F3F003F3F3F003F3F80
:103D10000000003F3F0000000000000000003F3FA7
:103D20000000003F3F003F3F3F003F3F3F00003F5C
:103D30003F3F3F3F000000003F3F3F000000003F8B
:103D40003F3F3F3F00003F3F3F003F3F3F003F3F7F
:103D50000000003F3F000000000000000000003FA6
:103D60003F00003F3F00003F3F00003F3F00003F5B
:103D70003F00003F3F0000003F3F3F3F000000008A
:103D8000003F3F0000000000003F3F000000000037
:103D9000003F3F00000000000000000000003F3F27
:103DA0003F3F3F3F3F00000000003F3F3F0000001B
:103DB000003F3F3F000000003F3F3F000000003F4A
:103DC0003F3F000000003F3F3F00000000003F3F3A
:103DD0003F3F3F3F3F00000000000000003F000069
:103DE0003F3F3F003F00003F3F003F3F00003F3F5D
:103DF0000000003F3F003F3F0000003F3F003F3FCB
:103E00003F3F3F3F3F003F3F0000003F3F003F3FFD
:103E10000000003F3F00FEFE05050505FEFEFE0515
:103E2000FF0505FF05FE0005050505050500000564
:103E3000FFFFFFAD0500FE05FFFFADAD05FE000570
:103E40000505050505000005FFFFFFAD0500FE05A2
:103E50000505050505FEFEFE000005FFFEFEFEFE53
:103E600000FFFF0505FE000005FFFFFF05FF000541
:103E70000505FFFFAD0505FFFF0505ADAD00050517
:103E8000FFAD05050000FE0505AD0500FEFEFEFECA
:103E900005050000FEFEFE0000FE0000FEFE05051A
:103EA0000505050505FE05FF05FFFF05FF0505FFE7
:103EB00005FFFF05050505FF05FFAD05050505AD7A
:103EC00005ADAD05FF0505050505050505FEFE006B
:103ED00000FE0000FEFEFEFE05050000FEFEFE05E3
:103EE00005AD0500FEFE0505FFAD0505000005FF5B
:103EF000FF0505ADAD0000050505FFFFAD050000A0
:103F000005FFFFFF05FFFEFE00FFFF0505FEFEFEAD
:103F1000000005FFFEFEFE050505050505FE000582
:103F2000FFFFFFAD05000005050505050500FE05C1
:103F3000FFFFFFAD05FE0005FFFFADAD050000056D
:103F4000050505050500FE05FF0505FF05FEFEFE4E
:103F500005050505FEFEFEFE7F7F7F7FFEFEFE7FE0
:103F6000FF7F7FFF7FFE007F7F7F7F7F7F00007F5F
:103F7000FFFFFFAD7F00FE7FFFFFADAD7FFE007F47
:103F80007F7F7F7F7F00007FFFFFFFAD7F00FE7F91
:103F90007F7F7F7F7FFEFEFE00007FFFFEFEFEFE36
:103FA00000FFFF7F7FFE00007FFFFFFF7FFF007F9E
:103FB0007F7FFFFFAD7F7FFFFF7F7FADAD007F7F06
:103FC000FFAD7F7F0000FE7F7FAD7F00FEFEFEFE27
:103FD0007F7F0000FEFEFE0000FE0000FEFE7F7FF1
:103FE0007F7F7F7F7FFE7FFF7FFFFF7FFF7F7FFFE2
:103FF0007FFFFF7F7F7F7FFF7FFFAD7F7F7F7FAD75
:104000007FADAD7FFF7F7F7F7F7F7F7F7FFEFE0065
:1040100000FE0000FEFEFEFE7F7F0000FEFEFE7F33
:104020007FAD7F00FEFE7F7FFFAD7F7F00007FFFC3
:10403000FF7F7FADAD00007F7F7FFFFFAD7F000082
:104040007FFFFFFF7FFFFEFE00FFFF7F7FFEFEFE84
:1040500000007FFFFEFEFE7F7F7F7F7F7FFE007F71
:10406000FFFFFFAD7F00007F7F7F7F7F7F00FE7FB0
:10407000FFFFFFAD7FFE007FFFFFADAD7F00007F44
:104080007F7F7F7F7F00FE7FFF7F7FFF7FFEFEFEC3
:104090007F7F7F7FFEFE0002060000FB00FF000224
:1040A000090000F100FF0002090000FE00FF00010E
:1040B000050000E219010302050000FF00010000F5
:1040C00000E232010102050000FF0001280000FEAD
:1040D000FA010102050000FF0001000000FB96014B
:1040E0000302050000FF0001000000E20F010302CF
:1040F000050000FF0001030000F64B01030205006C
:1041000000FF0001020000EC1901FF03050000FFA1
:104110000001FF0000CE0501FF03050000FF0002C3
:104120000800085504085A0000F8000990000A1E0B
:1041300032050000FF000000964000000000000073
:10414000009E4000000000000000A64000000000AB
:10415000010000AE4000000000010000BC40000073
:104160000000010000CA4000000000010000D8402B
:1041700000000000010000E6400000000001000017
:10418000F4400000000001000002410000000001B6
:1041900000001041000000000000001E410000006F
:1041A0000000FF06015300B0077F005C00000B7F9A
:1041B00000C0010090214000B1077F005C00000BAF
:1041C0007F00C10000912D400F90214000913040B0
:1041D0000F902140009132400F90214000913440D7
:1041E00010902140009145400F902140009148409F
:1041F0000F90214000914040109021400091434099
:104200000F902140009132400F90214000913440A6
:1042100010901F40009137400F901E400091394090
:104220000F90214000913C401090214000913E4071
:104230000F902140009137400F902140009139406C
:1042400010902140009140400F9021400091434048
:104250000F90214000914540109021400F214000D7
:104260009145400F9021400091484010901F400F11
:104270001E40009148400F90214000914A4010900C
:1042800021400F21400F214010214000914A400F52
:10429000902140009149400F9021400091484010EA
:1042A000902140009147400F902140009145400FE0
:1042B0009021400091444010901F40009143400FD6
:1042C000901E40009140400F90214000913E4010D0
:1042D00090214000913C400F9021400F214010213F
:1042E000400F21400F21401021400F2140009145F7
:1042F000400F9021400091484010901F4000914095
:10430000400F901E40009143400F32400F33401049
:1043100034401E41401042400F43400F444010487B
:10432000400F45402E9021400F21401021400F2189
:10433000400F21401021400F21400F21401021400B
:104340000F21400F1F40101E400F21400F21401031
:1043500021400F21400F21401021400F21400F210B
:10436000401021400F21400F1F40101E400F2140E0
:1043700000912B400F90214000912D401090214042
:10438000009130400F902140009132400F90214029
:104390000091454010902140009143400F902140F2
:1043A000009140400F90214000913E4010902140EC
:1043B000009130400F902140009132400F901F40FB
:1043C000009134400F901E400091374010902140E2
:1043D000009140400F90214000913E400F902140BD
:1043E000009139401090214000913C400F902140B5
:1043F000009134400F9021400091374010902140AF
:10440000009139400F90214000913C400F90214095
:10441000009139401090214000913C400F901F4086
:10442000009134400F901E40009137401090214081
:1044300000912D400F90214000912E400F9021407F
:1044400000912F4010902140009130400F9021406A
:10445000009132400F902140009133401090214054
:10446000009134400F902140009137400F9021403F
:1044700000913940109021400F1F400F1E40102125
:1044800040009139400F90214000913C400F902115
:10449000401021400F214000913C400F90214000EE
:1044A000913F40109021400F21400F2140102140AA
:1044B0000F1F400F1E401021400F21400F214010C0
:1044C00021400F21400F21401021400F21400F219A
:1044D000400F2140101F400F1E400F214000913718
:1044E0004010902140009139400F902140009137B9
:1044F000400F90214000913940109021400F214001
:104500000F21401021400F2140009140400F902189
:10451000400091404010901F40009140400F901E7D
:1045200040009140400F9021400091434010902165
:1045300040009143400F902140009143400F902153
:10454000400091434010902140009145400F902140
:1045500040009145400F902140009145401090212E
:1045600040009145400F902140009148400F90211C
:10457000400091484010901F40009148400F901E0D
:1045800040009148400F90214000914A40109021F6
:104590004000914A400F90214000914A400F9021E5
:1045A0004000914A401090214000914C400F9021D2
:1045B0004000914E400F90214000914F40109021BB
:1045C00040009151400F9021400F2140101F400F9B
:1045D0001E400FFF06014500FF2F0000B0076F00CF
:1045E0005C00000B7F00C00000FF06015300902D0F
:1045F0004000B1077F005C00000B7F00C10200910A
:1046000021400F902D400F3440009124400F902DF9
:10461000400091214010902D40009121400F902D9D
:1046200040009121400F9034400091284010902D7F
:104630004000912B400F9042400091214004904057
:1046400040033E40043B40043B40043940043740B3
:104650000436400334400091244004903240042D3D
:1046600040089121400F214008902B4007912140A4
:104670001028400790374004394004374000912B00
:104680004004903240043440033240042D400091F5
:1046900021400F902D40103440009124400F902D68
:1046A00040009121400F902D400091214010902D0D
:1046B00040009121400F903440009128400F902DF0
:1046C0004000912B4010902D40009121400F902DE3
:1046D000400F2D400091244008902F40072D4000AE
:1046E00091214008902F40083240009121400790CE
:1046F0002F4008324000912140089034400732405A
:10470000009128400890344008364000912B400723
:10471000903440082D40009121400F902D400F34DF
:10472000400091244010902D40009121400F902D89
:1047300040009121400F902D400091214010903475
:1047400040009128400F902D4000912B400F904247
:10475000400091214004904040043E40043B40040E
:104760003B40033940043740043640043440009154
:10477000244004903240032D40089121400F2140F5
:1047800008902B40089121400F28400890374003A3
:10479000394004374000912B4004903240043440AB
:1047A000043240042D40009121400F902D400F34E1
:1047B00040009124400F902D400091214010902DF9
:1047C00040009121400F902D40009121400F9034E6
:1047D000400091284010902D4000912B400F902DCB
:1047E00040009121400F902D40102D400091244019
:1047F00007902F40082D400091214007902F40083E
:1048000032400091214008902F4007324000912112
:1048100040089034400832400091284007903440CE
:1048200008364000912B40089034400734400091F6
:1048300021403D90324000911F403E903140009118
:104840001E403D90284000911C401E902B4000913E
:104850001F401F903440009121403D903240009114
:104860001F403D90314000911E403D9028400091F6
:104870001C401F902B4000911F401F903940009119
:1048800026403D903B40009128403D903E400091A5
:104890002B403D90404000912D403D90394000918B
:1048A00026403E903B40009128403D903E40009184
:1048B0002B403D90404000912D403D902D40009177
:1048C00021400F902D40103440009124400F902D36
:1048D00040009121400F902D40009121400F902DDC
:1048E000400091214010903440009128400F902DBD
:1048F0004000912B400F9042400091214004904095
:1049000040043E40043B40043B40033940043740F0
:104910000436400434400091244004903240042D79
:10492000400791214010214007902B4008912140E1
:104930000F28400890374004394003374000912B3E
:104940004004903240043440043240042D40009131
:1049500021400F902D400F34400091244010902DA5
:1049600040009121400F902D40009121400F902D4B
:1049700040009121400F9034400091284010902D2C
:104980004000912B400F902D40009121400F902D21
:1049900040102D400091244007902F40082D4000EA
:1049A00091214008902F400732400091214008900B
:1049B0002F40083240009121400790344008324097
:1049C000009128400790344008364000912B400861
:1049D000903440072D400091214010902D400F341D
:1049E00040009124400F902D400091214010902DC7
:1049F00040009121400F902D40009121400F9034B4
:104A000040009128400F902D4000912B4010904283
:104A1000400091214004904040033E40043B40044C
:104A20003B40043940043740043640033440009191
:104A3000244004903240042D40089121400F214031
:104A400008902B40079121401028400790374004E0
:104A5000394004374000912B4004903240033440E9
:104A6000043240042D40009121400F902D4010341D
:104A700040009124400F902D40009121400F902D37
:104A8000400091214010902D40009121400F903422
:104A900040009128400F902D4000912B400F902D09
:104AA000400091214010902D400F2D400091244056
:104AB00008902F40072D400091214008902F40087A
:104AC00032400091214007902F4008324000912150
:104AD000400890344007324000912840089034400C
:104AE00007364000912B4008903440083440009134
:104AF00021403D90324000911F403D903140009157
:104B00001E403D90284000911C401F902B4000917A
:104B10001F401E903440009121403E903240009151
:104B20001F403D90314000911E403D902840009133
:104B30001C401F902B4000911F401E903940009157
:104B400026403D903B40009128403E903E400091E1
:104B50002B403D90404000912D403D9039400091C8
:104B600026403D903B40009128403D903E400091C2
:104B70002B403D90404000912D403E90434000919D
:104B800021401E904340009124400F21401090434B
:104B900040009121400F21400F904040009128405B
:104BA000102B400F903E40009124401E904040004A
:104BB0009128401024400F904340009124400F243E
:104BC000401090404000912B400F2F400F903E40EE
:104BD000009126401F90404000912A400F26400F30
:104BE000904340009126401026400F904040009195
:104BF0002D400F304010903940009126403D9030BC
:104C000040009124401E902F40009123401F90436C
:104C100040009121401F904840009124400F2140C6
:104C20000F904A40009121400F21401028400F2B47
:104C3000400F904A40009124401F90484000912826
:104C4000400F24400F904340009124401024400F17
:104C500090404000912B400F2F4010903E4000911B
:104C600026401E903C4000912A400F26401090376D
:104C700040009126400F26400F90394000912D4072
:104C80001030400F903940009126403D9030400058
:104C90009124401F902F40009123401E90454000DA
:104CA0009121400590434005404006454005434062
:104CB0000540400545400091244005904340054093
:104CC0004005454000912140059043400540400586
:104CD0004A400091214006904840054540054A4021
:104CE0000091214005904840054540054A4000910B
:104CF000284005904840054540054A4000912B401A
:104D000005904840064540054840009124400590E4
:104D1000454005434005484005454005434005489A
:104D2000400091284005904540054340064840001A
:104D300091244005904540054340054A4000912498
:104D40004005904840054540054A400091244005F3
:104D5000904840054540054A4000912B4006904848
:104D600040054540054A4000912F400590484005C8
:104D70004540054540009126400590434005404090
:104D800005454005434005404006454000912A4006
:104D90000590434005404005454000912640059060
:104DA0004340054040054A40009126400590484058
:104DB000054540054A40009126400690484005457B
:104DC00040054A4000912D4005904840054540056A
:104DD0004A40009130400590484005454005484014
:104DE0000091264005904540064340054840054552
:104DF00040054340054840054540054340054840BF
:104E0000054540054340064A40009124400590482E
:104E100040054540054A40054840054540054A4093
:104E20000091234005904840054540054A4005480B
:104E300040064540054540009121407AFF06014566
:104E400000FF2F0000B00758005C00000B7F0090AF
:104E5000244000FF06015300C00100B1077F005C41
:104E600000000B7F00C10013902440009140400ED1
:104E700090244005244000914040099024400A2499
:104E800040009143400A90244000914540099027FA
:104E900040009145400A9027400927400091474033
:104EA0000A9027400A914740099027400A2740006E
:104EB00091474013902940009147400A90294009AA
:104EC00029400A29401329400A29400929400A2972
:104ED00040009145400943400A90294000914040DC
:104EE0000A434009902440132440009140400F9011
:104EF000244005244000914040099024400A244069
:104F00000091434009902440009145400A90274079
:104F1000009145400A902740092740009147400AE8
:104F2000902740099147400A9027400A2740009166
:104F300047401390294000914740099029400A2991
:104F4000400A29401329400929400A29400A2940DA
:104F5000009145400947400A90294000914A400984
:104F600047400A902440132440009140400F902471
:104F700040042440009140400A9024400A2440000C
:104F800091434009902440009145400A90274000F9
:104F9000914540099027400A2740009147400A90D8
:104FA0002740099147400A90274009274000914730
:104FB000401490294000914740099029400A294017
:104FC0000929401429400929400A2940092940009B
:104FD0009145400A43400A902940009140400943CE
:104FE000400A902440132440009140400E902440F9
:104FF000052440009140400A90244009244000913B
:1050000043400A902440009145400A902740009177
:105010004540099027400A274000914740099027C2
:10502000400A9147400A9027400927400091474095
:1050300013902940009147400A9029400A294009CD
:1050400029401329400A29400A29400929401329E7
:105050004014244000914F40044C40054840054313
:10506000400590244000914840054C40044F4005C5
:1050700090244000914C4005902440009148400508
:1050800043400590244000914840044C4005902442
:105090004000914F40054C4005902440009148400D
:1050A0000543400490274000915240054F40059031
:1050B000274000914B400546400590274000914B0A
:1050C00040044F400590274000915240054F400555
:1050D0004B400546400490274000914B40054F400F
:1050E0000590274000915240054F40054B40044633
:1050F00040059029400091544005514005902940B9
:1051000000914D400548400490294000914D4005D4
:1051100051400590294000915440055140054D40B3
:105120000448400590294000914D400551400590AC
:105130002940009154400551400490294000914D70
:105140004005484005902940009154400A514009CB
:1051500090294000914D400A484009902440009118
:105160004F40054C40054840054340059024400011
:10517000914840044C40054F400590244000914C1C
:10518000400590244000914840054340049024404D
:1051900000914840054C400590244000914F400547
:1051A0004C4005902440009148400443400590271E
:1051B0004000915240054F400590274000914B40E0
:1051C0000546400490274000914B40054F40059014
:1051D000274000915240054F40054B400446400592
:1051E00090274000914B40054F400590274000918B
:1051F0005240054F40044B40054640059029400071
:105200009154400551400590294000914D4004487B
:10521000400590294000914D40055140059029409E
:1052200000915440055140044D40054840059029E7
:105230004000914D40055140059029400091544057
:105240000451400590294000914D4005484005908B
:105250002940009154400951400A90294000914C46
:10526000400A4F400990244000914F40054C4005B2
:1052700048400543400490244000914840054C407C
:10528000054F400590244000914C4005902440007B
:105290009148400443400590244000914840054C0B
:1052A000400590244000914F40054C40049024401C
:1052B0000091484005434005902740009152400529
:1052C0004F400590274000914B40044640059027F1
:1052D0004000914B40054F400590274000915240BF
:1052E000054F40044B400546400590274000914B38
:1052F00040054F400590274000915240044F400523
:105300004B400546400590294000915440055140CE
:105310000490294000914D400548400590294000E7
:10532000914D400551400590294000915440045151
:1053300040054D400548400590294000914D4005ED
:105340005140049029400091544005514005902956
:105350004000914D4005484005902940009154403F
:105360000951400A90294000914D400948400A9057
:10537000244000914F40054C4005484004434005FF
:1053800090244000914840054C40054F4005902432
:105390004000914C40049024400091484005434017
:1053A0000590244000914840054C40059024400061
:1053B000914F40044C4005902440009148400543E3
:1053C000400590274000915240054F4004902740EF
:1053D00000914B400546400590274000914B400509
:1053E0004F400590274000915240044F40054B40EC
:1053F0000546400590274000914B40054F400490E2
:10540000274000915240054F40054B40054640055E
:10541000902940009154400451400590294000914A
:105420004D400548400590294000914D40055140B0
:105430000490294000915440055140054D400548D5
:10544000400590294000914D40045140059029406D
:10545000009154400551400590294000914D400570
:1054600048400490294014294013FF06014500FFDD
:105470002F0000B0077F005C00000B7F00C0000021
:1054800090375F00B1077F005C00000B7F00C10117
:105490000890375F08375F08395F083B5F11375F57
:1054A000083C5F11375F00911F5F0890435F0091D8
:1054B0002B5F21235F08235F08FF2F0000B00767E1
:1054C000005C00000B7F00C0000090515F0A495F44
:1054D0000A4C5F0A515F0A485F0A4C5F0B515F0A32
:1054E000475F0A4A5F0A515F0A465F0B495F0A47F6
:1054F0005F1EFF2F0000B1077F005C00000B7F00E4
:10550000C10000FF0601530091265F00B0077F0035
:105510005C00000B7F00C0001091265F08245F092B
:10552000265F10265F08245F09265F10265F082982
:105530005F15295F15265F10265F08245F09265F27
:1055400010265F08245F09265F10265F082B5F1571
:105550002B5F15265F10265F08245F09265F102643
:105560005F08245F09265F10265F08295F15295F01
:1055700015265F10265F08245F09265F10265F0846
:10558000245F09265F10265F082B5F152B5F152609
:105590005F10265F08245F09265F10265F08245FDE
:1055A00009265F10265F08295F15295F15265F1001
:1055B000265F08245F09265F10265F08245F0926FE
:1055C0005F10265F082B5F2A245F08265F10225F8A
:1055D00009245F10245F09265F18215F09225F08F4
:1055E000265F08245F08265F09245F08295F0826D4
:1055F0005F3A245F08265F11225F082E5F10245F48
:1056000009305F18215F09225F08265F08245F08C0
:10561000265F09245F08295F08265F3A245F082671
:105620005F11225F08245F10245F09265F18215F45
:1056300009225F08265F08245F08265F09245F08A7
:10564000245F08295F08265F32245F08265F112245
:105650005F082E5F10245F09305F18215F09225F09
:1056600008225F08245F08225F09245F08225F0880
:10567000295F08265F321F5F00903F5F0891215F1E
:1056800000903E5F083C5F0991245F00903B5F08FB
:1056900091215F21215F0090415F0891235F00907D
:1056A0003F5F093E5F0891265F00903C5F089123B1
:1056B0005F211F5F0090435F0891215F0090415F71
:1056C000093F5F0891245F00903E5F0891215F21B0
:1056D000215F0090445F0891235F0090435F094180
:1056E0005F0891265F00903F5F0891235F21235F51
:1056F00000903F5F0891245F00903E5F093C5F0887
:1057000091275F00903B5F0891245F21245F009008
:10571000415F0891265F00903F5F093E5F08912935
:105720005F00903C5F0891265F21235F0090435FFC
:105730000891245F0090415F093F5F0891275F0057
:10574000903E5F0891245F21245F0090465F08919E
:10575000265F0090445F09435F0891295F009041F4
:105760005F0891265F21245F08265F11225F0824CD
:105770005F11245F08265F19215F08225F08265FFA
:1057800008245F09265F08245F08295F08265F3A1E
:10579000245F08265F11225F082E5F11245F083006
:1057A0005F19215F08225F08265F08245F09265FD2
:1057B00008245F08295F08265F3A245F09265F10E6
:1057C000225F08245F11245F08265F19215F0822E9
:1057D0005F08265F09245F08265F08245F08245FAE
:1057E00009295F08265F31245F09265F10225F08C0
:1057F0002E5F11245F08305F19215F08225F0822A5
:105800005F09245F08225F08245F08225F09295F7F
:1058100008265F31245F09265F10225F08245F118C
:10582000245F08265F0890325F42305F4291245F18
:1058300009265F08245F10265F09295F08265F108C
:10584000902E5F322B5F10305F4391245F08265FFC
:1058500008265F08265F09245F08295F08265F1174
:1058600090325F312B5F11305F4291245F08265FD9
:1058700010225F092E5F10245F08305F0990305FAF
:10588000312B5F11355F10325F32FF06014500FF9B
:105890002F000D1EC8D716E7F432000000000000EC
:1058A0001032C87D0DD41FF3000000000000131655
:1058B000DC02CB7DEBFEF0E9000000001400CD7BA4
:1058C0007AEB9A992900000000000C20FCEACDDE5A
:1058D000FA1F0000000000001D15DC010272E1E962
:1058E0009B2B8EFAE8001514C829850C05E0F5FD00
:1058F00000000000112B917201DCE8320000000072
:1059000000001C167BCC7DEB9AE9988C796F000027
:105910001632FCEAFF7CCDDF0BC81F000000555A91
:1059200045424F5800434F5252494441204E454250
:105930004F534F53410050524553532053544152FB
:105940005400284329203230313020464CC3815640
:10595000494F205A4156414E003120504C41594543
:1059600052003220504C4159455253004F50544937
:105970004F4E5300545241434B20454449544F52DB
:10598000004352454449545320414E44204C49431E
:10599000454E53455300444946464943554C545996
:1059A0003A0045415359004D454449554D00484141
:1059B000524400484F524E3A0043415220434F4C0C
:1059C0004C4953494F4E533A004E4954524F3A00B6
:1059D0004F4E004F4646004D555349433A005346FB
:1059E000583A00534F554E4420544553543A0043BF
:1059F0004C45415220454550524F4D20284C205295
:105A000020414E4420422900454550524F4D2043ED
:105A10004C454152454400594F55204C4F53450089
:105A200053545245455400594F552057494E004E46
:105A3000454220524F414400484947485741590088
:105A40004D454E550054494C45202020202000450E
:105A500052524F522020202000454550524F4D2099
:105A6000202000474F2020202020202000524541A8
:105A70004459205345540042554D502020202020A9
:105A800000484F524E2020202020004E4954524FB3
:105A900020202020004B4C494E472020202000543D
:105AA0004945442020004649525354200053454361
:105AB0004F4E440057494E4E4552004C4F534552AD
:105AC00020004C3A203A004E3A2020202500504138
:105AD0005553454400524553554D45005155495481
:105AE0000044454D4F0053454C20524556455253B6
:105AF0004500545241434B00435553544F4D004CC5
:105B000041505300545241434B2053415645442089
:105B1000494E20534C4F54004E4F2046524545208D
:105B2000534C4F5453005245504C4143452043552C
:105B300053544F4D20545241434B0043414E434533
:105B40004C005341564500545241434B20434F4D66
:105B5000504C45544544005752495454454E2042F8
:105B60005920464CC38156494F205A4156414E0058
:105B70004C4943454E53454420554E4445522054CC
:105B8000484500474E552047504C205633204F5231
:105B9000204E4557455200435245415449564520F1
:105BA000434F4D4D4F4E530041545452494255546A
:105BB000494F4E20534841524520414C494B4500E6
:105BC000563320554E504F52544544204C4943457E
:105BD0004E53450043415253204C4F474F20414EB6
:105BE000442054484520534F4E4753004D454E5591
:105BF00020524F414420414E442053545245455475
:105C0000004259204C5543415320534552555200B0
:105C10005346582054494C4553455420414E442046
:105C2000594F552057494E00425920464CC3815682
:105C3000494F205A4156414E00484947485741591B
:105C400020414E4420594F55204C4F535420425927
:105C50000049444552414C444F204C55495320443F
:105C6000412053494C56410011241FBECFEFD0E1D3
:105C7000DEBFCDBF14BE88E10FB6F89480936000FC
:105C8000109260000FBE12E0A0E0B1E0EEE3F9EE8A
:105C900002C005900D92A632B107D9F71BE0A0E42F
:105CA000B2E001C01D92A433B107E1F70E94F738BA
:105CB000882311F40E94D538F894E1E0F8E080E000
:105CC00090E03E2F2F2F40E84193019652E08C3018
:105CD0009507D1F730930D0A20930E0A10920F0A00
:105CE00081E08093260A8093270A8093250A1092E8
:105CF000120A1092180A10921E0A1092240A109288
:105D0000D40792E19093D50790EE9093DE0790939D
:105D1000DC0794E19093DD079093DB071092E20794
:105D20001092E1071092E6071092E5078093110A9E
:105D30000E94CD4480E090E0FC01EE0FFF1FE05692
:105D4000FF4F25913491F901F0703083019687312E
:105D5000910591F778940E94CC440E9486720C942D
:105D60009D740C94000006E00A95F1F7E2E9F7E073
:105D7000C0E4D2E02091B10A0027A081B181AC0F2C
:105D8000BD1F1C911283021708F4102F1C93339629
:105D90000395083090F307E316E01A95F1F70A959A
:105DA000D9F7C0E4D2E000EEA02E662778E07BD2DF
:105DB00034E23A95F1F7000000000E94052F3BE025
:105DC0003A95F1F7AA9489F06395C895683029F05F
:105DD000C895C895C8950000EACF662700243EE123
:105DE000C30FD01DC8950000E2CF35E03A95F1F71A
:105DF00000C059D211240E940044E1E0E093D6078C
:105E0000E2E0E093360011240895DE01679F000070
:105E10000091D0071091D10700501240000D111DC4
:105E2000180102E915E0000D111D280130E41EE102
:105E30002D9128306FB660FA239FA1010EF4A201C4
:105E4000040E151EF001F6F0059108B92D9105918B
:105E500008B9239F059108B928306FB6059108B994
:105E600008F4A201059108B960FA040E059108B979
:105E7000151E1A95059108B9059139F1F00108B977
:105E80001EF700C0019108B92D910191000008B9D9
:105E9000239F0191000008B928306FB660FA019184
:105EA00008B90EF0A1010191040E08B9151E00C039
:105EB000019108B9000000C0019108B901911A953B
:105EC00021F0F00108B906F6DDCF08B90027C89522
:105ED000000008B905E00A95F1F7089520E4E09183
:105EE000D007F091D1078850829FE00DF11DA2E903
:105EF000B5E0629FA00DB11D002405900D920590A4
:105F00000D9205900D9205900D9205900D920590C1
:105F10000D9205900D9205900D9205900D920590B1
:105F20000D9205900D9205900D9205900D920590A1
:105F30000D9205900D9205900D9205900D92059091
:105F40000D9205900D9205900D9205900D92059081
:105F50000D9205900D9205900D9205900D92059071
:105F60000D9205900D9205900D9205900D92059061
:105F70000D9205900D9205900D9205900D92059051
:105F80000D9205900D9205900D9205900D92059041
:105F90000D9205900D9205900D9205900D92059031
:105FA0000D9205900D9205900D9205900D92059021
:105FB0000D9205900D9205900D9205900D92059011
:105FC0000D9205900D9205900D9205900D92059001
:105FD0000D9205900D9205900D9205900D920590F1
:105FE0000D9205900D9205900D9205900D920590E1
:105FF0000D9205900D9205900D92112408950F9326
:106000001F9395E0899FE8E8F5E0E00DF11D04811C
:1060100082819381E0E48E9FD0019E9FB00D98E035
:10602000099FEAEAF7E00024E10DF01D00801180ED
:10603000F001EA0FFB1FA2E9B5E090E4699FA00D13
:10604000B11D1124403051F4A20FB11D822F122F27
:1060500000FF11C0379610E1121B0DC088E0821BB3
:1060600000FD04C0182FE80FF11D05C018E0120F45
:10607000E20FF11D3197503031F498E0939FA00D5D
:10608000B11D932F06C098E0931B58E0599FE00D77
:10609000F11D11243EEFE89400FD689458E0591B6F
:1060A00048E0481B3EF0259123132C9311964A9506
:1060B000D1F707C02491319723132C9311964A9559
:1060C000C9F7E10FF11DA80FB11D5A9549F7112429
:1060D0001F910F9108950F921F92EF93FF93EFB7C7
:1060E000EF93E0918400E251F1E0EF1700F0F395B7
:1060F000FA30D8F30C947C30E091D507EA95E09320
:10610000D507F091D407F0FD57C0EC3098F0F3E0DC
:10611000F0938900FDE8F0938800E0FB289826F4CE
:10612000E1E00E942F32B8C0E5E1EA95F1F7000006
:10613000289AB2C0E63038F100C000C02898E0FBD1
:10614000E4E016F40E942F32E4E0E0933600E6E04B
:10615000E0936F00A1C0EF93EFB7EF93E09184005D
:10616000ED55E13000F0E23000F0E33000F0E430D3
:1061700000F0E53000F0289AE2E0E0936F00EF9144
:10618000EFBFEF91189500C0E0FB289826F4E1E0FE
:106190000E942F3205C0E5E1EA95F1F70000289A48
:1061A000E091D507E03009F077C0EDEFE093D50737
:1061B000E1E0E093D40770C0E7E0E0938900EBE111
:1061C000E093880000C02898E2E000C00E942F32CF
:1061D000FDEF0090DB07F019E091D507EF17E0F431
:1061E000FDEF0090DB07F0190090DC07F019EF17C6
:1061F00098F0EDE1FF2700800F92EA95E1F70FE1BB
:106200000A95F1F7000000000E94B32EE1E0FF279D
:106210000F900192EE31E0F3E091D507E03009F004
:106220003BC02F933F934F935F936F937F938F93D5
:106230009F93AF93BF9378941124EE27E093D407F4
:10624000E2E1E093D507F091DD07F093DB07F091F1
:10625000DE07F093DC07E091D707F091D807E1154E
:10626000F10509F009950E94C4380E94D3440E94A8
:106270005E311124E091D907F091DA07E115F105BB
:1062800009F00995BF91AF919F918F917F916F9187
:106290005F914F913F912F91EF91EFBFFF91EF9160
:1062A0001F900F9018952898E2E000C00E942F32AE
:1062B000E091D507EA95E093D5070895E091110A9A
:1062C000E0FD0E949E3A00900F0A002019F4A1E020
:1062D000B8E002C0A7E0B9E021E0022600920F0A70
:1062E00022E02093100AE091110AE0FF08952F9216
:1062F0003F924F925F926F927F928F929F92AF9256
:10630000BF92CF92DF92EF92FF920F931F93CF93A2
:10631000DF935091240A6091260A7091270A809198
:10632000280A2090130A3090140A4090160A5090C0
:10633000170A6090150A1091120A7090190A80903D
:106340001A0A90901B0AA0901C0AB0901D0A209176
:10635000180AC0901F0AD090200AE090220AF090FC
:10636000230A0091210A30911E0A9FEF620C431C00
:10637000F2014491410300240008C12DD02D970C57
:10638000A81CF5014491420300240008C10DD01D52
:106390008A956AF44091250A842F8695062E0694E4
:1063A000062600FA7695679576F940FF66F940E88B
:1063B00060FD4FE7450300240008C10DD01D0024F7
:1063C000C038D0050CF0CFE70A94C038D0050CF4E3
:1063D000C0E8C058CD939A9509F0C8CF4091100AF3
:1063E0004A954093100A97E009F0C0CF6092150AD1
:1063F0004092160A90921B0AA0921C0A0093210A4E
:10640000E092220A6093260A7093270A8093280A52
:10641000DF91CF911F910F91FF90EF90DF90CF9080
:10642000BF90AF909F908F907F906F905F904F90B4
:106430003F902F900895E0910D0AF0910E0A01917E
:1064400000000093B3000AE0ED30F00701E018E02F
:1064500008F0F801E0930D0AF0930E0A08950F93E7
:106460001F932F93EF93E0910D0AF0910E0A019183
:106470000093B3000AE0ED30F00701E018E008F007
:10648000F801E0930D0AF0930E0AE8E0EA95F1F7BF
:10649000EF912F911F910F91E0FD289AE0FF01C02D
:1064A0000895F4E1FA95F1F700C0E1FD289AE1FFC3
:1064B00000C0089599277727833008F00895E8E011
:1064C000FCE7660F771FE60FF71FA591B491E2E195
:1064D000FAE026E0289FE00DF11DA183B28311248C
:1064E00008959091250A9170880F892B8093250A31
:1064F000089599277727E2E1FAE026E0289FE00D4A
:10650000F11D6E3F31F46091250A6E7F6093250A7C
:106510000BC06F3F31F46091250A6E6F6093250ABE
:1065200003C07EE7760F7583112408959927772796
:10653000E2E1FAE026E0289FE00DF11D60831124DE
:106540000895CF92DF92EF92FF920F931F936B010A
:106550007C0120E030E040E05FE40E943E3587FDB2
:1065600011C0C701B60120E030E040E05FE40E94C6
:106570005A340E94E6358B019C01005010402040A7
:10658000304806C0C701B6010E94E6358B019C0168
:10659000B801C9011F910F91FF90EF90DF90CF904C
:1065A0000895A0E0B0E0E7EDF2E30C948173EC0114
:1065B0004B01FA018881823008F442C1DB019C91D1
:1065C000923008F43AC1843059F4943009F038C15B
:1065D000998111968C911197981709F02BC130C1B0
:1065E000943009F42AC19230A9F4823009F028C10C
:1065F000CE0128E0DC010D90CD01DA010D92AD0154
:106600002150C1F7D40111968C911197998189235A
:10661000818315C1823009F410C1AA80BB80DB01DF
:1066200012964D915C911397CC80DD80EE80FF80B7
:1066300014960D911D912D913C911797C501841BC6
:10664000950BDC0197FF04C0AA27BB27A81BB90B39
:10665000A032B1050CF06AC0181619068CF5280195
:1066600039010A2E04C076946794579447940A948B
:10667000D2F741E050E060E070E004C0440F551FE5
:10668000661F771FAA95D2F7415050406040704076
:10669000402351236223732381E090E0A0E0B0E027
:1066A000411551056105710521F480E090E0A0E0FD
:1066B000B0E08C019D01042915292629372942C003
:1066C000009709F43FC0AA0EBB1E260137010A2E0F
:1066D00004C076946794579447940A94D2F741E0A3
:1066E00050E060E070E004C0440F551F661F771F44
:1066F000AA95D2F741505040604070404C215D2136
:106700006E217F2181E090E0A0E0B0E041155105CD
:106710006105710521F480E090E0A0E0B0E06C013B
:106720007D01C428D528E628F7280CC04A155B054A
:106730002CF400E010E020E030E004C05A01CC244A
:10674000DD2476018981D40111969C9111978917D6
:1067500009F445C0882329F00C191D092E093F09A9
:1067600008C0D701C601801B910BA20BB30B8C0193
:106770009D0137FD04C01182B382A2820BC081E06B
:106780008183B382A28230952095109501951F4F89
:106790002F4F3F4F04831583268337830DC0880F07
:1067A000991FAA1FBB1F84839583A683B783828109
:1067B000938101979383828384819581A681B78198
:1067C000AC01BD0141505040604070404F3F2FEF41
:1067D00052072FEF62072FE3720708F30BC0818384
:1067E000B382A2820C0D1D1D2E1D3F1D0483158337
:1067F0002683378383E08083448155816681778156
:1068000077FF1DC0DB01CA0181709070A070B0706D
:106810007695679557954795842B952BA62BB72B87
:1068200084839583A683B783828193810196938322
:10683000828305C0CAE1D1E003C0E40101C0EF01D9
:10684000CE01CDB7DEB7E0E10C949D73A0E2B0E0DD
:10685000ECE2F4E30C948F73DC01CB018D839E8317
:10686000AF83B88729833A834B835C83CE01059637
:10687000BE01675E7F4F0E946637CE010196BE0162
:106880006F5E7F4F0E946637CE014996BE016F5EF4
:106890007F4FAE01475F5F4F0E94D1320E948C361E
:1068A000462F572F682F792FCB01BA01A096E2E02F
:1068B0000C94AB73A0E2B0E0E0E6F4E30C948F73C9
:1068C000DC01CB018D839E83AF83B88729833A8314
:1068D0004B835C83CE010596BE01675E7F4F0E94AD
:1068E0006637CE010196BE016F5E7F4F0E9466370C
:1068F0008A8991E089278A8BCE014996BE016F5E15
:106900007F4FAE01475F5F4F0E94D1320E948C36AD
:10691000462F572F682F792FCB01BA01A096E2E0BE
:106920000C94AB73A8E1B0E0E8E9F4E30C9489734C
:10693000DC01CB018D839E83AF83B88729833A83A3
:106940004B835C83CE010596BE016F5E7F4F0E9434
:106950006637CE010196BE01675F7F4F0E946637A2
:106960009989923008F476C08985823008F475C020
:106970002A893A8523272A8B943011F0923021F40A
:10698000981709F067C06CC0843039F41D8A1E8ADC
:106990001F8A188E1C8A1B8A5DC0823019F484E01D
:1069A000898B58C02B893C898B859C85281B390B8A
:1069B0003C8B2B8B8D899E89AF89B88DCD84DE84ED
:1069C000EF84F8888C159D05AE05BF0540F4880F4F
:1069D000991FAA1FBB1F215030403C8B2B8BEFE12E
:1069E000F0E000E010E020E030E440E050E060E063
:1069F00070E08C159D05AE05BF0540F0402B512B76
:106A0000622B732B8C199D09AE09BF09369527950A
:106A100017950795880F991FAA1FBB1F319749F734
:106A20008A019B010F7710702070307000341105BF
:106A30002105310559F447FD09C00097A105B105AD
:106A400029F0405C5F4F6F4F7F4F40784D8B5E8BDE
:106A50006F8B788FCE01419605C0CE01099602C09A
:106A60008AE191E00E948C36462F572F682F792FAC
:106A7000CB01BA016896E8E00C94A573A8E1B0E0F8
:106A8000E4E4F5E30C948F73DC01CB018D839E83EA
:106A9000AF83B88729833A834B835C83CE01059605
:106AA000BE016F5E7F4F0E946637CE010196BE0128
:106AB000675F7F4F0E9466378989823058F08985E9
:106AC000823040F0CE014196BE01675F7F4F0E9449
:106AD000CF3701C08FEF6896E2E00C94AB73CF9292
:106AE000DF92EF92FF92CF93DF93CDB7DEB7289777
:106AF0000FB6F894DEBF0FBECDBF6B017C0183E003
:106B00008983D701C6018827B7FD83959927AA27CE
:106B1000BB27282F8A83C114D104E104F10419F49E
:106B200082E0898335C08EE190E09C838B832223B1
:106B300089F080E0C81680E0D80680E0E80680E8AA
:106B4000F80659F1F094E094D094C094C11CD11C83
:106B5000E11CF11CCD82DE82EF82F886C701B6010E
:106B60000E94383601971816190694F4082E04C0AE
:106B7000CC0CDD1CEE1CFF1C0A94D2F7CD82DE8209
:106B8000EF82F8862EE130E0281B390B3C832B8303
:106B9000CE0101960E948C3604C060E070E080E077
:106BA0009FEC382F292F862F972FA32FB22FBC01B0
:106BB000CD0128960FB6F894DEBF0FBECDBFDF9192
:106BC000CF91FF90EF90DF90CF900895ACE0B0E0D0
:106BD000ECEEF5E30C948D73DC01CB0189839A8391
:106BE000AB83BC83CE010196BE016B5F7F4F0E94D9
:106BF00066378D81823069F1823058F1843039F006
:106C00002F81388537FD25C02F31310544F08E8125
:106C1000882321F100E010E020E030E823C08EE17D
:106C200090E0821B930B09851A852B853C8504C057
:106C300036952795179507958A95D2F78E818823E3
:106C400089F030952095109501951F4F2F4F3F4F9C
:106C500009C000E010E020E030E004C00FEF1FEFBB
:106C60002FEF3FE7B801C9012C96E4E00C94A9731B
:106C7000CF92DF92EF92FF920F931F938B019C01B3
:106C8000003080E0180781E0280780E0380758F4DA
:106C90000F3F11052105310509F090F480E090E0E7
:106CA000A0E0B0E016C00030E0E01E07E0E02E07F4
:106CB000E1E03E0750F480E190E0A0E0B0E009C0E0
:106CC00088E090E0A0E0B0E004C088E190E0A0E0BF
:106CD000B0E040E250E060E070E0481B590B6A0B06
:106CE0007B0B6801790104C0F694E794D794C794AC
:106CF0008A95D2F7D701C6018E5D9E4FFC01808137
:106D0000481B510961097109CA011F910F91FF9038
:106D1000EF90DF90CF900895CF92DF92EF92FF92A5
:106D20000F931F93DC0114964D915D916D917C91B1
:106D300017971196EC9111978C91823020F4606135
:106D40008FEF90E0A8C0843009F49FC0823009F42E
:106D500096C0411551056105710509F493C012965D
:106D60008D919C9113972FEF823892070CF05BC0A6
:106D700022E83FEF281B390B2A3131056CF56A01F7
:106D80007B01022E04C0F694E794D794C7940A942A
:106D9000D2F781E090E0A0E0B0E004C0880F991F36
:106DA000AA1FBB1F2A95D2F70197A109B109842315
:106DB0009523A623B72341E050E060E070E0009700
:106DC000A105B10521F440E050E060E070E04C29FD
:106DD0005D296E297F2904C040E050E060E070E04A
:106DE000DB01CA018F779070A070B070803491057C
:106DF000A105B10539F447FF09C0405C5F4F6F4FF3
:106E00007F4F04C0415C5F4F6F4F7F4F81E090E048
:106E1000403020E0520720E0620720E4720738F596
:106E200080E090E024C0803891057CF58A019B01C8
:106E30000F77107020703070003411052105310576
:106E400039F447FF09C0405C5F4F6F4F7F4F04C06C
:106E5000415C5F4F6F4F7F4F77FD03C081589F4F5D
:106E600006C0769567955795479580589F4F97E050
:106E700076956795579547959A95D1F70CC080E020
:106E800090E005C080E090E006C08FEF90E040E029
:106E900050E060E070E0982F979599279795A62F7E
:106EA000AF77E795EE27E79586953A2F392B282F70
:106EB0002E2B842F952FA32FB22FBC01CD011F9114
:106EC0000F91FF90EF90DF90CF900895DC01FB01D0
:106ED0004C9111965C91119712968C911297682F94
:106EE0006F7770E0982F991F9927991F13962C910F
:106EF0001397822F880F892B90E0221F2227221FB1
:106F00002183009739F5411551056105710511F48B
:106F100082E029C082E89FEF9383828327E0440FB9
:106F2000551F661F771F2A95D1F783E0808309C01C
:106F3000440F551F661F771F8281938101979383AA
:106F40008283403080E0580780E0680780E478075B
:106F500078F320C08F3F910579F441155105610503
:106F6000710519F484E08083089564FF03C081E013
:106F7000808310C010820EC08F579040938382830D
:106F800083E0808387E0440F551F661F771F8A9533
:106F9000D1F7706444835583668377830895CF93D4
:106FA000FC01DB019081923008F44CC08C9182305E
:106FB00008F448C0943069F42181843039F4119682
:106FC0008C91119790E0821B910944C02223D1F14A
:106FD0003FC0843021F0923041F48230B1F11196FB
:106FE0008C9111978823A1F12DC0C181823001F1CC
:106FF00011968C911197C817D9F4828193811296BA
:107000002D913C9113972817390794F08217930715
:10701000BCF0448155816681778114968D919D9154
:107020000D90BC91A02D84179507A607B70718F4FB
:10703000CC2341F00DC0481759076A077B0728F495
:10704000CC2331F081E090E005C080E090E002C008
:107050008FEF9FEFCF9108958093AA079093AB078E
:107060000895E8E4F3E0A0E4B2E068E06D933197BE
:10707000E9F711240895992777272EE1629F080EDA
:10708000191EA0E4B2E0A00DB11D485F4C9311247D
:10709000089599272EE1629F080E191EA0E4B2E020
:1070A000A00DB11D5091D207450F4C9311240895A6
:1070B0008093D20708958093D0079093D1070895C5
:1070C0008091D607089511241092D6070895882339
:1070D00029F48091DF079091E00708958091E307FC
:1070E0009091E4070895F999FECF92BD81BD60BDEE
:1070F000F894FA9AF99A78940895F999FECF92BD86
:1071000081BDF894F89A80B57894089528E088E1D4
:1071100090E00FB6F894A895809360000FBE20937E
:107120006000FFCF129AC895C895129840E180E0A0
:1071300090E020E030E03695279596958795139856
:10714000C895C895009B3068019B9068139AC895B4
:10715000C895415081F73093E0072093DF07909363
:10716000E4078093E3078091DF079091E0078F3079
:10717000910539F08091E3079091E4078F309105F4
:1071800011F40E94863808951092460A009903C0AF
:1071900081E08093460A019905C08091460A826089
:1071A0008093460A0E9492380895CF93DF93C0E0FF
:1071B000D0E0FE01E058FF4F6491CE010E94733889
:1071C0002196C032D105A9F7C0E2D0E0CE016FEF21
:1071D0000E947338CE0101966FEF0E947338A0961B
:1071E00088E0C030D80791F7DF91CF910895CF9311
:1071F00080E090E00E947D38C82F81E090E00E94FE
:107200007D38382F20E02C0F311D81E095E52A359F
:10721000390709F080E0CF910895A0E0B0E0E3E104
:10722000F9E30C9488737C010E94F738882309F4F1
:107230004BC0F70180819181FFEF8F3F9F0709F4D9
:1072400045C025E58A35920709F440C000E210E008
:10725000C0E0D1E0C8010E947D38B82EC801019677
:107260000E947D38D82ECC24C6018B0D911DF701CC
:10727000208131818217930719F4CC23B1F00EC01D
:10728000FFEF8F3F9F0719F4CC2309F4CD2FDF5F69
:10729000005E1F4FD034F1F6CC23D1F00C2F10E05C
:1072A000E5E0000F111FEA95E1F7E70170E2E72E34
:1072B0000C1B1D0BCE01800F911F69910E9473382A
:1072C000EA94C1F780E005C084E003C081E001C01A
:1072D00082E0CDB7DEB7E9E00C94A473A0E0B0E0A3
:1072E000E4E7F9E30C9488738C017B010E94F73882
:1072F000882379F18FEF0F3F180769F1C0E0D0E0E4
:10730000CE010E947D38B82ECE0101960E947D38B4
:10731000D82ECC24C6018B0D911D8017910731F416
:107320008701F0E2FF2EC01BD10B07C0A096E4E05E
:10733000C030DE0729F783E00FC0C8018C0F9D1F06
:107340000E947D38F80181938F01FA94B1F780E0B3
:1073500003C084E001C081E0CDB7DEB7E9E00C9462
:10736000A473FC014587089581E091E09093270A7A
:107370008093260A4093250A0895862F642F0E9441
:1073800079320895FC01862F9181490F4183642F42
:107390000E945A320895FC01862F9181941B91839B
:1073A000692F0E945A320895FC0180818F75808375
:1073B0000895FC018081806480830895FC014487E6
:1073C0000895A1E0B0E0E7EEF9E30C948D738C0131
:1073D000862F642F49830E945A324981F8014183E4
:1073E0002196E4E00C94A973FC0147830895FC0105
:1073F00040870895CF93DF93EC01262F898190E099
:10740000FC01EE0FFF1FE85FF34865917491E42FD4
:10741000FF27E7FDF095E80FF91FEE0FFF1FE85F6C
:10742000F34885919491861B970B60914E0A70E00A
:107430000E942F736115710511F461E070E0822FD5
:1074400090E0FC01EE0FFF1FE80FF91FEE0FFF1F8A
:10745000EE5EF54F81819281860F971F9283818323
:107460007B836A838881886088838981840F8C8389
:10747000DF91CF91089540934E0A08959093A40A06
:107480008093A30A8FE68093A80A10920008E7E58C
:10749000FAE084E020E19FEF38E1DF011E972C93B2
:1074A000DF0113971C92DF0115979C93DF0114975E
:1074B0009C931082DF0116973C93DF0119972C9360
:1074C00081507696882349F70895E9E4FAE024E0AC
:1074D00030813F773083215076962223C9F7019679
:1074E0009093AC0A8093AB0A9093480A8093470A22
:1074F0009093AE0A8093AD0A1092AA0A1092A90A3C
:107500001092A20A1092A10A1092A50A81E080931B
:1075100000081092A70A1092A60A08958AEF809395
:10752000560A80936C0A8093820A8093980A10927C
:107530000008089581E0809300080895A0E0B0E07D
:10754000E4EAFAE30C948573C3E1DAE060E070E00A
:10755000E6E1EE2EF12C6E9DD0016F9DB00D7E9D6B
:10756000B00D1124A75BB54F1D968C911D978823F4
:10757000A9F01C962C911C97992787FD9095820F56
:10758000911D8F3F910519F014F08FEF90E097FF58
:1075900002C080E090E01C968C931C974C9143FFB6
:1075A00026C012960D911C91139728813981200FC6
:1075B000311F3983288314968C91149790E0880F9B
:1075C000991F885F9348FC018591949110161106CC
:1075D00024F42817390738F40AC00115110539F0C9
:1075E0008217930720F099838883477F4C936F5FBE
:1075F0007F4F26966430710509F0ADCF8091000869
:10760000882309F0E3C0FEC02091AB0A3091AC0A98
:10761000B9016F5F7F4F7093AC0A6093AB0AF901B9
:1076200044914F3F69F5C90102969093AC0A80934B
:10763000AB0AFB0164916F3219F410920008D4C0B8
:10764000663009F0B6C0C90104969093AC0A8093E5
:10765000AB0A2D5F3F4FF9012491233529F4909314
:10766000AE0A8093AD0AA5C0253409F0A2C080916E
:10767000AD0A9091AE0A9093AC0A8093AB0A99C080
:1076800047FF02C04093A50A9091A50A892F8F70E9
:1076900047FF08C02E5F3F4F3093AC0A2093AB0AE0
:1076A000FB014491292F30E0207F3070203B3105D1
:1076B00029F1203C310509F471C02039310509F068
:1076C00078C0E091AB0AF091AC0A9F012F5F3F4F69
:1076D0003093AC0A2093AB0A2491682F70E06C9F22
:1076E000D0016D9FB00D7C9FB00D1124A75BB54FED
:1076F000220F1E966C910E94AD3D5BC0E091AB0ADB
:10770000F091AC0A9F012F5F3F4F3093AC0A20935A
:10771000AB0AE491473079F490E08C9FD0018D9FC3
:10772000B00D9C9FB00D1124A75BB54FEE0F1A96BC
:10773000EC931A973EC04B3079F490E08C9FD001C7
:107740008D9FB00D9C9FB00D1124A75BB54FEE0F20
:107750001996EC9319972DC04C3579F490E08C9FD5
:10776000D0018D9FB00D9C9FB00D1124A75BB54F2C
:10777000EE0F1796EC9317971CC04436D1F490E0A7
:107780008C9FD0018D9FB00D9C9FB00D1124A75BE5
:10779000B54FEE0F1896EC9318970BC090E08C9FA6
:1077A000F0018D9FF00D9C9FF00D1124E75BF54FCC
:1077B00046878BEA9AE00E94D73C9093AA0A80936E
:1077C000A90A1092A20A1092A10A02C0C6E1D0E052
:1077D000A091A10AB091A20A8091A90A9091AA0A47
:1077E000A817B90709F410CF1196B093A20AA09375
:1077F000A10A8091A60A9091A70A01969093A70AE0
:107800008093A60AC2E1CC2ECAE0DC2EEE24FF242F
:10781000D6E18D2E912C0FEFA02EB12C0E2DE89CD1
:10782000E001E99CD00DF89CD00D1124C75BD54F29
:10783000888186FD3BC08C899D89009709F433C0FF
:107840009A898989981758F52EC0EC89FD89AF016E
:107850004F5F5F4F5D8B4C8B84918F3F31F48881FC
:107860008F7788831D8A1C8A1EC03296FD8BEC8B15
:10787000FA01449190E0880F991F82539F4FFC01B9
:1078800025913491CE01602FF9010995EC89FD898C
:10789000CF0101969D8B8C8BE491E98B1A8A9A8992
:1078A0008989981791F28A898F5F8A8B888185FFF1
:1078B00069C08B898F3F11F08F5F8B8B9B859923DC
:1078C00009F459C02C85222309F455C08A858823E0
:1078D00009F451C04091A80A442309F44CC0989F70
:1078E000C001112480509F4F692F772730E0629F9D
:1078F000C001639F900D729F900D112480509F4F87
:10790000692F7727298530E0629FC001639F900D22
:10791000729F900D112480509F4F692F7727242F3D
:1079200030E0629FC001639F900D729F900D112403
:1079300080509F4F492F55278F818823F1F0EE818A
:10794000F0E0E050F248E491E0588E9FF0011124FD
:10795000E050FF4FEF2FFF2795012E1B3F0B249F79
:10796000C001259F900D349F900D112480509F4F92
:10797000492F552702C040E050E08E819885890F3D
:107980008E8302C040E050E0F60140830894E11C81
:10799000F11C86E090E0C80ED91E94E0E916F104CF
:1079A00009F03CCFCDB7DEB7ECE00C94A173DC015D
:1079B000ED91FC9111979F012F5F3F4F11963C93E2
:1079C0002E93849190E087FF14C08F7790709695E6
:1079D000982F882797958795F9012F5F3F4FE4915E
:1079E0004E2F4F77840F911DE7FDF1CF11963C93F9
:1079F0002E930895FF920F931F93CF93DF93082F39
:107A0000162FA82FB0E0E6E1F0E0AE9FE001AF9FB7
:107A1000D00DBE9FD00D1124C75BD54F8881FF24A8
:107A2000F39487FFFF241A8A1D869FEF9C874B875C
:107A30001B8A8062877B88831F8299872983033012
:107A400069F4FF2009F4122F81E091E09093270A56
:107A50008093260A81E08093250A08C0802F622F38
:107A60000E945A32802F60E00E947932FF2011F08C
:107A70001F8701C01E87212F30E0C901A3E0880FB6
:107A8000991FAA95E1F7820F931FE091A30AF09145
:107A9000A40AE80FF91F339685919491009719F481
:107AA0001D8A1C8A06C0FC012491298B01969D8B9E
:107AB0008C8BCDB7DEB7E5E00C94A873982F562FCA
:107AC000682F70E09B01B3E0220F331FBA95E1F7F6
:107AD000260F371FE091A30AF091A40AE20FF31FCB
:107AE000E491E130E9F0E230E9F080915F0A87FF4C
:107AF0001BC080916E0A891711F44423A9F4809168
:107B0000750A87FF13C08091840A891711F44423F2
:107B100069F42091720A8091880A821738F404C0AF
:107B200083E005C084E003C081E001C082E0A82FAB
:107B3000B0E026E130E0A29FF001A39FF00DB29FDC
:107B4000F00D1124E75BF54F208120682083692F19
:107B5000452F20E50E94FA3C0895CF93DF93942FA0
:107B6000E82FF0E0C6E1D0E0EC9FD001ED9FB00D32
:107B7000FC9FB00D1124A75BB54F3C9135FF02C0AF
:107B800037FD29C02223B1F486E190E0E89FD001BF
:107B9000E99FB00DF89FB00D1124A75BB54F3F7B57
:107BA0003C931D968C911D978823A9F41B961C92DB
:107BB0001B9711C0C6E1D0E0EC9FD001ED9FB00D46
:107BC000FC9FB00D1124A75BB54F3F773C93422F2C
:107BD000292F0E94FA3CDF91CF9108958093A80A43
:107BE00008950000000000000000000000000000F8
:107BF0000000000000000000000000000000000085
:107C000080E08093110A08952200240026002800B5
:107C10002B002D0030003300360039003D004000BD
:107C2000440048004C00510056005B0060006600B4
:107C30006C00730079008100880090009900A20018
:107C4000AC00B600C100CC00D800E500F300010193
:107C5000100121013201440157016C018101980199
:107C6000B001CA01E5010202210241026402880258
:107C7000AE02D7020303300361039403CB03050470
:107C800042048304C70410055D05AF0505066106BF
:107C9000C206290796070908830805098E09200AE4
:107CA000BA0A5D0B0A0CC10C840D510E2B0F121079
:107CB00007110A121D1340147415BA1614188319EB
:107CC000071BA31C571E24200E22142439267F28AC
:107CD000E82A752D293006330F364539AD3C494029
:107CE0001B442848734CFE50CF55EA5A51600C662D
:107CF0001D6C8B725A79928037885090E598FDA15F
:107D00009FABD3B5A3C0000000000000000000003E
:107D10000000000000000000000000000000000063
:107D20000000000000000000000000000000000053
:107D30000000000000000000000000000000000043
:107D40000000000000000000000000000000000033
:107D50000000000000000000000000000000000023
:107D60000000000000000000000000000000000013
:107D70000000000000000000000000000000000003
:107D800000000000000000000000000000000000F3
:107D900000000000000000000000000000000000E3
:107DA00000000000000000000000000000000000D3
:107DB00000000000000000000000000000000000C3
:107DC00000000000000000000000000000000000B3
:107DD00000000000000000000000000000000000A3
:107DE0000000000000000000000000000000000093
:107DF0000000000000000000000000000000000083
:107E0000000306090C101316191C1F2225282B2EFF
:107E1000313336393C3F414447494C4E5153555814
:107E20005A5C5E60626466686A6B6D6F70717374D1
:107E3000757678797A7A7B7C7D7D7E7E7E7F7F7F8A
:107E40007F7F7F7F7E7E7E7D7D7C7B7A7A79787670
:107E500075747371706F6D6B6A68666462605E5C86
:107E60005A585553514E4C494744413F3C3936339B
:107E7000312E2B2825221F1C191613100C0906035E
:107E800000FDFAF7F4F0EDEAE7E4E1DEDBD8D5D265
:107E9000CFCDCAC7C4C1BFBCB9B7B4B2AFADABA830
:107EA000A6A4A2A09E9C9A9896959391908F8D8C53
:107EB0008B8A88878686858483838282828181817A
:107EC0008181818182828283838485868687888A74
:107ED0008B8C8D8F9091939596989A9C9EA0A2A43E
:107EE000A6A8ABADAFB2B4B7B9BCBFC1C4C7CACD09
:107EF000CFD2D5D8DBDEE1E4E7EAEDF0F4F7FAFD26
:107F0000808182838485868788898A8B8C8D8E8FF9
:107F1000909192939495969798999A9B9C9D9E9FE9
:107F2000A0A1A2A3A4A5A6A7A8A9AAABACADAEAFD9
:107F3000B0B1B2B3B4B5B6B7B8B9BABBBCBDBEBFC9
:107F4000C0C1C2C3C4C5C6C7C8C9CACBCCCDCECFB9
:107F5000D0D1D2D3D4D5D6D7D8D9DADBDCDDDEDFA9
:107F6000E0E1E2E3E4E5E6E7E8E9EAEBECEDEEEF99
:107F7000F0F1F2F3F4F5F6F7F8F9FAFBFCFDFEFF89
:107F8000000102030405060708090A0B0C0D0E0F79
:107F9000101112131415161718191A1B1C1D1E1F69
:107FA000202122232425262728292A2B2C2D2E2F59
:107FB000303132333435363738393A3B3C3D3E3F49
:107FC000404142434445464748494A4B4C4D4E4F39
:107FD000505152535455565758595A5B5C5D5E5F29
:107FE000606162636465666768696A6B6C6D6E6F19
:107FF000707172737475767778797A7B7C7D7E7F09
:1080000000020406080A0C0E10121416181A1C1E80
:1080100020222426282A2C2E30323436383A3C3E70
:1080200040424446484A4C4E50525456585A5C5E60
:1080300060626466686A6C6E70727476787A7C7E50
:108040007F7D7B79777573716F6D6B696765636130
:108050005F5D5B59575553514F4D4B494745434120
:108060003F3D3B39373533312F2D2B292725232110
:108070001F1D1B19171513110F0D0B090705030100
:10808000FFFDFBF9F7F5F3F1EFEDEBE9E7E5E3E1F0
:10809000DFDDDBD9D7D5D3D1CFCDCBC9C7C5C3C1E0
:1080A000BFBDBBB9B7B5B3B1AFADABA9A7A5A3A1D0
:1080B0009F9D9B99979593918F8D8B8987858381C0
:1080C00080828486888A8C8E90929496989A9C9EC0
:1080D000A0A2A4A6A8AAACAEB0B2B4B6B8BABCBEB0
:1080E000C0C2C4C6C8CACCCED0D2D4D6D8DADCDEA0
:1080F000E0E2E4E6E8EAECEEF0F2F4F6F8FAFCFE90
:108100007F7F7F7F7F7F7F7F7F7F7F7F7F7F7F7F7F
:108110007F7F7F7F7F7F7F7F7F7F7F7F7F7F7F7F6F
:108120007F7F7F7F7F7F7F7F7F7F7F7F7F7F7F7F5F
:108130007F7F7F7F7F7F7F7F7F7F7F7F7F7F7F7F4F
:108400000309131E28313A40464C5054585B5E61B4
:10841000636567696B6C6E6F707172737475767774
:10842000777879797A7A7B7B7C7C7C7D7D7D7E7E9A
:108430007E7E7F7F7F7F7F7F7F7F7F7F7F7F7F7F4E
:108440007F7F7F7F7F7F7F7F7F7F7F7F7F7E7E7E3F
:108450007E7D7D7D7C7C7C7B7B7A7A797978777771
:10846000767574737271706F6E6C6B69676563613A
:108470005E5B5854504C46403A31281E13090300A5
:10848000C6CCD5DBDFE3E5E7E9EAEBECEDEEEFEFB9
:10849000F0F0F0F1F1F1F1F2F2F2F2F2F2F2F2F3C5
:1084A000F3F3F3F3F3F3F3F3F3F3F3F3F3F3F3F39C
:1084B000F3F3F3F3F3F3F3F3F3F3F3F3F3F3F3F38C
:1084C000F3F3F3F3F3F3F3F3F3F3F3F3F3F3F3F37C
:1084D000F3F3F3F3F3F3F3F3F3F3F3F3F3F3F3F36C
:1084E000F2F2F2F2F2F2F2F2F1F1F1F1F0F0F0EF79
:1084F000EFEEEDECEBEAE9E7E5E3DFDBD5CCC60038
:1085000000283D42302D2C2B2C2D2E2F3032333590
:1085100037393B3D3F414345484A4C4E50535557F0
:10852000595B5D5F61636567696B6C6E70717374D5
:10853000757778797A7B7C7D7D7E7E7F7F7F7F7F7C
:108540007F7F7F7F7F7F7E7E7D7D7C7B7A79787762
:1085500075747371706E6C6B69676563615F5D5B89
:1085600059575553504E4C4A484543413F3D3B397E
:1085700037353332302F2E2D2C2B2C2D30423D28E9
:1085800000E9E5FED4D7D7D7D6D4D2D0CECCCAC84E
:10859000C6C3C1BFBDBAB8B6B4B1AFADABA9A7A58C
:1085A000A3A19F9E9C9A999795949391908F8D8C5F
:1085B0008B8A89888887868585848484838383835E
:1085C0008383838383848484858586878888898A56
:1085D0008B8C8D8F909193949597999A9C9E9FA147
:1085E000A3A5A7A9ABADAFB1B4B6B8BABDBFC1C35F
:1085F000C6C8CACCCED0D2D4D6D7D7D7D4FEE5E918
:10860000F9F8F9F5EBE1DDDEE0E2E4E5E6E5E4E2E8
:10861000DED9D2CAC1B7ACA299918A868381808003
:108620008182838586888A8C8D8F90929395969788
:1086300098999A9B9B9C9D9D9D9E9E9E9F9F9F9F70
:108640009F9F9F9E9E9E9D9D9D9C9B9B9A99989768
:1086500096959392908F8D8C8A888685838281806F
:10866000808183868A9199A2ACB7C1CAD2D9DEE251
:10867000E4E5E6E5E4E2E0DEDDE1EBF5F9F8F9005A
:108680000708070B151F2322201E1C1B1A1B1C1E6C
:1086900022272E363F49545E676F767A7E7F7F7F32
:1086A0007F7E7D7B7A7876747371706E6D6B6A698C
:1086B0006867666565646463636262626161616183
:1086C000616161626262636363646565666768696C
:1086D0006A6B6D6E7071737476787A7B7D7E7F7F46
:1086E0007F7F7E7A766F675E54493F362E27221E43
:1086F0001C1B1A1B1C1E2022231F150B070807001A
:108700001F313D444E5354565A5F64696E747679F6
:108710007C7F7F7F7F7F7F7F7F7F7F7F7F7F7F7F6C
:108720007F7F7F7F7F7F7F7F7F7F7F7F7F7F7F7F59
:108730007F7F7F7F7F7F7F7F7F7F7F7F7F7F7F7F49
:108740007F7F7F7F7F7F7F7F7F7F7F7F7F7F7F7F39
:108750007F7F7F7F7F7F7F7F7F7F7F7F7F7F7F7F29
:108760007F7F7F7F7F7F7F7F7F7F7F7F7F7F7F7F19
:108770007F7F7F7F7F7F7F7F7F7F7F7C7871684C6B
:108780002C1C120C0A0B0A05FDF3E9DFD4CAC0B792
:10879000AEA69E97918B8685828080808080808027
:1087A00080808080808080808080808080808080C9
:1087B00080808080808080808080808080808080B9
:1087C00080808080808080808080808080808080A9
:1087D0008080808080808080808080808080808099
:1087E0008080808080808080808080808080808089
:1087F000808080808087919DACC4CBD4DDF2FAFA72
:108800009091B10AE4E9F7E080E00BC02081DF013C
:1088100012970D90BC91A02DA05CBD4F2C938F5F43
:108820003396891799F70895A7E0B0E0EAE1F4E4F8
:108830000C947F731092B10A80910001882309F48F
:10884000A7C0F9E8AF2EF5E0BF2E40E08501F801A2
:1088500031972081203F09F493C0F8013081832FA4
:1088600090E0C22EC694C694C694277019F433249F
:10887000339402C0E2E03E2E73E0969587957A9598
:10888000E1F7582F832F877019F46624639402C090
:1088900062E0662E8A83198289819A81820F911DF6
:1088A0009E838D83AA24BB2424EED22ED50E32EED5
:1088B000732E7C0C280145C0802F8C0D8E3110F05A
:1088C000872D800F9701280F311DB0E48B2EB2E069
:1088D0009B2E820E931EF40170817830E8F0609137
:1088E000B10A683018F5862F90E0FC01EE0FFF1FEB
:1088F000E80FF91FEE56F84F318320837283872FDC
:108900000E946E2F7091B10AF4017083872F8F5FE0
:108910008093B10A783050F44B815C81400F511F35
:10892000822D672F2D813E810E94FF2F0F5F1F4FE9
:10893000031510F25F81422D0894A11CB11CA614EE
:10894000F0F42A2D8A2D850F8C3110F02D0D01C0E9
:10895000282F822F90E09C01220F331F7C0175E0AD
:10896000EE0CFF1C7A95E1F7E21AF30A9A2D88279C
:108970009C838B8300E010E05F83242E9DCF8201D7
:108980004F5F0B5F1F4F423009F061CF0E940044E0
:108990002796E2E10C949B73089580EF80938805FD
:1089A00080938D0508950E9471450E941444089596
:1089B000AF92BF92CF92DF92EF92FF921F93CF932D
:1089C000DF93FA01749131961491A72EBB24C0E075
:1089D000D0E020E0A82FB0E0A05CBD4F28C0F60199
:1089E000E80FF91F3491E62FF0E07F01EE0CFF1C39
:1089F000689414F8EE0FFF1F1694E1F7EE19FF09C3
:108A0000EA0FFB1FEC0FFD1FE80FF91F385F3083E3
:108A1000019607C080E090E032E0C32ED12CC40E56
:108A2000D51E8717E0F22F5F4A0D5B1D6E9621174A
:108A300089F7DF91CF911F91FF90EF90DF90CF905A
:108A4000BF90AF9008956F927F928F929F92AF9256
:108A5000BF92DF92EF92FF920F931F93CF93DF931A
:108A6000E82ED62E3A014901580100E010E011C06D
:108A70008C2F8E0D6F2DA5010E943B38219604C0CE
:108A8000C0E0D0E0F02EFD0CC615D7058CF30F5FCB
:108A90001F4F08151905A4F3DF91CF911F910F9176
:108AA000FF90EF90DF90BF90AF909F908F907F905E
:108AB0006F9008950F931F93CF93DF938C01C0E0C5
:108AC000D0E007C00E9460388823E1F30E94633839
:108AD0002196C017D107B4F3DF91CF911F910F9169
:108AE00008958091B20A8823F9F08091B30A88230F
:108AF000C1F48091AF0A8093B30A8091B40AE82F41
:108B0000F0E0E951FF4FE491E7B99091B00A980F76
:108B10009093B40A992311F09D3031F41092B20A67
:108B2000089581508093B30A0895AF92BF92DF9267
:108B3000EF92FF920F931F93CF93DF938C01EB0182
:108B40005A01D22E80E090E07C010894E11CF11CD7
:108B5000F501E80FF91F4491433C39F422E0E22E7D
:108B6000F12CE80EF91E41E31AC04532B9F0842F0A
:108B70008852823010F44E5112C0842F81548C30B0
:108B800010F445530CC0842F8D548E3010F44A528B
:108B900006C0442391F04F77485101C049E0DD20E1
:108BA00029F4802F0F5F1F4F6C2F03C06C2F21966D
:108BB000802F0E944938C701C7CFDF91CF911F9105
:108BC0000F91FF90EF90DF90BF90AF900895AF921C
:108BD000BF92DF92EF92FF920F931F93CF93DF9399
:108BE0000F92CDB7DEB75C018B01F42EEE243AE094
:108BF000D32EFF2011F4EE2061F48F2D6D2D0E94F5
:108C00000F73985E8A2D602F492F29830E9449385F
:108C10002981222319F00150104003C00894A108B3
:108C2000B1088F2D6D2D0E940F73F82EE39483E011
:108C3000E816F9F60F90DF91CF911F910F91FF90F9
:108C4000EF90DF90BF90AF9008958230910571F062
:108C50008330910531F08130910561F48BED95E41D
:108C600002C085EF94E50E94653A089584E49EE48D
:108C70000E94653A089589E392E09093B70A809341
:108C8000B60A66EB7AE00E946E398091D40A90E0D1
:108C90009C0146E0369527954A95E1F73093320BD3
:108CA0002093310B21E081FF20E020932C0B21E069
:108CB00082FF20E02093300B21E083FF20E020930F
:108CC0002D0B21E084FF20E02093B50A91E085FF81
:108CD00090E09093330BA8EBBAE0EAE2FAE080E090
:108CE00090E02D91219301968E309105D1F7A6EC5D
:108CF000BAE0E8E3FAE080E090E02D91219301965C
:108D00008E309105D1F78091C60A882321F4809195
:108D1000C70A882319F08CE090E00DC08091B80A52
:108D2000882321F48091B90A882319F08BE090E020
:108D300002C08AE090E090932F0B80932E0B089551
:108D400089E392E09093B70A8093B60A8091310B41
:108D50009091320B83709070880F991F2091330B84
:108D6000820F911D880F991F2091B50A820F911DC6
:108D7000880F991F20912D0B820F911D880F991F2D
:108D80002091300B820F911D880F991F20912C0B81
:108D9000820F911D880F8093D40AAAE2BAE0E8EB13
:108DA000FAE080E090E02D91219301968E309105BC
:108DB000D1F7A8E3BAE0E6ECFAE080E090E02D918C
:108DC000219301968E309105D1F786EB9AE00E94AF
:108DD0000D3908950F931F930E948E3A89E392E014
:108DE0009093B70A8093B60AE8EBFAE080E090E04F
:108DF000119201968E319105D9F786EB9AE00E9487
:108E00000D390E943B468091B50A882329F485E0FC
:108E10006FEF41E00E945E3D84E090E06FE070E023
:108E200048E05AE520E00E94954588E790E00E94DE
:108E30005A4584E090E06FE070E04EE050E021E0C1
:108E400030E000E010E00E9423451F910F9108954B
:108E50000E94313885E064E044EF50E00E94D8443D
:108E600087E090E062E070E045E259E520E00E9492
:108E7000954584E090E069E170E042E459E520E046
:108E80000E9495458091330B882321F481EA91E477
:108E90000E94653A80EF8093880580938D05089540
:108EA0000F931F93CF93C82F82E090E060E170E0B2
:108EB00041E050E028E030E000E010E00E9423456F
:108EC0006C2F605F82E046EA50E00E943B38CF9111
:108ED0001F910F9108950F931F93CF93DF93EC0190
:108EE00086E190E060E170E048E050E026E030E0AC
:108EF00000E010E00E94234583E190E066E170E02D
:108F00004BE050E021E030E00E9423458091310B9E
:108F10009091320B009739F486E190E060E170E0C7
:108F200047EA59E510C08130910539F486E190E0B7
:108F300060E170E042EA59E506C086E190E060E158
:108F400070E04EEA59E520E00E94954580912C0B97
:108F5000882339F486E190E061E170E040ED59E565
:108F600006C086E190E061E170E043ED59E520E064
:108F70000E9495458091300B882339F486E190E07A
:108F800062E170E040ED59E506C086E190E062E103
:108F900070E043ED59E520E00E94954580912D0B4E
:108FA000882339F486E190E063E170E040ED59E513
:108FB00006C086E190E063E170E043ED59E520E012
:108FC0000E9495458091330B882339F486E190E027
:108FD00064E170E040ED59E506C086E190E064E1AF
:108FE00070E043ED59E520E00E9495458091B50A77
:108FF000882339F486E190E065E170E040ED59E5C1
:1090000006C086E190E065E170E043ED59E520E0BF
:109010000E949545209739F483E190E066E170E085
:1090200040E45AE545C0C130D10539F483E190E010
:1090300066E170E04FE25AE53BC0C230D10539F439
:1090400083E190E066E170E048E35AE531C0C33067
:10905000D10539F483E190E066E170E040E25AE541
:1090600027C0C430D10539F483E190E066E170E0B7
:1090700047E25AE51DC0C530D10539F483E190E0DF
:1090800066E170E047E15AE513C0C630D10598F0BB
:10909000AE01440F551FB3E0CC0FDD1FBA95E1F7C9
:1090A0004C0F5D1F475F554A83E190E066E170E039
:1090B00020E00E949545DF91CF911F910F91089577
:1090C000A0E0B0E0E6E6F8E40C94857380E090E080
:1090D0006DE070E04EE150E02CE030E000E010E0A8
:1090E0000E94234584E090E060E170E046E959E5A4
:1090F00020E00E94954584E090E061E170E043EB60
:1091000059E520E00E94954584E090E062E170E03E
:1091100049EB59E520E00E94954584E090E063E149
:1091200070E049EC59E520E00E94954584E090E02C
:1091300064E170E047ED59E520E00E94954584E048
:1091400090E065E170E04EED59E520E00E94954524
:1091500084E090E066E170E043EE59E520E00E9493
:10916000954584E090E067E170E04FEE59E520E03E
:109170000E94954580E090E00E94504780E090E09A
:109180000E946B47C1E0CC2ED12CC0E0D0E022E0A1
:10919000822E912C81E090E00E945A4580E00E944E
:1091A00067385C0180E00E9467387601E826F9267E
:1091B000EA20FB20E5FE08C00730110528F40F5F08
:1091C0001F4FC8010E945047E4FE08C00115110559
:1091D00041F001501040C8010E945047011511058F
:1091E00081F5E7FEF9C08091310B9091320B009729
:1091F00029F49092320B8092310B07C08130910597
:1092000021F41092320B1092310BCE010E946B4769
:10921000E3C08091310B9091320B009739F481E0DB
:1092200090E09093320B8093310B07C08230910510
:1092300021F41092320B1092310BCE010E946B4739
:10924000CDC001301105A1F4C701807C907000975A
:1092500009F461C080912C0B882321F481E0809374
:109260002C0B02C010922C0BCE010E946B4753C0F6
:1092700002301105A1F4C701807C9070009709F4B9
:1092800082C08091300B882321F481E08093300BE1
:1092900002C01092300BCE010E946B4774C00330A5
:1092A000110589F4C701807C9070009709F488C08B
:1092B00080912D0B882321F481E080932D0B72C0C7
:1092C00010922D0B6FC00430110589F4C701807C0A
:1092D0009070009709F474C08091330B882321F4B7
:1092E00081E08093330B5EC01092330B5BC005307E
:1092F000110589F4C701807C9070009709F460C063
:109300008091B50A882321F481E08093B50A4AC090
:109310001092B50A47C006301105A9F5E0FE61C0FC
:109320000E948E3AC230D105C9F0C330D10530F465
:10933000209771F0C130D105F9F40DC0C430D105CA
:1093400099F0C430D10568F0C530D105A9F40FC03B
:1093500081EA91E40EC08BED95E40BC084E49EE4B9
:1093600008C085EF94E505C082E794E502C08CEB68
:1093700094E50E94653A35C08C2F83506FEF41E031
:109380000E945E3D2EC00730110581F019C0CE301D
:10939000D10548F52196CE010E946B4724C0209745
:1093A00079F02197CE010E946B470AC080E00E94AD
:1093B00067382CE08130920719F40E94EA4618C001
:1093C000C601887090709501209530958223932373
:1093D000009761F46501DECEE6FC1BCF00E010E0F3
:1093E00072CFE7FCD4CFE6FCDACFEACF0E94A046EA
:1093F000CDB7DEB7ECE00C94A173A0E0B0E0E3E001
:10940000FAE40C94897380E090E06DE070E04EE146
:1094100050E02CE030E000E010E00E94234584E0C2
:1094200090E060E170E049E559E520E00E94954553
:1094300084E090E061E170E042E659E520E00E94BE
:10944000954584E090E062E170E04CE659E520E06B
:109450000E94954584E090E063E170E044E759E5BF
:1094600020E00E94954584E090E064E170E041E8EE
:1094700059E520E00E94954580E090E00E94504729
:10948000C0E0D0E002C0CD2DDC2D81E090E00E9454
:109490005A4580E00E9467387C01D82ECF2C80E0AE
:1094A0000E946738C827D927CE21DF21C5FF08C011
:1094B0000430110528F40F5F1F4FC8010E94504768
:1094C000C4FF08C00115110529F001501040C80162
:1094D0000E945047C0FFD7CFC801CDB7DEB7E8E044
:1094E0000C94A5734F925F926F927F928F929F928E
:1094F000AF92BF92CF92DF92EF92FF920F931F93A2
:109500000E942847CC24DD2476013CE3832E912C55
:10951000A12CB12C4EE1442E512C612C712C45C054
:1095200081E090E00E945A45C701B601A50194016F
:109530000E944273DC01CB010097A105B10569F4DB
:109540008AE090E066E170E04BE050E021E030E03E
:1095500000E010E00E94234515C0C701B601A30139
:1095600092010E944273DC01CB010097A105B10575
:1095700049F48AE090E066E170E046E359E520E0D6
:109580000E94954588E5C81682E0D80680E0E80686
:1095900080E0F80629F40E948E3A81E090E00EC047
:1095A0000894C11CD11CE11CF11C80E00E946738AA
:1095B0008830910509F0B4CF80E090E01F910F91C1
:1095C000FF90EF90DF90CF90BF90AF909F908F90E3
:1095D0007F906F905F904F900895A0E0B0E0E3EF30
:1095E000FAE40C948473C82FF92E0E94313883E07A
:1095F00090E062E070E048E150E028E130E00EE702
:1096000010E00E942345AC2EBF2CE3E0CE2ED12CDF
:1096100051C0F40181914F01833031F184303CF429
:109620008130C1F08230DCF4882341F032C08530D3
:1096300029F18530F4F0863061F525C08E2D972D07
:10964000BE0144E050E024E030E00EE710E00E946C
:1096500023451FC08F2D6C2F4AEA51E018C08F2D73
:109660006C2F4CEB51E013C08F2D6C2F4EEC51E062
:109670000EC08F2D6C2F40EE51E009C08F2D6C2F46
:1096800042EF51E004C08F2D6C2F44E052E00E9465
:10969000D8442496CA31D10509F0BBCF86E090E0CA
:1096A000A80EB91EE4E0F0E0CE0EDF1EFBE1CF16FF
:1096B000D10439F0EC2C7D2CFC2C4501C2E0D0E02B
:1096C000A8CFCDB7DEB7EDE00C94A073A0E0B0E07A
:1096D000ECE6FBE40C948873D82E0E948E3A80E06E
:1096E00090E00E94504784E090E06EE070E04EEC25
:1096F0005AE520E00E94954584E090E060E170E04A
:1097000045ED5AE520E00E94954584E090E061E156
:1097100070E04CED5AE520E00E949545C0E0D0E0B5
:1097200008E010E002C00B2D1C2D81E090E00E94AB
:109730005A458D2D0E9467387C01B82ECF2C8D2D77
:109740000E946738082719270E211F2104FF06C031
:10975000209721F02197CE010E94504705FF08C0B5
:10976000209731F481E090E00E945047C1E0D0E0C2
:1097700000FFD9CF209739F48091330B882329F447
:109780000E949A3A02C081E001C080E0CDB7DEB706
:10979000E9E00C94A4732F923F924F925F926F92E4
:1097A0007F928F929F92BF92CF92DF92EF92FF9221
:1097B0000F931F93CF93DF93CDB7DEB72E970FB6DE
:1097C000F894DEBF0FBECDBF4C012B016A01FE0134
:1097D00031968EE0DF011D928A95E9F78982FA01C0
:1097E00080818A838E010D5F1F4FA1E0B0E03401BC
:1097F0000894610871088EEF282E8FEF382E280C00
:10980000391C2AE0B22E92C0F601EA0FFB1FA61502
:10981000B70529F48081D8018C93730183C0A21508
:10982000B30508F077C05081319780816B2D0E947D
:109830000F73482F852F0E940F73652F70E09D01D5
:109840002F5F3F4F7901F601E20FF31F481731F503
:10985000808190E09B012A5030402817390749F455
:109860001296F601EA0FFB1F208130E0CB01099729
:1098700025C09B01265F3F4F2817390709F046C0D6
:109880001296F601EA0FFB1F208130E0CB010B9608
:109890002817390799F1CB0109962DC0808190E0F6
:1098A0009B01215030402817390791F41296F60198
:1098B000EA0FFB1F208130E0CB01099628173907FA
:1098C00029F0CB010B9728173907E1F45C5916C032
:1098D0009B012F5F3F4F28173907C1F41296F601FD
:1098E000EA0FFB1F208130E0CB010B9628173907C8
:1098F00029F0CB0109972817390721F4F801508383
:109900007D0110C05853D8015C930CC05853F80126
:10991000508308C080818853F80180837D010894BA
:10992000E11CF11CD70111960F5F1F4FA815B90557
:1099300008F46ACFDE011196FBE04F16510459F48A
:10994000EAE2FAE080E090E02D91219301968E30DA
:109950009105D1F70AC0E8E3FAE080E090E02D91AC
:10996000219301968E309105D1F70E94A0460E9466
:109970003B462E960FB6F894DEBF0FBECDBFDF91EB
:10998000CF911F910F91FF90EF90DF90CF90BF90FC
:109990009F908F907F906F905F904F903F902F900F
:1099A00008956AE00E940F73892F08952AE0622FBC
:1099B0000E940F730E940F73892F0895A0E0B0E0FA
:1099C000E4EEFCE40C947F732C015B01FB0180E06E
:1099D00090E008C032010894611C711C71E0872E70
:1099E000912C53C11082118212821382148215822B
:1099F0000196369686309105A9F7ECCF21E08216C4
:109A0000910421F094012150304001C09C0188163E
:109A1000990629F064010894C11CD11C03C061E0BF
:109A2000C62ED12C1201220E331EF1010081802F8F
:109A30000E94D64CF82EF301C0818C2F0E94D64C88
:109A4000D82F8F1560F48C2F0E94D14C182FF20163
:109A5000EC0DFD1D80810E94D14C181798F0F20189
:109A6000EC0DFD1DE0808E2D0E94D64C182FD817CE
:109A7000D0F48C2F0E94D14CC82E802F0E94D14C44
:109A8000C81688F48C2F0E94D14C90E0FC01EE0F98
:109A9000FF1FE80FF91FEE0FFF1FEA0DFB1DED0F73
:109AA000F11D21E06AC0DF1548F48C2F0E94D14CD3
:109AB000C82E8E2D0E94D14C8C1558F0D117D0F4A1
:109AC0008C2F0E94D14CC82E802F0E94D14C8C1517
:109AD00088F48C2F0E94D14C90E0FC01EE0FFF1F08
:109AE000E80FF91FEE0FFF1FEA0DFB1DED0FF11D33
:109AF00082E057C0FD1648F48C2F0E94D14CC82E2E
:109B00008E2D0E94D14CC81658F01D17D0F48C2F02
:109B10000E94D14CC82E802F0E94D14CC81688F4C8
:109B20008C2F0E94D14C90E0FC01EE0FFF1FE80F3C
:109B3000F91FEE0FFF1FEA0DFB1DED0FF11D93E066
:109B400035C0802F0E94D14C082F8C2F0E94D14C01
:109B5000C82F0817A1F48E2D0E94D14C801779F4DC
:109B600090E0FC01EE0FFF1FE80FF91FEE0FFF1F43
:109B7000EA0DFB1DED0FF11D25E0208318C08C2F91
:109B800090E0FC01EE0FFF1FE80FF91FEE0FFF1F23
:109B9000EA0DFB1DFD1639F41F1529F4E10FF11D27
:109BA00086E0808304C0ED0FF11D94E09083F30103
:109BB000D0818D2F0E94D64CC82FF1011081812FAA
:109BC0000E94D64CC817B9F58D2F0E94D14CC82FD2
:109BD000812F0E94D14C4C2F50E0282F30E0C81725
:109BE00080F48A010F5F1F4F6901EE24FF24E80112
:109BF000CC0FDD1FC00FD11FCC0FDD1FCA0DDB1D29
:109C000016C089010F5F1F4F6A01EFCFF3018081FA
:109C10000E94D64CFE01EE0DFF1DE80FF11D26E05F
:109C200020830F5F1F4F86E090E0E80EF91E0C15B1
:109C30001D0560F324C04C2F50E0282F30E0C817DA
:109C400020F4EA012196890117C0E90121968A01D1
:109C500013C0F30180810E94D14C90E0FC01EE0F13
:109C6000FF1FE80FF91FEE0FFF1FEA0DFB1DEC0FA2
:109C7000FD1F25E020832196C017D10750F30894DB
:109C8000811C911C0894611C711CF201808190E080
:109C90008815990508F0B2CECDB7DEB7E2E10C9495
:109CA0009B73A2E1B0E0E7E5FEE40C947F732B0127
:109CB000FC013297EB30F10538F4EE0FFF1FEC5F3B
:109CC000FE4F2081318102C022E938E58B309105B9
:109CD00070F4DE01119680E090E0F901E80FF91FC1
:109CE000E491ED9301968E309105B9F70BC0F9011F
:109CF000DE01119680E090E021912D9301968E3047
:109D00009105D1F72980F20120821A81812F0E94CA
:109D1000D64C082F812F0E94D14C000F902F990F05
:109D2000990F900F980FF201918333249E012D5FBC
:109D30003F4F3A8B298B82E090E0A2E0AA2EB12C13
:109D400013C19C012F5F3F4F388B2F87E989FA8918
:109D5000F190FA8BE98B42018A0C9B1CF7ECFF1502
:109D600008F4A8C0A214B30408F08EC08F2D0E947E
:109D7000D64C182F8F2D0E94D14C912F990F192F4F
:109D8000110F110F190F180FF401108365010894BA
:109D9000C11CD11CC40CD51C812F0E94D64C082F8D
:109DA000812F0E94D14C902F990F092F000F000F87
:109DB000090F080FF6010083F40180810E94D14C45
:109DC000182FF401319780810E94D14CF3E61817C7
:109DD00031F4FF1510F4015007C00F5F05C0FF15E7
:109DE00010F40A5001C0065FF6010083C501029617
:109DF0008215930519F06F84788803C0F1E06F2E07
:109E0000712C7201E80EF91EF6010081802F0E946C
:109E1000D64C182F802F0E94D14C110F012F000F0C
:109E2000000F010F080FF7010083F60180810E94E7
:109E3000D14C182FF40180810E94D14CE1E0F0E078
:109E4000EC0FFD1FE60DF71D181769F480810E94C5
:109E5000D14C182F802F0E94D14C181710F40150AC
:109E60000EC00F5F0CC080810E94D64C182F802F2F
:109E70000E94D64C181710F40A5001C0065FF70173
:109E8000008323E030E06CC0A214B30499F48F2D5A
:109E90000E94D64C182F8F2D0E94D14C110F912F5C
:109EA000990F990F910F980FF40190830894A11CBA
:109EB000B11C58C08F2D0E94D64C182F8F2D0E9498
:109EC000D14C912F990F192F110F110F190F180F36
:109ED000F401108375010894E11CF11CF2018081EA
:109EE00090E0E816F90619F0CF84D88803C0E1E0C5
:109EF000CE2ED12C812F0E94D14C082FF201EA0DD9
:109F0000FB1D319780810E94D14CE40CF51C081791
:109F1000A1F4812F0E94D64C182FE1E0F0E0EC0F65
:109F2000FD1FEC0DFD1D80810E94D14C110F912F62
:109F3000990F990F910F980F0FC0E1E0F0E0EC0F2F
:109F4000FD1FEC0DFD1D80810E94D64C880F982FBF
:109F5000990F990F980F900FF701908322E030E04E
:109F6000A20EB31E8F8598892A143B0408F0E9CE0F
:109F70006296E2E10C949B73EF92FF920F931F9312
:109F8000CF93DF937C01FC01D1818D2F0E94D14CB6
:109F9000C82FF7011281812F0E94D14CC81708F0F9
:109FA00049C08D2F0E94D64C2C2F30E0220F331F3A
:109FB000220F331F682F70E0660F771F660F771F21
:109FC0006E5F7F4FC901069641E050E024E030E02B
:109FD0000DEB10E00E94234582E090E090938B050A
:109FE00080938A0587E090E09093900580938F0599
:109FF00010928C0510929105F7011181812F0E941A
:10A00000D14CC8E8D5E08295880F807E885D80932A
:10A010008805812F0E94D64C8295880F807E8B5EAA
:10A020008983F70181810E94D14C8295880F807EBF
:10A03000885D4CC08C1708F053C08D2F0E94D64C01
:10A040002C2F30E0220F331F220F331F682F70E0B8
:10A05000660F771F660F771F6E5F7F4FC9010396EC
:10A0600041E050E024E030E00DEB10E00E94234599
:10A0700082E090E090938B0580938A0587E090E0E2
:10A080009093900580938F0581E080938C05809359
:10A090009105F7011181812F0E94D14CC8E8D5E0CC
:10A0A0008295880F807E805E80938805812F0E9434
:10A0B000D64C8295880F807E8B5E8983F7018181E3
:10A0C0000E94D14C8295880F807E805E8D83F7013F
:10A0D00081810E94D64C8295880F807E8D5DA1C0C3
:10A0E0008D2F0E94D64CD82F812F0E94D64C2C2F1A
:10A0F00030E06D2F70E08D1708F049C0C901880F5E
:10A10000991F880F991F660F771F660F771F6E5F65
:10A110007F4F039644E050E021E030E00DEB10E08B
:10A120000E94234510928B0510928A0585E090E0ED
:10A130009093900580938F0510928C051092910555
:10A14000F7011181812F0E94D14CC8E8D5E082959A
:10A15000880F807E835E80938805812F0E94D64C75
:10A160008295880F807E885E8983F70181810E94B5
:10A17000D14C8295880F807E855D8D83F70181812A
:10A180000E94D64C8295880F807E885E4AC0C901A5
:10A19000880F991F880F991F660F771F660F771F0B
:10A1A0006B5F7F4F039644E050E021E030E00DEB21
:10A1B00010E00E94234584E090E090938B0580930B
:10A1C0008A0589E090E09093900580938F05109226
:10A1D0008C0510929105F7011181812F0E94D14CBD
:10A1E000C8E8D5E08295880F807E835E80938805DD
:10A1F000812F0E94D64C8295880F807E805E898355
:10A20000F70181810E94D14C8295880F807E855D07
:10A210008D83F70181810E94D64C8295880F807EC4
:10A22000805E8E8383E090E060E070E048E150E083
:10A2300022E030E00EE710E00E94234583E090E04A
:10A240006AE170E048E150E022E030E00E942345FE
:10A25000CDB7DEB7E6E00C94A7730F931F93CF93AF
:10A26000DF93EC0180E090E060E070E043E050E0DC
:10A270002CE130E000E010E00E9423458BE190E00B
:10A2800060E070E043E050E02CE130E00E942345C4
:10A29000CB30D10550F082E090E062E070E048EF12
:10A2A0005AE521E00E9495452A9782E090E069E016
:10A2B00070E042EF5AE521E00E94954582E090E08F
:10A2C00060E170E04C2F21E00E94E7458BE190E0D7
:10A2D00062E070E046EE5AE521E00E9495458BE190
:10A2E00090E066E170E04FEF5AE521E00E9495456D
:10A2F0008BE190E064E170E04091010121E00E9477
:10A30000E745DF91CF911F910F910895CF93DF9390
:10A310008091D80AC1E0D0E0882331F08091030B0E
:10A32000882311F0C0E0D0E0CC0FDD1F8091DA0A65
:10A330009E01280F311DA901A3E0440F551FAA95C6
:10A34000E1F7421B530B4156554A82E090E063E02F
:10A3500070E021E00E9495458091050BC80FD11D4A
:10A36000AE01B3E0440F551FBA95E1F74C1B5D0BEE
:10A370004156554A8BE190E063E070E021E00E9495
:10A380009545DF91CF9108950F931F9382E090E060
:10A3900066E170E041E050E023E030E000E010E0F2
:10A3A0000E9423458BE190E066E170E041E050E0DF
:10A3B00023E030E00E9423454091D70A469582E091
:10A3C00090E068E170E021E00E94E7454091020BD7
:10A3D00046958BE190E068E170E021E00E94E7455E
:10A3E0001F910F9108958091D80A4091010148175B
:10A3F00010F0481B01C040E082E090E060E170E0B6
:10A4000021E00E94E7458091030B4091010148172C
:10A4100010F0481B01C040E08BE190E060E170E08B
:10A4200021E00E94E74508950F931F93CF93DF9398
:10A4300080E090E060E070E043E050E02CE130E04C
:10A4400000E010E00E9423458BE190E060E070E0C6
:10A4500043E050E02CE130E00E942345C7ECDAE510
:10A4600082E090E064E170E0AE0121E00E94954559
:10A470008BE190E064E170E0AE0121E00E9495453F
:10A48000C2ECDAE582E090E06EE070E0AE0121E03F
:10A490000E94954582E090E062E170E04091010108
:10A4A00021E00E94E7458BE190E06EE070E0AE01B4
:10A4B00021E00E9495458BE190E062E170E04091DF
:10A4C000010121E00E94E7450E9486510E94C4518B
:10A4D0000E94F351DF91CF911F910F910895CF9377
:10A4E000DF93EC01888190E0019762E070E00E94C8
:10A4F0002F73DB011296AC0FBD1F22C0E881F0E084
:10A500003196E61BF70BEC0FFD1F80819E9189278A
:10A510008C93E881F0E03196E61BF70BEC0FFD1F02
:10A52000908198279083E881F0E03196E61BF70B45
:10A53000EC0FFD1F8C91908189278C9361507040A6
:10A5400061157105D9F6DF91CF9108950E943138D8
:10A5500088EE8093880510928D0582E380938905AB
:10A560008EEA80938E0582E090E090938B05809335
:10A570008A0587E090E09093900580938F0581E0B5
:10A5800080938C05109291050EC081E090E00E94AE
:10A590005A458091880582508093880580918D0569
:10A5A0008E5F80938D05E8E8F5E080918805893617
:10A5B00060F784E090E093838283148285E090E0EA
:10A5C000908787830EC081E090E00E945A45809179
:10A5D00089058E5F8093890580918E0582508093D6
:10A5E0008E05809189058C3670F38BE06FEF41E02A
:10A5F0000E945E3D80EF8093880580938D058CE0FE
:10A6000090E06EE070E04EE159E520E00E94954553
:10A6100088E790E00E945A4508950F931F9380E0C9
:10A6200090E063E070E04EE150E029E130E000E0CE
:10A6300010E00E94234583E090E064E070E047E58D
:10A640005BE520E00E94954583E090E065E070E0E6
:10A6500040E75BE520E00E94954583E090E066E0FE
:10A6600070E043E85BE520E00E94954583E090E0E0
:10A6700068E070E040E15CE520E00E94954583E001
:10A6800090E069E070E048E25CE520E00E949545DA
:10A6900083E090E06BE070E044ED5BE520E00E9439
:10A6A000954583E090E06CE070E04CEE5BE520E0E7
:10A6B0000E94954583E090E06DE070E041E05CE54C
:10A6C00020E00E94954583E090E06FE070E049E370
:10A6D0005CE520E00E94954583E090E060E170E059
:10A6E00041E55CE520E00E94954583E090E062E171
:10A6F00070E040E75BE520E00E94954583E090E054
:10A7000063E170E047E95BE520E00E94954583E066
:10A7100090E064E170E048EA5BE520E00E94954546
:10A7200083E090E065E170E040EC5BE520E00E94B2
:10A73000954580E00E94673881FFFBCF1F910F9104
:10A7400008950F931F9380E090E060E070E043E095
:10A7500050E02CE130E000E010E00E9423458BE166
:10A7600090E060E070E043E050E02CE130E00E94D7
:10A77000234582E090E066E070E041E050E026E0B2
:10A7800030E004EB10E00E9423458BE190E066E0AE
:10A7900070E041E050E026E030E00E94234582E096
:10A7A00090E06CE070E041E050E023E030E004E94C
:10A7B00010E00E9423458BE190E06CE070E041E006
:10A7C00050E023E030E00E9423451F910F9108954F
:10A7D0006130710571F42BE230E0829FF001839FBC
:10A7E000F00D929FF00D1124EA52F54F20812F5F5A
:10A7F00010C06115710571F42BE230E0829FF00109
:10A80000839FF00D929FF00D1124EA52F54F2081A5
:10A81000215020832BE230E0829FF001839FF00DD6
:10A82000929FF00D1124EA52F54F20812F3F19F429
:10A8300027E0208303C0283009F410822BE230E0A7
:10A84000829FF001839FF00D929FF00D1124EA5238
:10A85000F54F40819C01220F331F220F331F820FBF
:10A86000931FFC01E857FA4F453070F021E0248334
:10A8700050E0840F951F24E030E0241B350B220F9D
:10A88000331F820F931F03C01482840F911D938383
:10A8900082830895A0E0B0E0E0E5F4E50C948573D0
:10A8A0002BE230E0829FF001839FF00D929FF00D2C
:10A8B0001124EA52F54FE081F0E0E830F10508F0AC
:10A8C000F1C0E85CFF4F2BE230E00C94B673829F3E
:10A8D000F001839FF00D929FF00D1124EA52F54F85
:10A8E000138614861586168683899489A589B68968
:10A8F000B095A095909581959F4FAF4FBF4F5AC08F
:10A90000829FE001839FD00D929FD00D1124CA52E7
:10A91000D54FCB88DC88ED88FE88C701B60127E4D7
:10A9200030E040E050E00E94F072F4E68F2E912C6F
:10A93000A12CB12CA50194010E9464732B873C8744
:10A940004D875E87C701B60129EB3FEF4FEF5FEF01
:10A950005EC0829FF001839FF00D929FF00D112445
:10A96000EA52F54F83899489A589B6896FC0829F81
:10A97000E001839FD00D929FD00D1124CA52D54F74
:10A980006B897C898D899E8927E430E040E050E026
:10A9900077C0829FF001839FF00D929FF00D1124EC
:10A9A000EA52F54F13861486158616868389948994
:10A9B000A589B6898787908BA18BB28B73C0829F44
:10A9C000E001839FD00D929FD00D1124CA52D54F24
:10A9D000CB88DC88ED88FE88C701B60129EB3FEF04
:10A9E0004FEF5FEF0E94F072E4E68E2E912CA12CC7
:10A9F000B12CA50194010E9464732B873C874D877D
:10AA00005E87C701B60127E430E040E050E00E94D5
:10AA1000F072A50194010E9464732F87388B498BD3
:10AA20005A8B40C0829FF001839FF00D929FF00DE2
:10AA30001124EA52F54F83899489A589B689B09586
:10AA4000A095909581959F4FAF4FBF4F8387948777
:10AA5000A587B6871786108A118A128A23C0829F1B
:10AA6000E001839FD00D929FD00D1124CA52D54F83
:10AA70006B897C898D899E8929EB3FEF4FEF5FEFD2
:10AA80000E94F07224E630E040E050E00E946473DF
:10AA900089019A010B871C872D873E870F87188BAA
:10AAA000298B3A8BCDB7DEB7ECE00C94A1732BE287
:10AAB00030E0829FF001839FF00D929FF00D1124F2
:10AAC000EA52F54F8789908DA18DB28D43855485CB
:10AAD00065857685840F951FA61FB71F878B908F7E
:10AAE000A18FB28F838D948DA58DB68D47855089AA
:10AAF00061897289840F951FA61FB71F838F948F5A
:10AB0000A58FB68F08954F925F926F927F928F922A
:10AB10009F92AF92BF92CF92DF92EF92FF920F93EC
:10AB20001F934B015C0129013A01FF2420E83CE01E
:10AB3000E29EC001E39E900DF29E900D1124AA2783
:10AB400097FDA095BA2F881A990AAA0ABB0A10E0A5
:10AB5000029FC001039F900D129F900D1124AA2700
:10AB600097FDA095BA2F481A590A6A0A7B0AC501AF
:10AB7000B401A50194010E94F0726B017C01C30134
:10AB8000B201A30192010E94F072DC01CB01C80E58
:10AB9000D91EEA1EFB1EC701B6010E946F350E9436
:10ABA000257420E030E048EC52E40E9492340E9488
:10ABB000A1321F910F91FF90EF90DF90CF90BF9047
:10ABC000AF909F908F907F906F905F904F9008957F
:10ABD000A0E0B0E0EEEEF5E50C9483735C013A0181
:10ABE0004901CBE2D0E08C9FF0018D9FF00D9C9F3E
:10ABF000F00D1124EA52F54F268130E0C901880F8B
:10AC0000991F820F931F880F991F680F791F8781E3
:10AC1000680F711DDB018C918530A1F5878D90A1A6
:10AC2000A1A1B2A14385548565857685840F951FC2
:10AC3000A61FB71F845F9140A040B0408C3F28E022
:10AC4000920720E0A20720E0B20708F4A6C213860C
:10AC50001486158616868AE08816910408F49FC229
:10AC600081E090E08A199B098C9FF0018D9FF00D87
:10AC70009C9FF00D1124EA52F54F13861486158619
:10AC800016868DC2863071F583A194A1A5A1B6A1C7
:10AC90004785508961897289840F951FA61FB71F48
:10ACA000845F9140A040B0408C3F28E0920720E0B4
:10ACB000A20720E0B20708F470C21786108A118A32
:10ACC000128A8AE08816910408F469C281E090E053
:10ACD0008A199B098C9FF0018D9FF00D9C9FF00DB0
:10ACE000112454C2813009F091C0478D50A161A157
:10ACF00072A183859485A585B685480F591F6A1F63
:10AD00007B1F03A114A125A136A1CB01BA01A90182
:10AD1000980101E0EE24E3940E948355DC01CB010D
:10AD20008C319105A105B10528F484309105A10568
:10AD3000B10528F52BE230E0A29EF001A39EF00DB4
:10AD4000B29EF00D1124EA52F54F13861486158633
:10AD50001686AAE08A169104A0F081E090E08A1994
:10AD60009B09829FF001839FF00D929FF00D1124AB
:10AD7000EA52F54F138614861586168602C0C0E087
:10AD800001C0C1E08BE290E0A89EF001A99EF00D09
:10AD9000B89EF00D1124EA52F54FC78CD0A0E1A067
:10ADA000F2A023A134A145A156A187859089A1894C
:10ADB000B289280F391F4A1F5B1FC701B60101E086
:10ADC000EE24E3940E948355DC01CB018C31910584
:10ADD000A105B10530F484309105A105B10508F055
:10ADE000DFC12BE230E0A29EF001A39EF00DB29EE7
:10ADF000F00D1124EA52F54F1786108A118A128A33
:10AE0000BAE08B16910408F4CAC1B5C1823009F0CA
:10AE10008FC0478D50A161A172A183859485A585BE
:10AE2000B685480F591F6A1F7B1F03A114A125A1D6
:10AE300036A1CB01BA01A901980101E0EE240E94DC
:10AE40008355DC01CB018C319105A105B10528F4B6
:10AE500084309105A105B10528F52BE230E0A29ED2
:10AE6000F001A39EF00DB29EF00D1124EA52F54FB1
:10AE70001386148615861686EAE08E169104A0F0D5
:10AE800081E090E08A199B09829FF001839FF00D79
:10AE9000929FF00D1124EA52F54F13861486158601
:10AEA000168602C0C0E001C0C1E08BE290E0A89E1F
:10AEB000F001A99EF00DB89EF00D1124EA52F54F55
:10AEC000C78CD0A0E1A0F2A023A134A145A156A136
:10AED00087859089A189B289280F391F4A1F5B1F76
:10AEE000C701B60101E0EE240E948355DC01CB01CD
:10AEF0008C319105A105B10530F484309105A1058F
:10AF0000B10508F04DC12BE230E0A29EF001A39EF6
:10AF1000F00DB29EF00D1124EA52F54F1786108AFB
:10AF2000118A128AFAE08F16910408F438C123C1FD
:10AF3000833009F091C0478D50A161A172A1838532
:10AF40009485A585B685480F591F6A1F7B1F03A1ED
:10AF500014A125A136A1CB01BA01A901980100E0F5
:10AF6000EE24E3940E948355DC01CB018C319105E2
:10AF7000A105B10528F484309105A105B10528F596
:10AF80002BE230E0A29EF001A39EF00DB29EF00DE8
:10AF90001124EA52F54F13861486158616868AE028
:10AFA00088169104A0F081E090E08A199B09829FA5
:10AFB000F001839FF00D929FF00D1124EA52F54F9E
:10AFC000138614861586168602C0C0E001C0C1E053
:10AFD0008BE290E0A89EF001A99EF00DB89EF00DC6
:10AFE0001124EA52F54FC78CD0A0E1A0F2A023A112
:10AFF00034A145A156A187859089A189B289280FDE
:10B00000391F4A1F5B1FC701B60100E0EE24E3941D
:10B010000E948355DC01CB018C319105A105B1055E
:10B0200030F484309105A105B10508F0B9C02BE2D8
:10B0300030E0A29EF001A39EF00DB29EF00D11240F
:10B04000EA52F54F1786108A118A128AAAE08A16E8
:10B05000910408F4A4C08FC0843009F09EC0478DCD
:10B0600050A161A172A183859485A585B685480FFD
:10B07000591F6A1F7B1F03A114A125A136A1CB0173
:10B08000BA01A901980100E0EE240E948355DC0179
:10B09000CB018C319105A105B10528F484309105CF
:10B0A000A105B10528F52BE230E0A29EF001A39E98
:10B0B000F00DB29EF00D1124EA52F54F138614865E
:10B0C00015861686BAE08B169104A0F081E090E018
:10B0D0008A199B09829FF001839FF00D929FF00DCA
:10B0E0001124EA52F54F138614861586168602C07F
:10B0F000C0E001C0C1E08BE290E0A89EF001A99EF3
:10B10000F00DB89EF00D1124EA52F54FC78CD0A077
:10B11000E1A0F2A023A134A145A156A18785908981
:10B12000A189B289280F391F4A1F5B1FC701B601C9
:10B1300000E0EE240E948355DC01CB018C319105A7
:10B14000A105B10528F484309105A105B10540F5AC
:10B150002BE230E0A29EF001A39EF00DB29EF00D16
:10B160001124EA52F54F1786108A118A128AEAE0F2
:10B170008E169104A0F081E090E08A199B09829FCD
:10B18000F001839FF00D929FF00D1124EA52F54FCC
:10B190001786108A118A128A02C0C0E001C0C1E07D
:10B1A000A614B70408F1CC23F9F08BE290E0A89E36
:10B1B0008001A99E100DB89E100D11240A52154F42
:10B1C000D8019A968C919A97882371F4C50161E011
:10B1D00070E00E94E853F801858190E0A0E0B0E0C3
:10B1E000838B948BA58BB68B8C2FCDB7DEB7EEE01F
:10B1F0000C949F73AEE0B0E0E0E0F9E50C947F734F
:10B200009E878D874090E10A5090E20A6090E30AA1
:10B210007090E40A20910C0B30910D0B40910E0BB5
:10B2200050910F0B29833A834B835C830091ED0A85
:10B230001091EE0A2091EF0A3091F00A8091180BDC
:10B240009091190BA0911A0BB0911B0B081B190BB5
:10B250002A0B3B0B040D151D261D371D89819A8174
:10B26000AB81BC81081B190B2A0B3B0B69ED262E09
:10B270006FEF362EACE0BBE02A0E3B1E8091E50A54
:10B280009091E60AA091E70AB091E80A8D839E8327
:10B29000AF83B8878091100B9091110BA091120B86
:10B2A000B091130B89879A87AB87BC87C090F10A4E
:10B2B000D090F20AE090F30AF090F40A80911C0B0F
:10B2C00090911D0BA0911E0BB0911F0BC81AD90AAB
:10B2D000EA0AFB0A8D819E81AF81B885C80ED91E0E
:10B2E000EA1EFB1E89859A85AB85BC85C81AD90ADA
:10B2F000EA0AFB0AC901B801A90198010E94F0728B
:10B300004B015C01C701B601A70196010E94F072D2
:10B31000DC01CB01880E991EAA1EBB1EC501B4011B
:10B320000E946F350E94257420E030E048EC52E422
:10B330000E9492340E94A132DC01CB018930910538
:10B34000A105B10508F078C069817A818B819C8163
:10B35000640D751D861D971D22E0C22ED12CE12C97
:10B36000F12CA70196010E9464732093E10A3093A7
:10B37000E20A4093E30A5093E40A20930C0B3093C3
:10B380000D0B40930E0B50930F0B6D817E818F81BF
:10B39000988529853A854B855C85620F731F841FCC
:10B3A000951FA70196010E9464732093E50AD101BD
:10B3B00011963C93119712964C93129713965C93A7
:10B3C00013972093100B3093110B4093120B509353
:10B3D000130BED85FE85309789F580912B0B882323
:10B3E00069F581E090E061E070E00E94E8538091AF
:10B3F000060B90E0A0E0B0E08093140B9093150B47
:10B40000A093160BB093170B8091000B8823B1F417
:10B4100080E090E061E070E00E94E8538091DB0AF8
:10B4200090E0A0E0B0E08093E90A9093EA0AA0934C
:10B43000EB0AB093EC0A02C080E001C081E02E96D6
:10B44000E2E10C949B73A0E0B0E0E9E2FAE50C9431
:10B4500088737C016B018BE290E0E89EF001E99E2D
:10B46000F00DF89EF00D1124EA52F54F2381DB0117
:10B470008C91223020F0C22FD0E0219702C0C82F3B
:10B48000D0E0281720F4E22FF0E0319602C0E1E08E
:10B49000F0E08BE290E0E89ED001E99EB00DF89ECE
:10B4A000B00D1124AA52B54F16963C9116971796D7
:10B4B0008C91179790E0AC01440F551F13E0880F53
:10B4C000991F1A95E1F7480F591F430F511DEC0DB5
:10B4D000FD1D808190E04817590729F42F5F1396CE
:10B4E0002C93139720C0F601EC0FFD1F808190E094
:10B4F00048175907C1F412968C911297882339F096
:10B50000213029F48F5F12968C930E94F3518BE2C5
:10B5100090E0E89EF001E99EF00DF89EF00D1124F8
:10B52000EA52F54FC3838BE290E0E89EF001E99E7A
:10B53000F00DF89EF00D1124EA52F54F9381D601DB
:10B540008C91891718F481E0838381A78BE290E0C6
:10B55000E89EE001E99ED00DF89ED00D1124CA525C
:10B56000D54F1A81112309F481C089A5882309F4D4
:10B570007DC0F6010281802F0E94D64CB82ED601E4
:10B580001196CC908C2D0E94D64CB81668F44BA125
:10B590005CA16DA17EA1443FB1E05B07B0E06B0709
:10B5A000B0E07B070CF452C08B15B8F42BE230E00E
:10B5B000E29EF001E39EF00DF29EF00D1124EA529E
:10B5C000F54F83A194A1A5A1B6A18932EAE09E0717
:10B5D000E0E0AE07E0E0BE07CCF5802F0E94D14C42
:10B5E000C82F8C2D0E94D14CC817B8F42BE230E044
:10B5F000E29EF001E39EF00DF29EF00D1124EA525E
:10B60000F54F478D50A161A172A1443FF1E05F0762
:10B61000F0E06F07F0E07F07CCF08C1738F58BE295
:10B6200090E0E89EF001E99EF00DF89EF00D1124E7
:10B63000EA52F54F878D90A1A1A1B2A189322AE0EB
:10B64000920720E0A20720E0B20784F08BE290E0AE
:10B65000E89EE001E99ED00DF89ED00D1124CA525B
:10B66000D54F11501A830E94F35119A6CDB7DEB7FA
:10B67000E9E00C94A473EF92FF920F931F93CF9382
:10B68000DF937B01EA013091D80A2091030B321736
:10B6900021F0321708F095C08AC02091FF0A30913E
:10B6A0002A0B231721F0222309F48BC080C020919C
:10B6B000D90A3091040B231721F0321708F081C00A
:10B6C00076C0FC013081231721F030E02F5F3F4F1F
:10B6D00002C021E030E0820F931FFC010081802F27
:10B6E0000E94D64C9091DD0A9817E8F44091F10A37
:10B6F0005091F20A6091F30A7091F40A80911C0B48
:10B7000090911D0BA0911E0BB0911F0B84179507F4
:10B71000A607B7070CF44BC0481759076A077B0701
:10B720000CF056C04EC08917D8F44091F10A5091E0
:10B73000F20A6091F30A7091F40A80911C0B9091C7
:10B740001D0BA0911E0BB0911F0B481759076A07DC
:10B750007B076CF184179507A607B707CCF531C0B6
:10B76000802F0E94D14C9091DC0A4091ED0A5091BB
:10B77000EE0A6091EF0A7091F00A0091180B109197
:10B78000190B20911A0B30911B0B891758F4401795
:10B790005107620773075CF0041715072607370780
:10B7A000BCF40FC004171507260737072CF481E0F7
:10B7B0008093DA0A82E009C04017510762077307D5
:10B7C0003CF482E08093DA0A81E08093050B04C0A8
:10B7D0001092DA0A1092050B8091DA0A90E08E1529
:10B7E0009F05E9F08091D80A8823C9F08091030B66
:10B7F0008823A9F00E948651C130D10529F4809197
:10B80000050B813061F402C0209749F48091B50A9C
:10B81000882329F489E06FEF41E00E945E3DCDB7B7
:10B82000DEB7E6E00C94A7732BE230E0829FF001D4
:10B83000839FF00D929FF00D1124EA52F54F8389FA
:10B840009489A589B6890296A11DB11D838B948B1D
:10B85000A58BB68B458150E060E070E04817590732
:10B860006A077B0724F4438B548B658B768B089592
:10B870002BE230E0829FF001839FF00D929FF00D4C
:10B880001124EA52F54F83899489A589B6890297D4
:10B89000A109B109838B948BA58BB68B2581269545
:10B8A00030E0309521953F4FA901662757FD6095FF
:10B8B000762F84179507A607B70724F4438B548B7C
:10B8C000658B768B08952BE230E0829FF001839F99
:10B8D000F00D929FF00D1124EA52F54F838994895F
:10B8E000A589B689181619061A061B0644F401978D
:10B8F000A109B109838B948BA58BB68B0895009712
:10B90000A105B10539F00196A11DB11D838B948B62
:10B91000A58BB68B08952BE230E0829FF001839FC8
:10B92000F00D929FF00D1124EA52F54F818188238A
:10B9300091F08150818386E985836B35710510F024
:10B940000E94C4518091B50A882329F48AE060E4FA
:10B9500041E00E945E3D0895A6E2B0E0E2EBFCE526
:10B960000C947F739E8F8D8F7CA36BA35A8B498B16
:10B970001A8619861C861B861E821D8218861F82C7
:10B980001A8219821C821B820E94A15380912D0B66
:10B9900091E0892708EC809F002D1124F09001018F
:10B9A0002EED3AE069E875E040E011E054E6F90177
:10B9B0003897DB0113968C911397880F880F119697
:10B9C0009C91890F841B8083F90113821482158254
:10B9D0001682D90117821086118612861386148664
:10B9E00015861686349710821C92F90137970083CA
:10B9F000F9013697F082F90135971083FB013197F1
:10BA00008081859FC0011124AA2797FDA095BA2F98
:10BA1000F9018787908BA18BB28BDB018C91859F7D
:10BA2000C0011124AA2797FDA095BA2F838B948B70
:10BA3000A58BB68B11A210A2178E4B5F255D3F4FD1
:10BA40006B5F7F4F4A3009F0B2CF29893A892115BF
:10BA5000310549F48DE090E06CE070E041EE5AE58C
:10BA600020E00E9495458CE390E00E945A4582E0D8
:10BA700090E066E070E041E050E023E030E00FE766
:10BA800010E00E9423458BE190E066E070E041E029
:10BA900050E023E030E00E9423458091B50A8823DE
:10BAA00029F487E06FEF41E00E945E3D8CE390E077
:10BAB0000E945A4582E090E069E070E041E050E089
:10BAC00023E030E00FE710E00E9423458BE190E097
:10BAD00069E070E041E050E023E030E00E9423455F
:10BAE0008091B50A882329F487E06FEF41E00E9436
:10BAF0005E3D8CE390E00E945A4582E090E06CE06D
:10BB000070E041E050E023E030E006EA10E00E94FF
:10BB100023458BE190E06CE070E041E050E023E0F1
:10BB200030E00E9423458091B50A882329F486E0FD
:10BB30006FEF41E00E945E3D1E861D861A8E198EB3
:10BB400089899A8901979EA38DA381E090E00E9444
:10BB50005A45AD85BE85AA35B10581F40E941452BF
:10BB60008091330B882379F40E94117463E070E0B4
:10BB70000E942F7301960E94254605C0ED85FE8523
:10BB8000EB35F10530F42D853E852F5F3F4F3E8725
:10BB90002D8779E0672E712C6C0E7D1E2E01089486
:10BBA000411C511C9E012B5F3F4F388B2F87E8E8CB
:10BBB000AE2EE5E0BE2EFCEDCF2EFAE0DF2E8601A4
:10BBC00006501040A7E08A2E912C800E911E19017C
:10BBD000EE24FF248E2D0E9467389C01D3018D93A3
:10BBE0009D933D01F201819191912F012095309516
:10BBF00082239323D1018D939D931D01F5018081B3
:10BC000090E0449760E270E00E942F73D6016C933D
:10BC1000818190E00C9760E270E00E942F73F40144
:10BC20006083D6018C9190E0E0E8FCE08E9FA0015B
:10BC30008F9F500D9E9F500D1124662757FD6095D4
:10BC4000762FF8018789908DA18DB28D841B950B7D
:10BC5000A60BB70B805D9740A040B040878F90A3A4
:10BC6000A1A3B2A3D4018C9190E0E0E8FCE08E9F08
:10BC7000A0018F9F500D9E9F500D1124662757FDE8
:10BC80006095762FF801838D948DA58DB68D841BDC
:10BC9000950BA60BB70B805B9440A040B04083A3EC
:10BCA00094A3A5A3B6A32DA13EA12E153F0590F404
:10BCB0008091310B9091320B8130910521F43BE45E
:10BCC0003093060B0BC08230910521F48AE68093F5
:10BCD000060B04C0E4E6D8011596EC93C7016D8D00
:10BCE0007E8D0E94235A0894E11CF11C25E030E06F
:10BCF000A20EB31E8BE290E0C80ED91E055D1F4F49
:10BD0000880E991E92E0E916F10409F063CF809144
:10BD1000D80AA989BA89A130B10579F08823C1F47C
:10BD20008091030B8823A1F4ED85FE85EB3FF1059F
:10BD3000C8F53196FE87ED870BC0882349F42D8521
:10BD40003E852B3F310570F52F5F3F4F3E872D8796
:10BD50008D859E858B35910551F46091DA0A8D8D24
:10BD60009E8D70E049895A890E943B5B1EC0AD855B
:10BD7000BE85AC35B105C9F40E9486518091330B64
:10BD8000882399F40E948E3AE989FA89E130F10515
:10BD9000C1F48091D80A882389F48091030B882309
:10BDA00069F00FC02224239401C0222409EE1AE076
:10BDB000EE24FF24AA24AA94BA2CE5C08CEB94E5C7
:10BDC00002C082E794E50E94653AEFCFCE2C8E2D1B
:10BDD0000E94673893FF0BC0C7016D857E850E9466
:10BDE0008B5CD80155961C921E92549781C0F80125
:10BDF000848995898A309105A9F480819181A281F5
:10BE0000B3814396A11DB11D87329105A105B105EE
:10BE100028F1C70161E070E00E94E85381E090E002
:10BE2000D8013DC0BFEF863F9B07C1F4F801808178
:10BE30009181A281B3814396A11DB11D87329105E5
:10BE4000A105B10558F0C70160E070E00E94E85319
:10BE5000D8015596BC92AE9254974AC08C2D0E9440
:10BE6000673887FF21C0F80184899589009789F494
:10BE700080819181A281B3814396A11DB11D87323A
:10BE80009105A105B10528F0C70161E070E00E94AD
:10BE9000E853D80154968D919C91559701965596EB
:10BEA0009C938E93549724C08C2D0E946738F80180
:10BEB00086FF1CC084899589009789F480819181CF
:10BEC000A281B3814396A11DB11D87329105A105C1
:10BED000B10528F0C70160E070E00E94E853D80186
:10BEE00054968D919C9155970197D9CF158A148AB4
:10BEF0008C2D0E94673880FF04C0C7010E94145C2B
:10BF00000CC08C2D0E94673881FF04C0C7010E94BD
:10BF1000385C03C0C7010E94635CAF85B8898D910E
:10BF20009D91B88BAF878830910571F0B4E0803077
:10BF30009B0721F580912C0B882301F589E06FEF99
:10BF400041E00E945E3D1AC0C7010E94664B282E48
:10BF50008BA19CA10E94ED4A8D8D9E8D0E94BC4FAD
:10BF60000E94145280E090E062E070E00E94E8538A
:10BF700081E090E062E070E00E94E8530894E11CE8
:10BF8000F11C055D1F4FE989FA89EE16FF0609F0DD
:10BF90001DCF9E01295F3F4F38A32F8F0BE01BE081
:10BFA000C80180969E8B8D8BD8011197BC8FAB8F6B
:10BFB000F8013297FC8BEB8B98012A503040388F78
:10BFC0002F8B81E090E0988B8F8755245394480104
:10BFD00099C1AD89BE891C92EB89FC89808185302D
:10BFE00009F41082AB89BC898C91882351F40E949A
:10BFF0001174EB8DFC8D8083AB89BC898C918F5F34
:10C000008C93EB8DFC8D4080A42CBB24F3E0AF22FD
:10C01000BB242091310B3091320B3AA329A322305B
:10C02000310529F432E0A316B10448F40CC089A10B
:10C030009AA1009741F493E0A916B10421F4AEEF60
:10C04000BFEFAA0EBB1EF40137978081ED8DFE8DE8
:10C050009081891718F490E0019602C081E090E089
:10C060002D8D3E8D820F931FDC016C90862D0E94DA
:10C07000D14C182FF401349770807816A8F5EF8909
:10C08000F88D0081023081F1D40159966D917D9136
:10C090008D919C915C9724E630E040E050E00E9456
:10C0A000647369017A01C501880F991F0796A0E0A2
:10C0B000B0E082179307A407B507B4F4882799273F
:10C0C0008A199B09880F991F4896A0E0B0E0C8160E
:10C0D000D906EA06FB0644F4802F825061E070E046
:10C0E000843008F0A4C0A1C0171588F5EF89F88D39
:10C0F000F080F6E0FF1659F1D40159966D917D91CB
:10C100008D919C915C9724E630E040E050E00E94E5
:10C11000647389019A01C501880F991F0796A0E0F1
:10C12000B0E080179107A207B3078CF488279927FE
:10C130008A199B09880F991F4896A0E0B0E008175C
:10C1400019072A073B071CF48F2D83506AC0862DE0
:10C150000E94D64C182FF40133977080871570F524
:10C16000EF89F88D0081002349F1D40155966D9136
:10C170007D918D919C91589724E630E040E050E00D
:10C180000E946473C501880F991F0796A0E0B0E074
:10C1900082179307A407B5078CF4882799278A1973
:10C1A0009B09880F991F4896A0E0B0E0281739072F
:10C1B0004A075B071CF4802F855033C0711608F0C6
:10C1C00040C0EF89F88DF080F4E0FF16D1F1D40182
:10C1D00055966D917D918D919C91589724E630E014
:10C1E00040E050E00E94647389019A01C501880F04
:10C1F000991F0796A0E0B0E080179107A207B30748
:10C2000004F5882799278A199B09880F991F489652
:10C21000A0E0B0E0081719072A073B0794F48F2D18
:10C22000815061E070E0833010F060E070E08F8555
:10C2300098890E94E853F4015082AD89BE895C92CE
:10C240002BC0F4018081882371F0842D869586951A
:10C25000AB8DBC8D8C93EB89FC8980818F5F808353
:10C26000D4011C9219C0E9A1FAA1E230F105A1F4B0
:10C27000F40181859285A385B48584369105A10555
:10C28000B10554F02D853E852B35310528F08F857D
:10C290009889B9010E948B5C8F8598890E94145CF3
:10C2A00089899A89009751F4AF8DB8A18D919C919D
:10C2B00011978830910511F422242394EF85F88991
:10C2C0003197F88BEF872F8D38A12250304038A35B
:10C2D0002F8F85ED9FEF880E991EAD89BE899B97A4
:10C2E000BE8BAD8BEB8DFC8DBB97FC8FEB8F2B89C1
:10C2F0003C892B5230403C8B2B8B8F89988D8B97B0
:10C30000988F8F8BAF85B889E989FA89AE17BF07F7
:10C3100028F0FFEFAF3FBF0709F05BCE80E090E071
:10C320000E944A5481E090E00E944A548091300B70
:10C33000882389F489899A890E94FA58282F30E045
:10C340008901000F111F53E0220F331F5A95E1F7A7
:10C35000020F131F02C000E010E080E090E06BA12C
:10C360007CA149895A8998010E94E855080F111D3E
:10C3700081E090E06BA17CA149895A8998010E94D3
:10C38000E8559801280F311DC901009771F0898D7A
:10C390009A8D009789F488E06FEF41E00E945E3D3E
:10C3A000AAE0B0E0BA8FA98F07C0E98DFA8D309767
:10C3B00019F03197FA8FE98F80E090E00E9457558D
:10C3C00081E090E00E9457556091ED0A7091EE0A6D
:10C3D0008091EF0A9091F00A24E6C22ED12CE12C34
:10C3E000F12CA70196010E94647320938805609147
:10C3F000F10A7091F20A8091F30A9091F40AA70170
:10C4000096010E946473209389056091180B7091C6
:10C41000190B80911A0B90911B0BA70196010E949A
:10C42000647320938D0560911C0B70911D0B80919E
:10C430001E0B90911F0BA70196010E94647320931D
:10C440008E0589859A859A8389838B859C859C83B3
:10C450008B83222009F479CBA696E2E10C949B739E
:10C46000A2E4B0E0E6E3F2E60C948C73F62E8E01C3
:10C470000F5F1F4F2EE1F80111922A95E9F7B801DD
:10C480000E94514EFF2019F0C8010E946F52C8014E
:10C49000BE01615E7F4F0E94DE4CCE014F960E942E
:10C4A000ED4AC8010E94BC4FC801BE01615E7F4FCA
:10C4B00040E050E00E94AC5CCE5BDF4FE5E00C94C6
:10C4C000A873A2E4B0E0E7E6F2E60C9481732C01D5
:10C4D00000910201109103017E010894E11CF11CFE
:10C4E0008EE1F70111928A95E9F7C801B7010E9420
:10C4F000514E2FE1C22ED12CCC0EDD1EC701B6014C
:10C500000E94DE4CC6010E94ED4AC7010E94BC4F4A
:10C51000C8010E942D5131E0A32EB12C49E0742EA8
:10C520006624639401C0540181E090E00E945A4562
:10C5300080E00E9467384C01A094B094A822B922F0
:10C54000A2FE04C0C7010E946F521BC0A7FE0CC010
:10C550000F5F1F4F80912E0B90912F0B801791072B
:10C5600060F401E010E009C0A6FE16C001501040C2
:10C5700021F400912E0B10912F0BC801B7010E94DE
:10C58000514EC701B6010E94DE4CC6010E94ED4A21
:10C59000C7010E94BC4F17C0A4FE0AC080910101D0
:10C5A0008F5F809301018A3070F0609201010BC0AF
:10C5B000A5FE0CC080910101815080930101882368
:10C5C00011F470920101C8010E942D51F8E0AF16DC
:10C5D000B10409F0A8CF0E948E3A10930301009392
:10C5E0000201CE010196BE01615E7F4FA2010E9451
:10C5F000AC5CCE5BDF4FE0E10C949D73A3E9B0E04F
:10C60000E4E0F3E60C947F739E012F593F4FCB5724
:10C61000DF4F39832883C558D04084E2F901119255
:10C620008A95E9F74FE1E42EF12CEC0EFD1E8EE128
:10C63000F70111928A95E9F70E948E3A0E943138EB
:10C6400083E090E062E070E048E150E028E130E013
:10C650000EE710E00E9423458FE090E06AE070E072
:10C6600044E050E024E030E004E910E00E9423457B
:10C670000E94117463E070E00E942F7301960E9483
:10C68000254601E010E05FEF252E312CC557DF4F26
:10C690001882CB58D040C957DF4F19821882C7582B
:10C6A000D04062E0C62ED12C73E0A72EB12C4501FC
:10C6B00056010BC0C557DF4F1882CB58D040C15729
:10C6C000DF4F08811981CF58D04081E090E00E946F
:10C6D0005A4580E00E946738C157DF4F99838883AD
:10C6E000CF58D04080E00E9467389801282739272A
:10C6F000C157DF4F48815981CF58D040242335237B
:10C70000C757DF4F39832883C958D04027FF49C115
:10C7100055E08516910408F044C1A4014F5F5F4FB6
:10C72000FA01EE0FFF1FE40FF51FEE0FFF1FEA0DDA
:10C73000FB1D81E690E08C0F9D1FE80FF91F8081A3
:10C7400018168CF4C501880F991F9501B3E0220FCC
:10C75000331FBA95E1F7820F931F840F951F82153F
:10C76000930509F01EC1C957DF4FE881F981C75809
:10C77000D040E230F105D8F0C1016AE070E00E94DB
:10C780001B739B01EDE1F0E0EC0FFD1FC957DF4F7C
:10C7900048815981C758D040E40FF51F80816AE075
:10C7A0000E940F7390E02817390709F4FAC0C401FA
:10C7B000880F991F880F991FB501660F771F660FA5
:10C7C000771F6E5F7F4F039644E050E024E030E037
:10C7D0000EE710E00E9423459501220F331FC5018B
:10C7E000F3E0880F991FFA95E1F7280F391F4F8D55
:10C7F000042F10E0C901880D991D8017910759F485
:10C80000C1016AE070E00E941B738816990618F057
:10C81000089481089108C9010196880D991D821517
:10C82000930519F554E085169104E0F4C1016AE01E
:10C8300070E00E941B730196FC01EE0FFF1FE80FD2
:10C84000F91FEE0FFF1FE60FF71F81E690E08C0F38
:10C850009D1FE80FF91F8081181624F00894811C91
:10C86000911C03C0089481089108C957DF4FE881E3
:10C87000F981C758D040E130F10551F5F5E08F1648
:10C88000910430F5C1016AE070E00E941B730196CB
:10C89000FC01EE0FFF1FE80FF91FEE0FFF1FE60F61
:10C8A000F71F81E690E08C0F9D1FE80FF91F808134
:10C8B000882369F0C901880D991D910121503040EC
:10C8C0008217930729F408948108910801C05B013D
:10C8D0000894811C911C3401660C771C660C771C33
:10C8E0006501CC0CDD1CCC0CDD1CC957DF4FE88189
:10C8F000F981C758D040E230F10508F445C0750110
:10C90000EE0CFF1CC50173E0880F991F7A95E1F7C3
:10C91000E80EF91EE80CF91CE016F10611F40C946F
:10C920002272842F6AE00E940F73682F70E086EFF6
:10C930009FEF689F9001699F300D789F300D112403
:10C94000240F311D220F331F220F331F660F771F55
:10C95000660F771F6E5F7F4FC901039644E050E07A
:10C9600024E030E00FE710E00E9423450C9422728F
:10C97000B6016E5F7F4FC301039644E050E024E0B0
:10C9800030E006EA10E00BC0B6016E5F7F4FC301D6
:10C99000039644E050E024E030E004E910E00E9417
:10C9A0002345C757DF4FF881C958D040F6FF47C12C
:10C9B0008114910409F443C1A40141505040FA018B
:10C9C000EE0FFF1FE40FF51FEE0FFF1FEA0DFB1D1B
:10C9D00021E630E02C0F3D1FE20FF31F8081181677
:10C9E0008CF4C501880F991F9501B3E0220F331F06
:10C9F000BA95E1F7820F931F840F951F8215930557
:10CA000009F01DC1C957DF4F48815981C758D0402F
:10CA100042305105D8F0C1016AE070E00E941B73FA
:10CA20009B01EDE1F0E0EC0FFD1FC957DF4F88815E
:10CA30009981C758D040E80FF91F80816AE00E94B1
:10CA40000F7390E02817390709F4F9C0C401880F63
:10CA5000991F880F991FB501660F771F660F771F03
:10CA60006E5F7F4F039644E050E024E030E00EE735
:10CA700010E00E9423459501220F331FC501F3E00A
:10CA8000880F991FFA95E1F7280F391F4F8D042F52
:10CA900010E0C901880D991D8017910759F4C10153
:10CAA0006AE070E00E941B738815990518F00894DD
:10CAB000811C911CC9010197880D991D8215930550
:10CAC00019F592E089169104E0F0C1016AE070E086
:10CAD0000E941B730197FC01EE0FFF1FE80FF91F67
:10CAE000EE0FFF1FE60FF71F81E690E08C0F9D1FF2
:10CAF000E80FF91F8081181624F008948108910826
:10CB000003C00894811C911CC957DF4FE881F9814B
:10CB1000C758D040E130F10549F58114910431F155
:10CB2000C1016AE070E00E941B730197FC01EE0FE7
:10CB3000FF1FE80FF91FEE0FFF1FE60FF71F81E63B
:10CB400090E08C0F9D1FE80FF91F8081882369F00A
:10CB5000C901880D991D91012F5F3F4F82179307DF
:10CB600029F40894811C911C01C05B010894810880
:10CB700091083401660C771C660C771C6501CC0C9F
:10CB8000DD1CCC0CDD1CC957DF4FE881F981C7588B
:10CB9000D040E230F10508F445C07501EE0CFF1CF1
:10CBA000C50123E0880F991F2A95E1F7E80EF91EC9
:10CBB000E80CF91CE016F10611F40C942B72842F8A
:10CBC0006AE00E940F73682F70E086EF9FEF689F06
:10CBD0009001699F300D789F300D1124240F311D75
:10CBE000220F331F220F331F660F771F660F771F29
:10CBF0006E5F7F4FC901039644E050E024E030E0CF
:10CC00000FE710E00E9423450C942B72B6016E5F73
:10CC10007F4FC301039644E050E024E030E006EA91
:10CC200010E00BC0B6016E5F7F4FC301039644E076
:10CC300050E024E030E004E910E00E942345C757AB
:10CC4000DF4FF881C958D040F5FF62C125E0A21638
:10CC5000B10408F05DC1F401EE0FFF1FE80DF91DEE
:10CC6000EE0FFF1F41E650E04C0F5D1FE40FF51F74
:10CC7000EA0DFB1D81811816A4F49401265F3F4F35
:10CC8000C501880F991FA50163E0440F551F6A95E0
:10CC9000E1F7840F951F280F391F2215330509F07E
:10CCA00037C1C957DF4F88819981C758D04082303A
:10CCB000910510F1EDE1F0E0EC0FFD1FE80FF91F19
:10CCC000E081C1016AE070E00E941B73DC018E2FDD
:10CCD0006AE00E940F73282F30E046EF5FEF249F39
:10CCE000C001259F900D349F900D11248E0F911D32
:10CCF000A817B90709F40CC1C401880F991F880F40
:10CD0000991FB501660F771F660F771F6E5F7F4F04
:10CD1000039644E050E024E030E00EE710E00E948B
:10CD200023451F8D412E5524C501880F991F95015C
:10CD3000A3E0220F331FAA95E1F7820F931F880DFE
:10CD4000991D8415950559F4C1016AE070E00E94AF
:10CD50001B73A616B70618F00894A108B108940131
:10CD6000265F3F4FC501880F991FA50163E0440F5F
:10CD7000551F6A95E1F7840F951F280F391F22155B
:10CD8000330511F594E0A916B104D8F4C1016AE0A5
:10CD900070E00E941B73FC01EE0FFF1FE80FF91FEC
:10CDA000EE0FFF1F21E630E02C0F3D1FE20FF31FB7
:10CDB000E60FF71F8181181624F00894A11CB11CFE
:10CDC00003C00894A108B108C957DF4F48815981B1
:10CDD000C758D0404130510591F555E0A516B10432
:10CDE00070F5C1016AE070E00E941B73FC01EE0F58
:10CDF000FF1FE80FF91FEE0FFF1F21E630E02C0F99
:10CE00003D1FE20FF31FE60FF71F21812223B1F030
:10CE10009501220F331FC50163E0880F991F6A95A2
:10CE2000E1F7280F391F280D391DC1010A9728176E
:10CE3000390729F40894A108B10801C04C010894ED
:10CE4000A11CB11C3401660C771C660C771C6501B3
:10CE5000CC0CDD1CCC0CDD1CC957DF4F488159813F
:10CE6000C758D0404230510508F445C07501EE0C5A
:10CE7000FF1CC50123E0880F991F2A95E1F7E80EF2
:10CE8000F91EE80CF91CE414F50411F40C94347246
:10CE9000812F6AE00E940F73682F70E086EF9FEF8A
:10CEA000689F9001699F300D789F300D1124210FEC
:10CEB000311D220F331F220F331F660F771F660F9E
:10CEC000771F6E5F7F4FC901039644E050E024E076
:10CED00030E00FE710E00E9423450C943472B60155
:10CEE0006E5F7F4FC301039644E050E024E030E0E2
:10CEF00006EA10E00BC0B6016E5F7F4FC3010396D8
:10CF000044E050E024E030E004E910E00E942345D2
:10CF1000C757DF4F5881C958D04054FF5BC1A11497
:10CF2000B10409F457C1F401EE0FFF1FE80DF91D1C
:10CF3000EE0FFF1F81E690E08C0F9D1FE80FF91F99
:10CF4000EA0DFB1D319780811816A4F494012A5034
:10CF50003040C501880F991FA50163E0440F551F9C
:10CF60006A95E1F7840F951F280F391F22153305A5
:10CF700009F030C1C957DF4FE881F981C758D04067
:10CF8000E230F10540F1EDE1F0E0EC0FFD1FC95793
:10CF9000DF4F28813981C758D040E20FF31FE0816D
:10CFA000C1016AE070E00E941B73DC018E2F6AE011
:10CFB0000E940F73282F30E046EF5FEF249FC001DF
:10CFC000259F900D349F900D11248E0F911DA81751
:10CFD000B90709F4FFC0C401880F991F880F991F72
:10CFE000B501660F771F660F771F6E5F7F4F039641
:10CFF00044E050E024E030E00EE710E00E942345DA
:10D000004F8D042F10E0C501880F991F9501A3E0F3
:10D01000220F331FAA95E1F7820F931F880D991DE8
:10D020008017910759F4C1016AE070E00E941B73F8
:10D030006A157B0518F00894A11CB11C9501220FFC
:10D04000331FC50153E0880F991F5A95E1F7280F48
:10D05000391F280D391DC9010A978215930541F51D
:10D0600052E0A516B104E0F0C1016AE070E00E9450
:10D070001B73FC01EE0FFF1FE80FF91FEE0FFF1FE0
:10D0800081E690E08C0F9D1FE80FF91FE60FF71F58
:10D0900031978081181624F00894A108B10808C0BF
:10D0A000C1010A962817390719F40894A11CB11C6C
:10D0B000C957DF4FE881F981C758D040E130F10509
:10D0C00001F5A114B104E9F0C1016AE070E00E9429
:10D0D0001B73FC01EE0FFF1FE80FF91FEE0FFF1F80
:10D0E00021E630E02C0F3D1FE20FF31FE60FF71F84
:10D0F00031972081222321F00894A11CB11C01C08A
:10D100004C010894A108B1083401660C771C660C28
:10D11000771C6501CC0CDD1CCC0CDD1CC957DF4F26
:10D1200088819981C758D0408230910508F445C064
:10D130007501EE0CFF1CC501B3E0880F991FBA956D
:10D14000E1F7E80EF91EE80CF91CE016F10611F4FF
:10D150000C943D72842F6AE00E940F73682F70E078
:10D1600086EF9FEF689F9001699F300D789F300D8B
:10D170001124240F311D220F331F220F331F660F7E
:10D18000771F660F771F6E5F7F4FC901039644E0DC
:10D1900050E024E030E00FE710E00E9423450C94BB
:10D1A0003D72B6016E5F7F4FC301039644E050E0CD
:10D1B00024E030E006EA10E00BC0B6016E5F7F4F5E
:10D1C000C301039644E050E024E030E004E910E0BD
:10D1D0000E942345C757DF4F9881C958D04090FF20
:10D1E000EEC31501220C331CC50103E0880F991F03
:10D1F0000A95E1F7280E391E280C391C9401220FDC
:10D20000331F220F331FC501880F991F880F991FE5
:10D21000C957DF4FE881F981C758D040BC016E5F24
:10D220007F4FC901039644E050E024E030E030979E
:10D2300009F50FE710E00E942345F401EE0FFF1FF0
:10D24000E80DF91DEE0FFF1FEA0DFB1D21E630E092
:10D250002C0F3D1FE20FF31F8FEF808335E0831605
:10D26000910420F40894811C911C6FC308948108D8
:10D2700091086BC304EB10E00E942345D401AA0F70
:10D28000BB1FA80DB91DAA0FBB1FAA0DBB1DE1E650
:10D29000CE2ED12CCC0EDD1ECA0EDB1E81E0F60197
:10D2A0008083C957DF4F28813981C758D04021502A
:10D2B0003040C357DF4F39832883CD58D040EFE14A
:10D2C000F0E0EC0FFD1FE20FF31F2081822F6AE0D8
:10D2D0000E940F73482F90E0A816B90609F0A5C068
:10D2E000622F70E026EF3FEFA29EC001A39E900D3B
:10D2F000B29E900D1124860F971F8815990508F08E
:10D3000052C0842F90E09C01220F331FF3E0880F5E
:10D31000991FFA95E1F7280F391F261B370B21506B
:10D3200030407A2D770F770F7E5F6901C80CD91CCA
:10D3300000E0662477248AEF9FEFC89E7001C99EA3
:10D34000F00CD89EF00C1124EA0EFB1E41E650E0D2
:10D350004C0F5D1FE40EF51E122F110F110F1095CB
:10D360001DC0F701E60DF71D86E08083812F800F39
:10D37000672F44E052E0CD56DF4F7883C359D04049
:10D380000E94D8440894C108D10886E090E0680E55
:10D39000791ECD56DF4F7881C359D0400C5FC11440
:10D3A000D104F9F6ABC001976C01C818D9080A2D51
:10D3B000000F000F0E5F20E0662477247C01EE0C46
:10D3C000FF1CE80EF91EEE0CFF1CEA0CFB1CE1E64C
:10D3D000F0E0EC0FFD1FEE0EFF1E66E0462E182F4C
:10D3E000110F110F195F1CC0F701E60DF71D4082E8
:10D3F000812F820F602F44E052E0CD56DF4F28830B
:10D40000C359D0400E94D8440894C108D1084AEFBB
:10D410005FEF640E751ECD56DF4F2881C359D04093
:10D420002450C114D10401F769C0282D220F220F06
:10D430008A159B05C8F5809590952C014A0C5B1CBC
:10D440002D5F00E0EE24FF246D01C418D508E1E64D
:10D45000F0E0EC0FFD1FCE0EDF1E35E0632E909541
:10D4600081959F4F182F110F110F125018C0F60100
:10D47000EE0DFF1D6082612F600F822F42EF51E0A1
:10D48000CD56DF4F2883C359D0400E94D84408941A
:10D49000E11CF11CCD56DF4F2881C359D0400C5FF1
:10D4A000E414F50421F72AC001977C01EA18FB086F
:10D4B0002D5F00E0360115E0C12E182F110F110F5E
:10D4C0001A5F18C0F301EE0DFF1DC082612F600FBF
:10D4D000822F42EF51E0CD56DF4F2883C359D04011
:10D4E0000E94D8440894E108F108CD56DF4F288106
:10D4F000C359D0400450E114F10421F7C957DF4F5C
:10D5000028813981C758D0402230310508F446C1FE
:10D51000EFE1F0E0EC0FFD1FC357DF4F28813981A9
:10D52000CD58D040E20FF31F30812AE0832F622FC5
:10D530000E940F73482FE82EFF2406EF1FEFE09E96
:10D54000D001E19EB00DF09EB00D1124A30FB11DCE
:10D55000EDE1F0E0EC0FFD1FC957DF4F88819981A5
:10D56000C758D040E80FF91FE0818E2F0E940F733B
:10D57000582F90E0809F9001819F300D909F300D3B
:10D5800011242E0F311DA217B3071CF4EA14FB045B
:10D5900028F0A815B905E8F54517D8F58A2F880FA2
:10D5A000880F642F660F660F6E5F8D5F4AEA51E049
:10D5B0000E94D844EFE1F0E0EC0FFD1FC357DF4FAE
:10D5C00028813981CD58D040E20FF31F2081822F6E
:10D5D0006AE00E940F73682F70E086EF9FEF689FEC
:10D5E000A001699F500D789F500D1124420F511DCD
:10D5F000FA01EE0FFF1FE40FF51FEE0FFF1FE60FFE
:10D60000F71F41E650E04C0F5D1FE40FF51F81E06E
:10D61000C4C02A173B072CF4842F90E08A159B0581
:10D6200028F08A169B06E8F54517D8F58A2F880F4B
:10D63000880F642F660F660F6E5F8D5F4CEB51E0B5
:10D640000E94D844EFE1F0E0EC0FFD1FC357DF4F1D
:10D6500028813981CD58D040E20FF31F2081822FDD
:10D660006AE00E940F73682F70E086EF9FEF689F5B
:10D67000A001699F500D789F500D1124420F511D3C
:10D68000FA01EE0FFF1FE40FF51FEE0FFF1FE60F6D
:10D69000F71F41E650E04C0F5D1FE40FF51F82E0DD
:10D6A0007CC08A2F880F880F642F660F660FA21721
:10D6B000B3072CF4242F30E0A216B30628F0A815E7
:10D6C000B905B8F55417A8F56E5F8D5F4EEC51E0C3
:10D6D0000E94D844EFE1F0E0EC0FFD1FC357DF4F8D
:10D6E00028813981CD58D040E20FF31F2081822F4D
:10D6F0006AE00E940F73682F70E086EF9FEF689FCB
:10D70000A001699F500D789F500D1124420F511DAB
:10D71000FA01EE0FFF1FE40FF51FEE0FFF1FE60FDC
:10D72000F71F41E650E04C0F5D1FE40FF51F83E04B
:10D7300034C06E5F8D5F40EE51E00E94D844EFE14F
:10D74000F0E0EC0FFD1FC357DF4F28813981CD5822
:10D75000D040E20FF31F2081822F6AE00E940F73F6
:10D76000682F70E086EF9FEF689FA001699F500DC2
:10D77000789F500D1124420F511DFA01EE0FFF1F2B
:10D78000E40FF51FEE0FFF1FE60FF71F41E650E015
:10D790004C0F5D1FE40FF51F84E08083C1016AE038
:10D7A00070E00E941B738B019C01EFE1F0E0EC0F35
:10D7B000FD1FC357DF4F88819981CD58D040E80FB6
:10D7C000F91F80816AE00E940F7390E00817190723
:10D7D000E1F59AE029163104E0F0F901EE0FFF1FA0
:10D7E000E20FF31FEE0FFF1F21E630E02C0F3D1F6D
:10D7F000E20FF31FE00FF11F31978081181624F01C
:10D800000894A108B10872C032E32316310408F06D
:10D8100052C0C1016AE070E00E941B73FC01EE0F70
:10D82000FF1FE80FF91FEE0FFF1F41E650E04C0FFE
:10D830005D1FE40FF51FE00FF11F818118160CF436
:10D8400041C00894A11CB11C51C025303105D8F449
:10D85000C9010196FC01EE0FFF1FE80FF91FEE0F43
:10D86000FF1FE00FF11F81E690E08C0F9D1FE80F76
:10D87000F91F8081181624F00894811C911C36C071
:10D880002115310531F1C9010197FC01EE0FFF1F90
:10D89000E80FF91FEE0FFF1FE00FF11F21E630E048
:10D8A0002C0F3D1FE20FF31F80811816CCF0089457
:10D8B000810891081BC031E0C557DF4F3883CB5832
:10D8C000D04014C041E0C557DF4F4883CB58D0400B
:10D8D0000DC051E0C557DF4F5883CB58D04006C02C
:10D8E00081E0C557DF4F8883CB58D040C957DF4F01
:10D8F000E881F981C758D040E230F10530F1950157
:10D90000220F331FC50113E0880F991F1A95E1F705
:10D91000280F391F280D391D8F8D90E028173907E2
:10D92000A1F4C401880F991F880F991FB501660FD4
:10D93000771F660F771F6E5F7F4F039644E050E0BE
:10D9400024E030E006EA10E013C0C401880F991FFC
:10D95000880F991FB501660F771F660F771F6E5FDF
:10D960007F4F039644E050E024E030E004E910E00B
:10D970000E942345EFE1F0E0EC0FFD1FC957DF4F98
:10D9800028813981C758D040E20FF31F20822F5FD2
:10D990003F4FC957DF4F39832883C758D040C557F9
:10D9A000DF4F3881CB58D040332349F48091B50AFA
:10D9B000882329F483E06FEF41E00E945E3DC75762
:10D9C000DF4F4881C958D04043FF8AC080E090E0D3
:10D9D0000E94664B882309F094C5CE018F599F4F52
:10D9E0000E94ED4AC957DF4F88819981C758D040BE
:10D9F000009709F458C02F8D9AE0E92E822F6E2DE2
:10DA00000E940F73682F70E036EFC32E3FEFD32EC6
:10DA10006C9DC0016D9D900D7C9D900D1124820F19
:10DA2000911D880F991F880F991F660F771F660F2A
:10DA3000771F6E5F7F4F039644E050E024E030E0B4
:10DA40000FE710E00E942345C957DF4FE881F981B5
:10DA5000C758D040E230F10530F1EC0FFD1F468D84
:10DA6000842F6E2D0E940F73682F70E06C9D9001C3
:10DA70006D9D300D7C9D300D1124240F311D220F22
:10DA8000331F220F331F660F771F660F771F6E5FDE
:10DA90007F4FC901039644E050E024E030E004EBFE
:10DAA00010E00E942345C401880F991F880F991F19
:10DAB000B501660F771F660F771F6E5F7F4F039666
:10DAC00044E050E024E030E004E910E00E94234507
:10DAD00021E030E0C157DF4F39832883CF58D04051
:10DAE000C957DF4F48815981C758D04041505040F5
:10DAF000C357DF4F59834883CD58D040EFE1F0E062
:10DB0000EC0FFD1FE40FF51F90818F8D981709F022
:10DB100092C1C957DF4F88819981C758D040823060
:10DB2000910508F488C10E94313887E090E062E0F6
:10DB300070E047E45BE520E00E94954584E090E0DA
:10DB400060E170E04BE35BE520E00E949545809149
:10DB50002E0B90912F0B8C30910561F588E090E0B1
:10DB600064E070E048E15BE520E00E94954584E0D8
:10DB700090E061E170E046E25BE520E00E949545BF
:10DB800084E090E062E170E046E25BE520E00E9424
:10DB900095458AE190E061E170E041E020E00E947B
:10DBA000E7458AE190E062E170E042E020E00E9417
:10DBB000E74509C084E090E061E170E042E45BE5A4
:10DBC00020E00E94954580E090E00E945047EE24BE
:10DBD000FF24C157DF4F48805980CF58D04002C042
:10DBE000462C5C2C81E090E00E945A4580E00E9427
:10DBF00067388C01682EC12E80E00E946738482665
:10DC000059264022512282010071107044FE09C041
:10DC1000E114F10431F00894E108F108C7010E9411
:10DC2000504745FE19C080912E0B90912F0B8C30E0
:10DC3000910529F492E0E916F10490F406C08C30C5
:10DC4000910570F4E114F10459F40894E11CF11CFD
:10DC5000C7010E94504704C00115110509F468C0AE
:10DC600080912E0B90912F0B8C30910509F060C0A4
:10DC7000E1E0EE16F10419F48BE090E006C0F2E06A
:10DC8000EF16F10499F48CE090E0BE016F5F7F4FD6
:10DC90000E94514ECE010196BE01635C7F4F0E94EF
:10DCA000DE4CCE01CD960E94ED4A02C00E94313872
:10DCB00087E090E062E070E047E45BE520E00E94EE
:10DCC000954584E090E060E170E04BE35BE520E0A7
:10DCD0000E94954588E090E064E070E048E15BE5F3
:10DCE00020E00E94954584E090E061E170E046E22A
:10DCF0005BE520E00E94954584E090E062E170E001
:10DD000046E25BE520E00E9495458AE190E061E112
:10DD100070E041E020E00E94E7458AE190E062E1A6
:10DD200070E042E020E00E94E745C7010E945047B2
:10DD300040FE56CFC757DF4F59824882C958D0405E
:10DD4000E114F10409F4CEC380912E0B90912F0BB6
:10DD50008C30910550F421E0E216F10409F0C5C3BE
:10DD60007C010894E11CF11C1CC031E0E316F104B5
:10DD700009F0BBC3BDC3CE018F599F4F0E94ED4A2E
:10DD8000C157DF4F6882CF58D040C057DF4FC8829D
:10DD9000C059D04041E0C557DF4F4883CB58D040F1
:10DDA0004AC0C357DF4F88819981CD58D040B70111
:10DDB000AE01415E5F4F0E94CB4B0E94313882E042
:10DDC00090E06FE070E044E05BE520E00E94954564
:10DDD0004E2D4A508AE190E06FE070E020E00E9412
:10DDE000E7458CE390E00E945A4580E00E94673846
:10DDF00082FF87C30E94313802E010E0F8015BE047
:10DE0000E516F10419F4E85DF54F02C0EA5CF54F40
:10DE100087E090E0B801408120E00E94E7450F5F75
:10DE20001F4F0031110551F780E00E9467388130A3
:10DE30009105D1F766C3C757DF4F8881C958D040D5
:10DE400081FD09C0C557DF4F9881CB58D040992339
:10DE500011F40C945F63C957DF4FE881F981C7580B
:10DE6000D040309711F40C945F63C401880F991F60
:10DE7000880F991FB501660F771F660F771F6E5FBA
:10DE80007F4F039644E050E024E030E00EE710E0DE
:10DE90000E942345C1016AE070E00E941B732B01C0
:10DEA0003C014C015B01FC01EE0FFF1FE80FF91F65
:10DEB000EE0FFF1FE60FF71F21E630E02C0F3D1F8E
:10DEC000E20FF31F1082AC01440F551F440F551F82
:10DED0004D5F5F4FC757DF4F59834883C958D040C4
:10DEE000CB01880F991F880F991F0296C557DF4FE6
:10DEF00099838883CB58D040CA01C557DF4F6881CA
:10DF00007981CB58D04044E050E024E030E00E94DA
:10DF10002345C957DF4FE881F981C758D040E33026
:10DF2000F10598F1EDE1F0E0EC0FFD1FC957DF4F6F
:10DF300028813981C758D040E20FF31F4081842FD8
:10DF40006AE00E940F73682F70E086EF9FEF689F72
:10DF50009001699F300D789F300D1124240F311DE1
:10DF6000220F331F220F331F660F771F660F771F95
:10DF70006E5F7F4FC901039644E050E024E030E03B
:10DF800004EB10E00E9423450AC0C957DF4F4881C7
:10DF90005981C758D0404230510509F0C8C1C9570E
:10DFA000DF4F88819981C758D0400297CF56DF4F05
:10DFB00099838883C159D040EFE1F0E0EC0FFD1F59
:10DFC000E80FF91F2081822F6AE00E940F73482F0B
:10DFD00090E04816590609F0B9C0622F70E026EFAC
:10DFE0003FEF429EC001439E900D529E900D112422
:10DFF000860F971F53018615970508F060C0089497
:10E00000A108B108842F90E09C01220F331F43E048
:10E01000880F991F4A95E1F7280F391F261B370BE8
:10E02000A20EB31E88249924222433246301CC0C2D
:10E03000DD1CC60CD71CCC0CDD1CC40CD51C8AEF17
:10E040009FEFA89E9001A99E300DB89E300D11241F
:10E05000C20ED31EE1E6F0E0EC0FFD1FCE0EDF1E78
:10E060007301EA18FB08EE0CFF1CEE0CFF1C089471
:10E07000E108F1081CC0F601E20DF31D1082C70192
:10E08000880D991DC557DF4F68817981CB58D040E5
:10E0900044E050E024E030E00EE710E00E94234529
:10E0A0000894A108B10826E030E0220E331E44E0B7
:10E0B00050E0840E951EA114B104E9F6E7C1A094C6
:10E0C000B094A80EB91E8824992422243324750103
:10E0D000E60CF71C6701CC0CDD1CCE0CDF1CCC0C55
:10E0E000DD1CC40CD51C81E690E08C0F9D1FC80E72
:10E0F000D91EEE0CFF1CEE0CFF1CE7E0F0E0EE0E6C
:10E10000FF1E1CC0F601E20DF31D1082C701880D31
:10E11000991DC557DF4F68817981CB58D04044E0C5
:10E1200050E024E030E00EE710E00E942345089420
:10E13000A108B1082AEF3FEF220E331E4CEF5FEF2C
:10E14000840E951EA114B104E9F6A0C184159505AD
:10E1500008F047C052010894A108B108A81AB90AEA
:10E1600022243324882499247301EE0CFF1CE60C2E
:10E17000F71CEE0CFF1CE40CF51CEA18FB0881E60A
:10E1800090E08C0F9D1FE80EF91E6201CA18DB0893
:10E19000CC0CDD1CCC0CDD1CEEEFFFEFCE0EDF1E39
:10E1A00018C0F701E80DF91D1082B601620D731D4C
:10E1B000C757DF4F88819981C958D04044E050E06B
:10E1C00024E030E00EE710E00E9423450894811C13
:10E1D000911C24E030E0220E331E8A149B0409F7C0
:10E1E00055C16201C094D094C80ED91E88249924C8
:10E1F0007301EE0CFF1CE60CF71CEE0CFF1CE40C8C
:10E20000F51C41E650E04C0F5D1FE40EF51E560173
:10E21000A40CB51CAA0CBB1CAA0CBB1C86E090E08D
:10E22000A80EB91E18C0F701EC0DFD1D1082B50136
:10E23000680D791DC757DF4F88819981C958D04033
:10E2400044E050E024E030E00EE710E00E94234577
:10E250000894C108D108ECEFFFEF8E0E9F1EC11489
:10E26000D10409F713C1C1016AE070E00E941B7379
:10E27000DB01AC01C957DF4FE881F981C758D040B5
:10E28000EC0FFD1F848D622F0E940F7390E0A81782
:10E29000B90701F5FAE02F163104B8F0FA01EE0FD4
:10E2A000FF1FE40FF51FEE0FFF1F21E630E02C0FDC
:10E2B0003D1FE20FF31FEA0FFB1F319780811816F5
:10E2C00024F00894A108B10835C058010894A11C95
:10E2D000B11C30C04530510530F5CA010196FC0132
:10E2E000EE0FFF1FE80FF91FEE0FFF1FEA0FFB1FD6
:10E2F00041E650E04C0F5D1FE40FF51F80811816BA
:10E3000094F00DC0C957DF4F88819981C758D0401C
:10E310008230910579F495E08916910420F40894EF
:10E32000811C911C07C008948108910803C0AFEFBD
:10E330002A2E312C4F8D842F6AE00E940F73682F94
:10E3400070E086EF9FEF689F9001699F300D789F86
:10E35000300D1124240F311D220F331F220F331FC4
:10E36000660F771F660F771F6E5F7F4FC901039699
:10E3700044E050E024E030E00FE710E00E94234545
:10E38000A401440F551F440F551FB501660F771F99
:10E39000660F771FC957DF4FE881F981C758D04012
:10E3A0006E5F7F4FE230F105D8F09501220F331FE9
:10E3B000C501F3E0880F991FFA95E1F7280F391F7F
:10E3C000280D391D8F8D90E02817390749F4CA01AF
:10E3D000039644E050E024E030E006EA10E008C094
:10E3E000CA01039644E050E024E030E004E910E084
:10E3F0000E942345EFE1F0E0EC0FFD1FC357DF4F14
:10E4000028813981CD58D040E20FF31F1082C957BF
:10E41000DF4F48815981C758D04041505040C957BB
:10E42000DF4F59834883C758D0408091B50A88236D
:10E4300011F00C945A6384E06FEF41E00E945E3D5E
:10E440000C945A638F8D90E0E816F90611F00C9445
:10E45000C4640C94B8648F8D90E0E816F90611F04E
:10E460000C9412660C9406668F8D90E0E816F906FF
:10E4700011F00C947B670C946F678F8D90E0E81619
:10E48000F90611F00C94DD680C94D168EFE1F0E02E
:10E49000EC0FFD1FCF56DF4F88819981C159D040C5
:10E4A000E80FF91F8081282E33242AE0622F0E9472
:10E4B0000F73082F10E086EF9FEF089F4001099F20
:10E4C000900C189F900C1124820C931C5801C95772
:10E4D000DF4FE881F981C758D040E330F10508F0FB
:10E4E000C2CE10CF8FEF9FEF05C08CE090E002C04E
:10E4F0008BE090E0FFEF8F3F9F0709F43CCC7C015D
:10E5000050CCCD56DF4FE2E10C949B730E943B460A
:10E5100085E391E40E943E3A80EB0E94EE3D86E165
:10E5200092E00E945B3886EC0E94583886E19EE3B8
:10E530000E942C380E94A65202E010E08091D50A79
:10E5400090E00E9416740E9411748093D50A86EBA5
:10E550009AE00E940D390E94724A009721F08130A2
:10E56000910561F726C00E94FD4982309105C1F0F6
:10E570008330910534F4009759F081309105F1F61C
:10E580000AC08330910579F084309105B9F60EC048
:10E5900081E090E002C082E090E00E946162CECF14
:10E5A0000E946048CBCF0E94FE62C8CF0E940D53EC
:10E5B000C5CF0E94117460912E0B70912F0B0E9499
:10E5C0001B73EC0121960E941174B8010E942F73F5
:10E5D00061E0009709F460E0CE010E943062AECFA6
:10E5E000629FD001739FF001829FE00DF11D649F37
:10E5F000E00DF11D929FF00D839FF00D749FF00DC3
:10E60000659FF00D9927729FB00DE11DF91F639F63
:10E61000B00DE11DF91FBD01CF0111240895991B13
:10E6200079E004C0991F961708F0961B881F7A9509
:10E63000C9F780950895AA1BBB1B51E107C0AA1F0B
:10E64000BB1FA617B70710F0A61BB70B881F991F93
:10E650005A95A9F780959095BC01CD01089597FB37
:10E66000092E07260AD077FD04D0E5DF06D000206A
:10E670001AF4709561957F4F0895F6F790958195FE
:10E680009F4F0895A1E21A2EAA1BBB1BFD010DC0CE
:10E69000AA1FBB1FEE1FFF1FA217B307E407F50752
:10E6A00020F0A21BB30BE40BF50B661F771F881F2E
:10E6B000991F1A9469F760957095809590959B01C4
:10E6C000AC01BD01CF01089597FB092E05260ED0A0
:10E6D00057FD04D0D7DF0AD0001C38F45095409580
:10E6E000309521953F4F4F4F5F4F0895F6F7909526
:10E6F0008095709561957F4F8F4F9F4F08952F9212
:10E700003F924F925F926F927F928F929F92AF92C1
:10E71000BF92CF92DF92EF92FF920F931F93CF930E
:10E72000DF93CDB7DEB7CA1BDB0B0FB6F894DEBFA5
:10E730000FBECDBF09942A88398848885F846E84CB
:10E740007D848C849B84AA84B984C884DF80EE8015
:10E75000FD800C811B81AA81B981CE0FD11D0FB61E
:10E76000F894DEBF0FBECDBFED010895EE0FFF1F81
:10E770000590F491E02D09948F929F92AF92BF92F1
:10E78000CF92DF92EF92FF92CF93DF93EC018881DB
:10E790009981AA81BB810097A105B10521F484E28A
:10E7A00099EDABE5B7E0BC01CD012DE133EF41E0E0
:10E7B00050E00E94647349015A0127EA31E440E0C5
:10E7C00050E00E94F0726B017C01C501B4012CEE97
:10E7D00034EF4FEF5FEF0E94F072DC01CB01C80E07
:10E7E000D91EEA1EFB1EF7FE08C08FEF9FEFAFEFAA
:10E7F000BFE7C80ED91EEA1EFB1EC882D982EA8274
:10E80000FB82C6019F77DF91CF91FF90EF90DF9061
:10E81000CF90BF90AF909F908F9008950E94BC734F
:10E82000089582E292E00E94BC730895A0E0B0E0F7
:10E830008093220290932302A0932402B093250296
:10E84000089511F40EF44DC03EC05DD0D0F399236D
:10E85000D9F3CEF39F57550B87FF46D00024A0E68F
:10E8600040EA900180585695979528F4805C660F91
:10E87000771F881F20F026173707480730F4621BE0
:10E88000730B840B202931294A2BA69517940794E2
:10E89000202531254A2758F7660F771F881F20F05B
:10E8A00026173707480730F4620B730B840B200DD3
:10E8B000311D411DA09581F7B901842F9158880F12
:10E8C0009695879508959F3F31F0915020F4879554
:10E8D00077956795B795880F911D9695879597F9C8
:10E8E00008959FEF80EC089591505040660F771F78
:10E8F000881FD2F7089557FD9058440F551F59F0BF
:10E900005F3F71F04795880F97FB991F61F09F3F1C
:10E9100079F087950895121613061406551FF2CF45
:10E920004695F1DF08C0161617061806991FF1CF95
:0EE9300086957105610508940895F894FFCF4F
:10E93E0001030100A058AE58BC58CA58D858E65822
:10E94E00F458025910592A0A380A00000000000033
:10E95E000000000102020303030304040404040480
:10E96E00040405050505050505050505050505054B
:10E97E00050506060606060606060606060606062B
:10E98E000606060606060606060606060606060619
:10E99E0006060707070707070707070707070707FB
:10E9AE0007070707070707070707070707070707E9
:10E9BE0007070707070707070707070707070707D9
:10E9CE0007070707070707070707070707070707C9
:10E9DE0007070808080808080808080808080808AB
:10E9EE000808080808080808080808080808080899
:10E9FE000808080808080808080808080808080889
:10EA0E000808080808080808080808080808080878
:10EA1E000808080808080808080808080808080868
:10EA2E000808080808080808080808080808080858
:10EA3E000808080808080808080808080808080848
:10EA4E000808080808080808080808080808080838
:06EA5E00080801000000A1
:00000001FF
